:020000040800F2
:100000004090002029020008DD6300085D550008CB
:100010007D6200083D1F0008E9780008000000002C
:10002000000000000000000000000000816B0008DC
:10003000892B00080000000041660008E96B0008F9
:10004000430200084302000843020008430200087C
:1000500043020008430200088D2B000843020008F9
:100060004302000843020008992B000843020008DD
:100070003D2A00084302000843020008430200082A
:10008000430200084302000843020008430200083C
:10009000411F0008511F000843020008A52B00085B
:1000A000430200084302000843020008430200081C
:1000B000430200084302000843020008430200080C
:1000C00043020008430200084302000843020008FC
:1000D00043020008A978000843020008B978000824
:1000E00043020008430200084302000843020008DC
:1000F00043020008430200084302000843020008CC
:1001000043020008430200084302000843020008BB
:1001100043020008430200084302000843020008AB
:10012000430200084D2A00085D2A00086D2A0008D5
:10013000430200084302000843020008430200088B
:10014000611F0008711F00084302000843020008F5
:100150007D2A00088D2A000843020008D178000893
:10016000430200084302000843020008430200085B
:100170004302000843020008430200080000000098
:10018000430200084302000800F002F800F03CF8C7
:100190000AA090E8000C82448344AAF10107DA45E2
:1001A00001D100F031F8AFF2090EBAE80F0013F0F8
:1001B000010F18BFFB1A43F001031847D0C7000016
:1001C000F0C70000103A24BF78C878C1FAD85207A7
:1001D00024BF30C830C144BF04680C6070470000C1
:1001E0000023002400250026103A28BF78C1FBD840
:1001F000520728BF30C148BF0B6070471FB50CF0D5
:100200006EFA1FBD10B510BD00F062F91146FFF780
:10021000F5FF07F0F5FC00F080F903B4FFF7F2FFFB
:1002200003BC00F083F900000948804709480047F3
:10023000FEE7FEE7FEE7FEE7FEE7FEE7FEE7FEE796
:10024000FEE7FEE704480549054A064B70470000F3
:10025000A16C000889010008406000204090002047
:10026000407000204070002053EA020C00F06980CA
:100270002DE9F04B4FF00006002B1FBFB3FA83F5BA
:1002800003FA05F424FA05F65E4012BF1643B2FAEB
:1002900082F502FA05F4C5F120051EBF22FA05FC1D
:1002A00044EA0C04203556EA044C4FEA144418BFC3
:1002B000641C4FF000084FF00009904271EB030CF2
:1002C00039D3002919BFB1FA81F701FA07F6B0FA5C
:1002D00080F700FA07F6C7F120071EBF20FA07FCD7
:1002E00046EA0C062037B6FBF4FCA7EB0507103FE7
:1002F00007F01F0BCBF120062CFA06F60CFA0BFBCD
:1003000044BFB3460026202FA4BF5E464FF0000B2B
:100310005BEA060C08BF4FF0010B19EB0B0948EB29
:100320000608ABFB027C06FB02CC0BFB03CCC01B1C
:1003300071EB0C01C1E70B46024641464846BDE859
:10034000F08B13B5084318BF4FF0FF300146AFF3F1
:100350000080BDE81C407047032A40F2308010F056
:10036000030C00F0158011F8013BBCF1020F624450
:1003700098BF11F801CB00F8013B38BF11F8013BE1
:10038000A2F1040298BF00F801CB38BF00F8013B8E
:1003900011F0030300F06280083AC0F0088051F8C1
:1003A000043B083A51F804CBA0E80810F5E7121D09
:1003B0005CBF51F8043B40F8043BAFF30080D20728
:1003C00024BF11F8013B11F801CB48BF11F8012BF4
:1003D00024BF00F8013B00F801CB48BF00F8012B17
:1003E000704702F0FF0343EA032242EA024200F0B0
:1003F00002B84FF0000200B51346944696462039E5
:1004000022BFA0E80C50A0E80C50B1F12001BFF4CD
:10041000F7AF090728BFA0E80C5048BF0CC05DF833
:1004200004EB890028BF40F8042B08BF704748BF81
:1004300020F8022B11F0804F18BF00F8012B7047F5
:1004400070477047704710B500F03AF8006810BD6B
:1004500010B5044600F034F8046010BD10B5203A21
:10046000C0F00B80B1E81850A0E81850B1E818505F
:10047000A0E81850203ABFF4F5AF5FEA027C24BF31
:10048000B1E81850A0E8185044BF18C918C0BDE81A
:1004900010405FEA827C24BF51F8043B40F8043BE3
:1004A00008BF7047D20728BF31F8023B48BF11F898
:1004B000012B28BF20F8023B48BF00F8012B7047F2
:1004C00000487047080100200048704708010020DC
:1004D0007546FFF7F9FFAE4605006946534620F022
:1004E0000700854618B020B5FFF7ACFEBDE82040F8
:1004F0004FF000064FF000074FF000084FF0000BE0
:10050000AC46ACE8C009ACE8C009ACE8C009ACE84E
:10051000C00921F007018D46704710B50446AFF3BE
:1005200000802046BDE81040FFF777BE0149182043
:10053000ABBEFEE72600020070470000B0B52DED0F
:10054000028B044600284FF0FF0061D00D460029C1
:100550005ED095ED000A95ED011A95ED022A95ED14
:10056000033A20EE010A22EE033A21EE011A22EEAE
:10057000022A31EE021A30EE030A31EE011AB7EE0A
:10058000008A30EE000A78EE410A0AF0B9FCB0EEBB
:10059000401A95ED000A95ED012A95ED023A95ED88
:1005A000034A20EE030A24EE022A30EE420A30EE1D
:1005B000000AB0EEC02AB4EE482AF1EE10FA84ED3B
:1005C000011A02DA0AF098F901E007F0BFFA84EDA7
:1005D000020A95ED000A95ED011A95ED032A95EDB5
:1005E000023A20EE020A21EE031A30EE010A23EE4F
:1005F000031A22EE022A32EE011A31EE011A30EE0F
:10060000000A78EE410A0AF07BFC002084ED000A23
:1006100040B2BDEC028BB0BD70B52DED028B002851
:100620004FD0B7EE001A81EE000A0D4604464FF097
:100630007E51002D80ED040A4FF00000C4E9001047
:10064000A060E06000F09F80D5E900600BF07CFFC7
:1006500041EC180B30460BF077FF41EC110BB0EE7C
:10066000480AF0EE680A0AF04BFB51EC100B0BF055
:10067000CBF895ED000AB5EE400AF1EE10FA22D162
:1006800095ED010AB5EE400AF1EE10FA1BD195ED99
:10069000020AB5EE400AF1EE10FA14D140F2C5603C
:1006A000C3F64D7044F62D214AF2564244F2AD7322
:1006B000C3F60D41CBF63932C3F619730FC40020CF
:1006C00061E0FF205FE09FED321A00EE100AB4EE09
:1006D000410AF1EE10FA1EDCB5EE400AF1EE10FA16
:1006E00019DB9FED2C2AB4EE420AF1EE10FA25DC5C
:1006F000B4EE410AF1EE10FA20DB9FED271AB4EEBA
:10070000410AF1EE10FA2CDCB4EE420AF1EE10FAD6
:1007100027DB002037E045F66E10C3F67F7045F208
:100720000C3148F6AB0249F28553C3F6B011CBF653
:10073000BB32C3F697530FC4002024E040F2C560DB
:10074000C3F64D7044F62D214AF2564244F2AD7381
:10075000C3F60D41CBF63932C3F619730FC400202E
:1007600011E040F2C560C3F64D7044F62D214AF207
:10077000564244F2AD73C3F60D41CBF63932C3F69F
:1007800019730FC4002040B2BDEC028B70BD00BFD6
:10079000DB0FC9BFDB0F49C00000B4C2B0B52DEDFF
:1007A000108B8EB0044600284FF0FF0018BF0029C0
:1007B00004D140B20EB0BDEC108BB0BD002AF8D011
:1007C00040F204054EF69E70C2F20005C3F62750B3
:1007D0002860C3B193ED00EA93ED01FAD3ED028AEC
:1007E000B5EE40EAF1EE10FA11D1B5EE40FAF1EEB5
:1007F00010FA0CD1F5EE408AF1EE10FA07D120463E
:1008000000F094FAD5E7204600F090FAD1E792ED97
:10081000000A92ED011A94ED014A94ED025A92ED0C
:10082000022A94ED036A94ED003A24EE407A61EED8
:10083000050A37EE607A62EE060A37EE607A60EEFD
:10084000030A62EE051A71EEA00A61EE061A70EE56
:10085000E10A61EE031A62EE042A22EE032A21EE77
:10086000041A91ED00DA71EEE21A20EE066A31EE1A
:10087000021A20EE050A36EE216AD1ED019AD1ED79
:1008800002AA31EE400AB6EE001AB5EE40DA27EEC3
:10089000015A60EE810A26EE017AF1EE10FA20EE9E
:1008A000016A0AD1F5EE409AF1EE10FA05D1F5EEA3
:1008B00040AAF1EE10FA00F0EC812DEE0D0A29EEBF
:1008C000A91A30EE010A2AEEAA1A30EE010A8DEDBD
:1008D0000D6A8DED0C7ACDED0B0A8DED0A5A04F000
:1008E0003FFE2DEE001A8DED071A29EE801A2AEE32
:1008F000800A8DED081A8DED090A2EEE0E0A2FEEF4
:100900000F1A30EE010A28EEA81A30EE010A04F0A0
:1009100027FE94ED001A6EEE00DA6FEE00AA94ED59
:10092000034A31EE01EA68EE808A94ED012A94EDE3
:10093000023A2AEE8E6A61EE01EA8DED026A28EE35
:100940008E0A2DEEAE5A26EE046A62EE02BA35EE3B
:10095000465A20EE036A36EE055A2DEEAB6A32EEA9
:1009600002FA36EE055A2AEE8F6A23EE066A36EE52
:10097000055A28EE8F6A26EE046A63EE03FA36EE15
:10098000055A2DEEAF6A24EE048A35EE465A2DEE56
:10099000886A2DEE8E9A35EE465A29EE046A2AEEC2
:1009A000AE7A37EE066A22EE000A2DEE8FAA36EEF8
:1009B000400A23EE0A6A36EE000A2AEEAB6A30EEEF
:1009C000460A2AEEAF6A73EE039A36EE000A28EE64
:1009D000A96A24EE066A36EE000A2AEE886A30EE2C
:1009E000460A25EE055A20EE000A35EE000A21EEF1
:1009F00002BA21EE035A21EE041A8DED051A22EEF9
:100A0000031A8DED031A23EE041A8DED041A34EE49
:100A1000041A8DED015A22EE04CA6EEE03CA8DED62
:100A2000061A29EE84DA04F09BFD94ED013A94ED68
:100A3000022A9DED021A29EE024A21EE031A31EE36
:100A4000444A94ED031A28EEAE5A35EE044A2AEED3
:100A5000015A35EE044A28EEAB5AF7EE001A34EE8E
:100A6000454A2AEEA95A81EE800A25EE015A35EE52
:100A7000044A28EEAF5A34EE454A28EE885A75EEFD
:100A8000042A3CEE0C4A9DED075A34EE6C4A34EED3
:100A9000454A3BEE0B5A9DED086A35EE0D5A35EE90
:100AA000465A2FEE056A29EE847AF6EE007A76EE43
:100AB000470A37EEEF6A36EE486A9DED018A20EE6E
:100AC000066A3CEE487A27EE227A36EE076A36EE60
:100AD0006D7A22EE226A66EE073A70EEE33ADDEDB9
:100AE000050ADDED034A60EE015A74EEE00ADDED21
:100AF000044A60EE200A7BEE244A64EEA24A70EEBD
:100B0000A40A63EE224A70EEEA0A74EEE56A66EE23
:100B1000A06A77EEEB7A76EEA33A78EE0C6A77EE7F
:100B2000EF7A60EE266A67EEA27A76EEA76A76EE34
:100B3000E86A60EE027ADDED068A27EEA68A38EED4
:100B400023CA68EE843A2EEE058A78EE233A3BEE0D
:100B5000AB8A71EEC81A3FEEAF8A71EEC81A9DEDEE
:100B6000098A21EE22AA71EEC81AB1EE008A23EE9C
:100B7000089A21EE899A73EEC93A94ED009A2AEE0A
:100B800007BA73EE8B3A29EE22BA77EE8B7A67EECC
:100B9000A07A72EEA22A77EEA33A63EE227A75EE7D
:100BA000E75A65EEA65A35EEA3DA68EE853A6EEEA0
:100BB000045A73EEE53A62EE085A65EEA11A73EE36
:100BC000E11AF8EE003A60EE233A62EE235A75EE2F
:100BD000CB5A65EE875A20EE033A71EEA51A73EEF2
:100BE0000A5A20EE090A22EE222A65EEA05A30EEB9
:100BF000422A75EEA11A22EE262A23EE811A32EE3F
:100C0000218A2FEE042A29EE854A31EE241A34EE89
:100C1000022A21EE071A36EE400A32EE011A20EEC1
:100C2000200A30EE010A23EE261A31EE009A2CEE4D
:100C30000C0A2DEE0D1A30EE010A28EE081A31EEDC
:100C4000000A29EE091A31EE000A04F089FC95ED3C
:100C5000004A9DED0A5A20EE0C1ADDED0B0A20EE3B
:100C60000D2A24EE011A9DED0C7A9DED0D6A20EE01
:100C7000083A20EE090A35EE415A24EE021A70EEC7
:100C8000C10A24EE031A24EE000A37EE417A36EE4A
:100C9000406A94ED043A94ED000A94ED011A25EEB1
:100CA000035A94ED022A30EE050A20EE835A94EDA1
:100CB000034A35EE011A27EE035A35EE022A26EED4
:100CC000033A84ED000A84ED011A20EE000A21EEB9
:100CD000011A33EE043A30EE010A22EE021A30EE27
:100CE000010A23EE031A30EE010A84ED022A84ED94
:100CF000033A04F035FC94ED001A94ED012A94EDCA
:100D0000023A94ED034A20EE011A20EE022A20EE68
:100D1000033A20EE040A002084ED001A84ED012A33
:100D200084ED023A84ED030A43E50000B0B52DEDF1
:100D3000108B044600284FF0FF0018BF002900F078
:100D40006981002A00F0668140F2040542F6023013
:100D5000C2F20005C3F60750286092ED000A92ED3A
:100D6000011A94ED014A94ED025A92ED022A94ED93
:100D7000036A94ED003A24EE407A61EE050A37EEFC
:100D8000607A62EE060A37EE607A60EE030A62EE7F
:100D9000051A71EEA00A61EE061A70EEE10A61EE24
:100DA000031A62EE042A22EE032A21EE041A91EDC0
:100DB00000CA71EEE21A20EE066A31EE021A20EE47
:100DC000050A36EE216A91ED01DA91ED02EA31EE83
:100DD000400AB6EE001AB5EE40CA27EE01BA20EE80
:100DE00081AA26EE019AF1EE10FA20EE018A0AD1CC
:100DF000B5EE40DAF1EE10FA05D1B5EE40EAF1EECB
:100E000010FA00F0BC802CEE0C0A2DEE0D1A30EE1C
:100E1000010A2EEE0E1A30EE010A04F0A1FB94ED49
:100E2000003A94ED025AF1EE001A2CEE001A94EDFD
:100E3000014A75EE050A63EE212A65EE053A62EE77
:100E4000A34A61EE205A74EEA54A64EE045A2DEED0
:100E5000002A94ED036A34EE047A62EEA52A72EE5B
:100E6000A42A62EE074A32EEE4CA76EE062A64EE5F
:100E7000214A66EE066A64EEA67A21EE22DA77EE61
:100E8000CD7A23EE03DA2DEE21DA2EEE000A24EEDF
:100E90000DEA33EE033A7EEE277A22EE03EA77EE8E
:100EA000CE7AB2EE00EA24EE0E4A77EEE47A24EE31
:100EB00025FA7FEE277A24EE234A34EE274A60EEA5
:100EC000244A34EE84FA2DEE054A21EE033A33EE3D
:100ED000043A25EE0E4A25EE215A65EE264A33EEF7
:100EE000243A62EE222A33EE623A33EE453A65EE58
:100EF000842A32EE833A24EE234A34EE033A20EE7B
:100F0000050A30EE03DA21EE070A25EEA11A21EEDA
:100F1000061A31EE400A23EEA11A26EE011A30EE2F
:100F2000010A22EE201A30EE41EA2CEE0C0A2FEED6
:100F30000F1A30EE010A2DEE0D1A31EE000A2EEED8
:100F40000E1A31EE000A04F00BFB95ED004A20EE7C
:100F50000C1A20EE0F2A24EE011A20EE0D3A20EE94
:100F60000E0A3BEE41BA24EE021A3AEE41AA24EEF2
:100F7000031A24EE000A39EE419A38EE408A94EDC5
:100F8000043A94ED000A94ED011A2BEE035A94ED05
:100F9000022A30EE050A2AEE035A94ED034A35EE92
:100FA000011A29EE035A35EE022A28EE033A84ED9F
:100FB000000A84ED011A20EE000A21EE011A33EE38
:100FC000043A30EE010A22EE021A30EE010A23EE54
:100FD000031A30EE010A84ED022A84ED033A04F08C
:100FE000BFFA94ED001A94ED012A94ED023A94EDC3
:100FF000034A20EE011A20EE022A20EE033A20EEE8
:10100000040A002084ED001A84ED012A84ED023ADE
:1010100084ED030A40B2BDEC108BB0BDB1EE601A96
:10102000B4EE600AF1EE10FAB4EE401AC8BFB0EEAA
:10103000600AF1EE10FAC8BFB0EE410A7047000036
:1010400080B541F24040C2F200000068082107F07C
:1010500039F880BD80B540F2D822C2F200020020EB
:101060001221132300F086F9002080BD80B50220F4
:1010700001214FF0FF3207F065F880BD9FED010AB6
:10108000704700BF0000C84380B541F24040C2F243
:1010900000000068102107F015F880BD80B540F20F
:1010A000D820C2F20000C21D01200221062300F058
:1010B00061F9002080BD000080B5042001214FF0BF
:1010C000FF3207F03FF880BDF0B581B000284FF047
:1010D000FE0700F097800C46002900F0938040F650
:1010E000D556C2F200060546307808B1FD2789E0E2
:1010F00007F086F841F24041C2F200010028086082
:101100007BD000207E21B622EC6200F08FF9012016
:101110001421B62200F08AF91E2000F073FE002090
:101120001E2100F04DF90020002100F049F91E2891
:1011300065D101200021012400F042F90F2860D17F
:10114000032000F04FFD042000F04CFD41F2253259
:10115000C0F6000200200121002700F029FE41F224
:101160004101C0F60001032000F07EFD41F289013B
:10117000C0F60001042000F077FD00204021AA22E3
:1011800000F054F900204121012200F04FF9002025
:101190005321082200F04AF900205821042200F0CF
:1011A00045F900207D21042200F040F9322000F0B2
:1011B00029FE01200F21012200F038F90120102121
:1011C000032200F033F901201621002200F02EF94D
:1011D00001201821012200F029F901201521802287
:1011E00000F024F90A2000F00DFE0320347000F016
:1011F0000FFD042000F00CFD04E0FE2702E0FC27B8
:1012000000E0FC2778B201B0F0BD0000002841D01A
:1012100040F2D821C2F20001B1F901209FED1F3A3E
:1012200000EE102AB8EEC00A80EE030AB1F90330CE
:10123000B1F905C001EE103A02EE10CAB8EEC11ABB
:10124000B8EEC22A81EE031A82EE032A4FF600039B
:10125000CFF6FF7380ED040A4A7C897CD20042EA13
:1012600051120021B1EB922F80ED051A80ED062A74
:1012700018BF1A4300EE102AB8EEC00AB4EE001AE6
:1012800020EE010AB3EE071A30EE010A80ED0A0AD9
:1012900048B27047FE2148B2704700BF00A0AA457F
:1012A000C0B340F2D821C2F20001B1F90720B1F970
:1012B0000930B1F90B1000EE102A01EE103A9FED43
:1012C000172A03EE101AB8EEC00AB8EEC11AB8EE2B
:1012D000C33A80EE020A81EE021A83EE022A9FEDE3
:1012E000103AC16A91ED014A91ED025A20EE030ACB
:1012F00021EE031A22EE032A91ED003A31EE441A50
:1013000030EE430A32EE452A80ED070A80ED081AD6
:1013100080ED092A6FF00100704700BF6F12034291
:1013200035FA8E3C10B5012000F088FC41F24044B3
:10133000C2F2000438B90120012100F0BBFC206892
:10134000022106F0BFFE022000F078FC002818BF42
:1013500010BD0220012100F0ADFC2068042106F040
:10136000B1FE10BD80B5182001214FF0FF3206F00C
:10137000E9FE80BD002A08BF704770B51C461546BF
:101380000E4618B1012805D1022000E001200021FD
:1013900000F090FC40F2EB2146F08000C2F2000128
:1013A000087000200122002300F012FD00202946D1
:1013B0002246012300F0E2FCBDE8704070470000C7
:1013C000F0B581B0044601200D46012600F01AFD5B
:1013D00014B1012C04D102263046002100F06AFC31
:1013E00040F2EB26C2F2000645F08000374607F8CF
:1013F000010B0020314601220023012500F0E8FC0A
:10140000002031460222002300F0B8FC34B1012C48
:1014100009D140F2EB27C2F200070225284601213C
:1014200000F048FC3878C0B201B0F0BDB0B5044659
:1014300001F07F0040F2EB21C2F2000108700120B0
:101440004A70012500F0DEFC14B1012C04D1022504
:101450002846002100F02EFC40F2EB21C2F20001F0
:1014600000200222002300F0B3FC24B1012C18BF9D
:10147000B0BD022000E00120012100F01BFCB0BD46
:101480002DE9F04381B041F27838C2F200080646F7
:10149000D8F8000014460D466421002A08BF0A242B
:1014A00006F07AFD08B1FB242FE041F27439C2F254
:1014B0000009D9F8000000E0006930B10178B142BC
:1014C000FAD14168A942F7D11AE0142000F00AFCD1
:1014D00088B1074620461C21002206F0B3FCB86004
:1014E00058B1D9F800003C7300243E707D6038612B
:1014F000C9F8007005E0FE2403E0384600F06EFBFA
:10150000FF24D8F8000006F0BDFD60B201B0BDE8D0
:10151000F08300007047000041F27432C2F2000212
:10152000126800E01269002A04BF00207047137897
:101530008342F7D153688B42F4D190687047000022
:10154000D0E90212081FB0FA80F14FF0020008BF84
:101550000320022A18BF48097047000040F6A8126D
:1015600040F68011C2F200020128C2F2000118BF49
:101570000022002818BF1146012888BF0021084614
:10158000704700002DE9F041154640F6D452C2F2F2
:1015900000021278012A11D1A5B141F27838C2F2C5
:1015A00000080746D8F800000E4664211C4606F0E5
:1015B000F3FC58B1FB2040B2BDE8F081FD2040B201
:1015C000BDE8F081FE2040B2BDE8F08138463146EA
:1015D000FFF7A2FFD8F800100646084606F052FDB5
:1015E00066B1304629460022234606F0E7FB002874
:1015F00018BF4FF0FF3040B2BDE8F081FC2040B290
:10160000BDE8F0812DE9F0478AB040F6D457C2F228
:101610000007387808B1FD248AE040F26810C2F271
:1016200000006821FEF7E5FE002400BFE0B200F0F4
:101630003BFA0134012CF9D040F6885041F21551A3
:10164000C2F20000C0F6000101600020002406F094
:10165000CDFC41F27831C2F200010028086066D06A
:10166000E8464FF001094046282187F80090FEF730
:10167000C0FE40F68016C2F200064FF00E0A304659
:101680004146CDE90244CDE90799CDF824A0049460
:1016900001F0F0FA304601F0B1FE41F2B172C0F64D
:1016A00000020020062100F051F841F64525C0F661
:1016B0000005002000212A4600F048F80020012102
:1016C0002A4600F043F8002002212A4600F03EF8A6
:1016D0003046032101F070FA40F6A816C2F2000667
:1016E00030464146CDE9049A01F0C4FA304601F093
:1016F00085FE41F67502C0F600020120082100F0C7
:1017000025F8012000212A4600F020F801200121BF
:101710002A4600F01BF8012002212A4600F016F8A4
:101720003046112101F048FA87F8009000E0FF24CC
:1017300060B20AB0BDE8F08780B540F68852C2F2C8
:1017400000021268002A18BF904780BD40F6D453AB
:10175000C2F200031B78012B1EBFFD2358B2704755
:101760003AB101284FF0FF0398BF0C2904D958B2B1
:101770007047FE2358B2704740F2681CC2F2000C5A
:10178000342310FB03C0002340F8212058B27047D7
:1017900080B540F6D453C2F200031B78012B03D16D
:1017A000FFF76EFE40B280BDFD2040B280BD00005C
:1017B0002DE9F04F93B003A80D3001904FF0000ACF
:1017C0000CAE002005E000BF0298002800F10100E7
:1017D0004CD15FFA80FB02905846FFF7BFFE00280D
:1017E000F2D0044609E000BF02F078F909903846CB
:1017F00003A90022002306F075FB2046002101F01A
:10180000BBFA0028E0D02046002132460AAB01F0A6
:10181000C3FA0028F1D10E980028304618BF0430D2
:1018200005683046FFF78CFE804628464146FFF7A4
:1018300083FF814658464946FFF76EFE0028DCD0FC
:101840000746DDE90F02CDF80CA00028CDE908AA73
:10185000CDE906AA8DF80C80CDE904598DF8182041
:10186000C2D101980AA9FEF777FDBDE713B0BDE824
:10187000F08F00002DE9F04F93B003A80D300190D8
:101880004FF0000A0CAE002005E000BF02980028CF
:1018900000F101004CD15FFA80FB02905846FFF73F
:1018A0005DFE0028F2D0044609E000BF02F016F900
:1018B0000990384603A90022002306F013FB2046B6
:1018C000012101F059FA0028E0D0204601213246DA
:1018D0000AAB01F061FA0028F1D10E9800283046D9
:1018E00018BF043005683046FFF72AFE80462846B8
:1018F0004146FFF721FF814658464946FFF70CFE57
:101900000028DCD00746DDE90F02CDF80CA0002846
:10191000CDE908AACDE906AA8DF80C80CDE90459D5
:101920008DF81820C2D101980AA9FEF715FDBDE770
:1019300013B0BDE8F08F00002DE9F04389B01746E1
:1019400040F6D452C2F200021278012A04D10446B1
:10195000012806D9FF2000E0FD2040B209B0BDE813
:10196000F08301F0FE001D460E46022802D00DB99C
:10197000FE20F2E7DDF84080B8F1080F01D9FF2022
:10198000EBE72046FFF7EAFD98B181460020032EE1
:101990000890CDE90600CDE90400CDE902000190F0
:1019A00009D8DFE806F0020A0D1101970021002096
:1019B0000DE0FE20D1E7FF20CFE70297002005E0F1
:1019C00001970220002102E0022002970421CDE9C4
:1019D00003100020002DCDF814808DF8180018BFDA
:1019E000B8F1000F05D001A8183029464246FEF78D
:1019F000B3FC484601F062FA38B101A901F11802BE
:101A00006B46484601F0ECF828B101A9204600F0E9
:101A1000A5F80138A1E700209FE7000079B180B563
:101A200082B00A6891F804C04B1D0021CDF800C0B7
:101A3000FFF782FF02B0BDE8804040B27047FE2051
:101A400040B270472DE9F04389B001AC04F11809A8
:101A50000025E84604E000BF002D05F1010520D176
:101A6000EFB23846FFF77AFD0028F5D0064600BFF2
:101A7000384600F027F80028EED1304601F01EFA73
:101A80000028E9D03846214600F02EF80028E3D09F
:101A9000304621464A46434601F0A2F80028E7D0E6
:101AA000DAE709B0BDE8F08341F2484100EBC0102D
:101AB000C2F2000101EBC0000021C0F80014C0F820
:101AC0000414704741F2484100EBC010C2F200011B
:101AD00001EBC000D0F80014D0F80404081AB0FAE2
:101AE00080F0400970470000002904BF00207047C3
:101AF0002DE9F04141F2484C00EBC012C2F2000C5B
:101B00000CEBC202D2F800E4D2F804349E451FD098
:101B100002F204452C6800EBC0100CEBC00000EB97
:101B20004412640150F804C0D2E901805769D2E937
:101B30000364C1E900C8C1E90447C1E90206D2E96A
:101B40000620C1E906202868013000F01F00286047
:101B5000BEEB030018BF0120BDE8F08101284FF063
:101B6000000238D8B9B32DE9F04741F2484C00EBF8
:101B7000C012C2F2000C0CEBC202D2F80034D2F850
:101B800004E4013303F01F0373451ED002F580699E
:101B9000D9F8004000EBC0100CEBC00000EB441281
:101BA0004FEA441AD1E904C6D1E90078D1E90254D8
:101BB00040F80A705661C2E9034CC2E90185D1E9D7
:101BC0000610C2E90610C9F80030B3EB0E0218BFC8
:101BD0000122BDE8F04710467047000080B507F0CD
:101BE000CFF980BD40B1042808D003281EBFFF20D4
:101BF00040B270470A2002E0062000E0172080B5BE
:101C000001F0E8FF0020BDE8804040B270470000CE
:101C100040B1042808D003281EBFFF2040B27047FF
:101C20000A2002E0062000E0172080B501F0D6FF70
:101C30000020BDE8804040B270470000072884BF04
:101C40000020704780B54CF2E071C0F6000101EB56
:101C5000C002526831F83010104601F033FF0138ED
:101C6000B0FA80F0400980BDB9B1072882BFFF20DB
:101C700040B270474CF2E072C0F6000232F830C059
:101C8000002000232CFA00F2D20709D10E2B03F119
:101C9000010300F10100F5D908E0FE2040B27047D1
:101CA00040F2D012C2F2000242F82010002040B2EE
:101CB00070470000072882BFFF2040B2704780B500
:101CC0000A464CF2E071C0F6000101EBC0035B680C
:101CD00031F83010184601F0FBFE0020BDE88040CE
:101CE00040B2704780B506F0D5FF80BD00281EBF0A
:101CF000FF2040B27047B7EE001A40F66840B4EEDD
:101D0000410AC2F20000F1EE10FAC8BFB0EE410A7B
:101D100000689FED0C1AC16AB5EE400A0131F1EE80
:101D200010FAB8BFB0EE410A01EE101AB8EE411A2F
:101D300020EE010ABCEEC00A80ED0D0A002040B280
:101D4000704700BF0000000010B510B1FF2460B262
:101D500010BD40F66840C2F200000021002403F0EC
:101D600057F860B210BD000040F61041C2F2000109
:101D7000002818BF002108467047000070B510B158
:101D8000FF2040B270BD1E4614460D46FFF7ECFF23
:101D90000028F5D02946224616B102F0A7FB02E042
:101DA000142302F0E9FA002818BF012040B270BDE8
:101DB000002A0FBFFE2040F21823C2F2000303EBFB
:101DC00040101CBF40F82120002040B270470000A6
:101DD00070B510B1FF2040B270BD1E4614460D46CE
:101DE000FFF7C2FF0028F5D02946224616B102F0BF
:101DF0006BFE02E0142302F013FC002818BF012040
:101E000040B270BD70B5044605F06EFF0546FF2672
:101E100005F04CFF411C05290BD80120884010F02B
:101E2000310F0BD110F0060F0AD0204601F044FD0F
:101E300011E06FF00041884218BF002670B270BDFB
:101E40004FF47A70B0FBF5F1B4FBF1F0A14288BF1A
:101E5000012005F001FF002670B270BD2DE9F041B0
:101E600005F042FF044608F045FA4FF47A784EF246
:101E70001806B8FBF4F4CEF20006376804FB00F550
:101E800008F038FA60433168854208BF394656F891
:101E9000042C01FB08F10132B1FBF2F100FB08F068
:101EA000401A00F57A700021BDE8F08140F64052FA
:101EB00040F6F841C2F200020128C2F2000118BF48
:101EC0000022002818BF11460846704780B582B02E
:101ED00001680A68D20614D5002201920A680192AC
:101EE00049680191019905F07DFB40F2382100EB32
:101EF000C000C2F2000101EB8000006A002818BF98
:101F0000804702B080BD00003AB101284FF0FF03C6
:101F100098BF082904D958B27047FE2358B27047B9
:101F200040F2382300EBC000C2F2000303EB800054
:101F3000002340F8212058B270470000FEE700005F
:101F400080B540F68010C2F2000000F0CBFF80BDEB
:101F500080B540F68010C2F2000000F0C3FF80BDE3
:101F600080B540F6A810C2F2000000F0BBFF80BDB3
:101F700080B540F6A810C2F2000000F0B3FF80BDAB
:101F80004FF0030160B146F200420068C4F2000263
:101F900002F58063984208BF0121801A08BF0146FC
:101FA000C8B270470A78012A09D04ABB897C032944
:101FB00026D8DFE801F002270202002123E091F891
:101FC0002320032A05D8D2004FF0807323FA02F2AF
:101FD000027191F82410032908D002290CD001299C
:101FE0000ED143F23331C3F6B37102E00021C4F2E3
:101FF00020014161002070470021C4F2A00141612D
:10200000002070470121017100207047002101600C
:102010000171704710B50A780446531E022B0ED387
:10202000032A14D0002A18BF10BD887C08B1487C50
:1020300040B9204600F010F80020206010BD91F853
:10204000260020B10846214600F00AF810BD2046BF
:1020500000F002F810BD000000210171704700007F
:10206000024612F8013B012B03D0002B18BF70472A
:1020700001E000F113029068D3688860CB601068BB
:10208000086170472DE9F04F81B02DED028B80463D
:1020900000284FF0FE0000F0B7800D46002900F048
:1020A000B380FFF7DBFED8E90023801A99410AF0DC
:1020B000A0FA9FED580A01EE100A81EE000A88EDA1
:1020C000020AFFF7CBFEC8E900014046294600F0AE
:1020D000A5F808B1FD2097E098F80C00012808D079
:1020E000002840F090800020C8E90400C8F81800DB
:1020F00015E095ED020A95ED031A95ED052A95ED8B
:10210000043A20EE020A22EE011A22EE033A88ED8A
:10211000040A88ED051A88ED063A88ED072A98ED3D
:10212000040A08F24C4003F08FFB88ED040A98ED96
:10213000050A08F26C4003F087FB88ED050A98ED6C
:10214000060A08F28C4003F07FFB404688ED060A41
:1021500000F0AEF89FED308A40F6F80A6FF00F06F7
:1021600040F2AC4940F22C5B4FF48077C2F2000A97
:1021700008EB060494ED180AD4ED380A84ED1C0A25
:10218000D8ED021A08EB07052846B0EE481A04F00D
:102190003DF90AEB060080ED040AD4ED340AD8EDCF
:1021A000021A05F1F000B0EE481A04F02FF908EB1E
:1021B0000B0084ED240A03F047FB04F2DC5080EDB1
:1021C000000A94ED100AD4ED2C0A84ED200AD8ED13
:1021D000021A05F5F070B0EE481A04F017F908EB92
:1021E000090084ED280A03F02FFB04F2CC500436DA
:1021F00009F120090BF1200B07F13C0780ED000AE3
:10220000B6D1002000E0FD2040B2BDEC028B01B051
:10221000BDE8F08F0024744900000000F0B1F0B573
:1022200081B004460D464FF4807700BFE61906F5ED
:10223000F07004F0EBF906F1F00004F0E7F9304635
:1022400004F0E4F93C37B7F5F87FEFD12879207333
:10225000002001B0BDE8F04040B27047FE2040B21F
:1022600070470000F0B581B0044600F5B766602500
:10227000D4F8280496ED010A2844371D03F0FCFC2D
:10228000D4F8280496ED050A2844203003F0F4FC25
:102290000835802D3E46EBD1D4F82804603003F099
:1022A000BFFBD4F82804803003F0BAFB01B0F0BDC6
:1022B0002DE9F04F81B02DED028B86B0077B0446EF
:1022C000012F3AD1206920F000400AF03DF99FED3E
:1022D0002A0B55EC106B32462B460AF075F960BBA1
:1022E000606920F000400AF02FF932462B460AF0D0
:1022F0006BF910BBA06920F000400AF025F93246C6
:102300002B460AF061F9C0B994F8D00304F1400CEF
:10231000002804BF012084F8D0030020C4E908008D
:10232000C4E90A00D4F8AC05D4F8B015D4F8B42543
:10233000D4F8B8358CE80F0030E2002084F8D003E0
:102340006FF00F0021180A6D0430C1F8BC25F9D1D7
:10235000002F00F01382012F1AD0022F40F01E82AE
:102360000020C4E90800C4E90A00C4E91000A06420
:1023700002E200BF00BF00BF9A9999999999B93FAD
:10238000CC3B7F669EA0E63FCD3B7F669EA0E63FAE
:10239000D4E9040AA5690AF0D7F880462846894698
:1023A0000AF0D2F81FED0A0B06465BEC102B5B46D9
:1023B0000F460292CDF814B009F05AFD42464B4642
:1023C00009F054FA02460B4609F052FD8146504688
:1023D00088460AF0B9F81FED140B05468A4653ECFF
:1023E000102B30463946CDE9032309F041FD2A463A
:1023F000534609F03BFA02460B4609F039FD024606
:102400000B464846414609F031FA41EC100B08F002
:102410004FFF51EC100B09F0F7F92062D4E90408E2
:10242000A5690AF091F8074628468A460AF08CF812
:10243000029A5B460646894609F01AFD3A4653461B
:1024400009F014FA02460B4609F012FD8246404696
:102450008B460AF079F8DDE9032305460F4630463E
:10246000494609F005FD02460B462846394609F063
:102470007DFF02460B4609F0FBFC02460B46504628
:10248000594609F0F3F941EC100B08F011FF51EC3B
:10249000100B09F0B9F96062D4E90401A569019152
:1024A0000AF052F80746284689460AF04DF8DDF84A
:1024B0000880059B424606468B4609F0D9FC024639
:1024C0000B463846494609F051FF02460B4609F0D3
:1024D000CFFC814601988A460AF036F8DDE90323ED
:1024E00007460D463046594609F0C2FC02460B46E7
:1024F0003846294609F03AFF02460B4609F0B8FC77
:1025000002460B464846514609F0B0F941EC100B23
:1025100008F0CEFE51EC100B09F076F9A062D4E978
:10252000040AA5690AF010F80746284689460AF009
:102530000BF8059B424606468B4609F099FC02467D
:102540000B463846494609F011FF02460B4609F092
:102550008FFC81465046884609F0F6FF0D465946E5
:10256000DDF80CA0DDF810B00746304652465B4659
:1025700009F07EFC3A462B4609F078F902460B46F4
:1025800009F076FC02460B464846414609F06EF9D2
:1025900041EC100B08F08CFE51EC100B09F034F9F3
:1025A000E062D4E90480A66909F0CEFF0546304612
:1025B000894609F0C9FF52465B4606460F4609F0B8
:1025C00057FC2A464B4609F051F941EC180B40469E
:1025D00009F0BAFF029A059B0546884630463946FF
:1025E00009F046FC2A46434609F040F941EC110B3C
:1025F000B0EE480AF0EE680A08F082FB51EC100BCE
:102600009FEDB10B53EC102BCDE9002309F030FC0A
:1026100009F0FAF82064D4E904A0A66909F094FF4F
:10262000054630468B4609F08FFFDDF80C90049B81
:102630004A4606460F4609F01BFC02460B46284652
:10264000594609F093FE41EC180B504609F07CFF07
:10265000DDF80880059B05468A46304639464246E5
:1026600009F006FC2A46534609F000F941EC110B2B
:10267000B0EE480AF0EE680A08F042FBDDE90023FC
:1026800051EC100B09F0F4FB09F0BEF86064D4E9DA
:1026900004A0A66909F058FF054630468B4609F0AC
:1026A00053FF4A46DDF8109006464B460F4609F0A8
:1026B000DFFB02460B462846594609F057FE41EC1F
:1026C000180B504609F040FF4246DDF814800546DD
:1026D0008A4630463946434609F0CAFB02460B4655
:1026E0002846514609F042FE41EC110BB0EE480A73
:1026F000F0EE680A08F004FBDDE9002351EC100B52
:1027000009F0B6FB09F080F8A064D4E904A0A6693A
:1027100009F01AFF054630468B4609F015FF039A6B
:102720004B4606460F4609F0A3FB2A465B4609F0D6
:102730009DF841EC180B504609F006FF029A054639
:102740008A4630463946434609F092FB02460B461C
:102750002846514609F00AFE41EC110BB0EE480A3A
:10276000F0EE680A08F0CCFADDE9002351EC100B1A
:1027700009F07EFB09F048F8E0640FE00020C4E9AE
:102780000800C4E90A0048F200000021C4F29D30AC
:10279000C4F23421C4E91001C4E912019FED4C0ACE
:1027A00004F14000002100BF421892ED001A0431EC
:1027B000B5EE401AF1EE10FABCBF31EE001A82ED10
:1027C000001A1029F0D19FED431A9FED432A9FED87
:1027D000433A9FED434A9FED435A40F2982100202F
:1027E000C2F200010FE000BFB1EE476A82ED0C6A51
:1027F00097ED006A93ED007A36EE076A01300428FF
:1028000082ED146A57D004EB800292ED106A92EDCB
:10281000347A01EB800336EE476AB4EE416AF1EE9A
:1028200010FA83ED006A08DD36EE026AB4EE416A02
:10283000F1EE10FAF8DC83ED006A93ED006AB4EE75
:10284000436AF1EE10FA08DA36EE006AB4EE436A33
:10285000F1EE10FAF8DB83ED006AB4EE446AF1EEB3
:1028600010FA02F1D0070FDDB4EE416AF1EE10FA72
:102870000ADC166A97ED006A166393ED007A36EE6D
:10288000076A36EE036AB9E792ED087AB4EE456A54
:10289000F1EE10FAA8DAB4EE436AF1EE10FAA3DB17
:1028A00082ED0C7A97ED006A93ED007A36EE076AB6
:1028B00036EE016AA2E706B0BDEC028B01B0BDE8BE
:1028C000F08F00BF00BF00BF00000000DCA54C403F
:1028D0000000B443000034430000B4C3000034C31C
:1028E0000000B4420000B4C2002870D0F0B581B03E
:1028F0002DED0C8B044603F073FA9FED399A9FED92
:1029000039AA9FED39BA9FED39CA9FED338B9FED00
:1029100038DA0025802600BFD4F82804304403F0BC
:102920001DF9183003F04EF880EE090AD4F8280497
:102930006719304420EE0A0A87ED340A03F00EF9D5
:10294000183003F047F880EE0B0AD4F8280430441E
:10295000203887ED300A03F001F9183003F03AF817
:1029600080EE0C0A07F5836097ED341A90ED002A8B
:1029700087ED280A31EE420A10EE100A09F0E4FD54
:1029800041EC100BB0EE481AF0EE681A08F00EFC9D
:1029900051EC100B08F038FF00EE100AB5EE400ABB
:1029A000F1EE10FA05F1040530EE0D1AB8BFB0EEE5
:1029B000410A102D06F1080687ED340AACD100203B
:1029C000BDEC0C8B01B0BDE8F04040B27047FE207A
:1029D00040B2704700BF00BF00000000008076409A
:1029E000DB0F4940000034430000A04300401C4678
:1029F0000000B443B5EE401AF1EE10FA30EE600A72
:102A0000D8BF7047B6EE002A21EE022AB4EE420A81
:102A1000F1EE10FAC4BF30EE410A7047B1EE422A1F
:102A2000B4EE420AF1EE10FAB8BF30EE010A704778
:102A300040F20800C2F200007047000080B540F686
:102A4000F020C2F2000000F0D7FD80BD80B540F656
:102A50005030C2F2000000F0CFFD80BD80B540F6DE
:102A6000D010C2F2000000F0C7FD80BD80B540F676
:102A70003020C2F2000000F0BFFD80BD80B540F6FE
:102A80009020C2F2000000F0B7FD80BD80B540F696
:102A9000B030C2F2000000F0AFFD80BDD0F800C041
:102AA0006FF00F024AF6AB2352FA8CF2CAF6AA2351
:102AB0000146A2FB0330000905A31B5C40F2FF3076
:102AC0002CEA00005F2A88BF0430C1E91603704772
:102AD00000061016000610168269816AB2F5005FC2
:102AE00006D06AB9022912D0012914D0D1B90EE05A
:102AF000032917D8DFE801F0020B020F012070470D
:102B000003293CBF012070471CBF00207047C06AEA
:102B1000C0F300607047C06AA0F1C070B0FA80F0E6
:102B2000400970470020704780B5D0F800C0D0F849
:102B300008E0DCF80000BEF1400F20F48020CCF863
:102B400000000846CCF8043004BF10460A46CCF812
:102B50000800CCF80C2080BD00284FF0FE0018BF04
:102B6000002901D140B27047032008700020C1F84D
:102B70000100C1F80500C1F80900C1F80D00A1F875
:102B8000110040B2704700007047000080B501207E
:102B900000F0BCFE80BD000080B5102000F0B6FE45
:102BA00080BD000080B5202000F0B0FE80BD000098
:102BB00072B600BFFEE7000090F82020013A012A1B
:102BC00004D8006800F11402002004E000F124029F
:102BD00001204FF4802113681943116070470000F1
:102BE00010B590F820E0D0F800C0AEF1010EBEF1B3
:102BF000010FDCF808E00ED81EF0E05F11D0CEF334
:102C0000016E012000FA0EF018608B687BB14868F5
:102C100043EAC0030DE000F1240101204FF48022BB
:102C200023E000F1240101204FF400121DE00868A8
:102C30004305D1E9030403430CEB0E10C0F88031C7
:102C4000C0F88441097D012905D100F5C2710B68E6
:102C500043F480730B605168C0F88C11126800F562
:102C6000C071C0F88821002001220B681A430A6055
:102C700010BD0000B0B590F82020013A012A2FD8ED
:102C800046F20060C4F20000026842F001020260F5
:102C9000026822F47C520260D1F814E0CC694A6ADE
:102CA0000368012C43EA022202600EF01F024FF07B
:102CB000010303FA02F2C3696FEA020C23EA02037A
:102CC000C36113D02CBBC36803EA0C03C360CB6899
:102CD0008C8844EA034300EBCE0423640B4611E0E6
:102CE000416A41F4802141620120B0BDC3681343B1
:102CF000C3600B688C8844EA034300EBCE04236472
:102D000001F10C038C681B8843EA044300EBCE04FA
:102D1000636443688D6943EA0204D1F810E0096AEC
:102D2000002D08BF03EA0C0444604369BEF1000FA4
:102D300043EA020408BF03EA0C040129446102D1FA
:102D4000C1691143C161016821F0010101600020E6
:102D5000B0BD000080B5FFF713F9032808BF80BDA0
:102D600040F26811C2F20001342210FB0210006B25
:102D7000002818BF804780BD90F82020013A012A22
:102D800084BF0020704700681022002908BF0C2271
:102D9000805800F00300704710B590F82040013CC7
:102DA000012C0AD8046871B12469A4070ED100F17E
:102DB000240101204FF4001276E000F124010120EB
:102DC0004FF4802270E0E468A40771D0046804EB3B
:102DD000011CDCF8B0410CF5D87E14F004049460BA
:102DE000DCF8B04119BFE4085460640D1460DEF8EB
:102DF00000400CF5DA7E04F00204D460DCF8B44143
:102E000024075ABFDEF8004004F00F0408241461C0
:102E1000DEF800400029C4F307249461DEF8004086
:102E20004FEA14445461DCF8B8211A70026802EBCE
:102E30000112D2F8B8214FEA12225A70026802EB4E
:102E40000112D2F8B8214FEA12429A70026802EBDE
:102E50000112D2F8B8214FEA1262DA70026802EB6E
:102E60000112D2F8BC211A71026802EB0112D2F8E9
:102E7000BC214FEA12225A71026802EB0112D2F809
:102E8000BC214FEA12429A71026802EB0112D2F899
:102E9000BC214FEA1262DA71006814BF00F1100120
:102EA00000F10C01002020220B681A430A6010BDBB
:102EB00000F1240101204FF40012F5E790F82010F2
:102EC0000139012984BF0020704700688168826849
:102ED0008068C1F38061C2F3C0621144C0F3007026
:102EE000084470472DE9F04F81B0044600684669F8
:102EF000D0F804908768D0F80CB0D0F810A0D0F8C3
:102F00001880F10703D1002530071CD423E0F9070E
:102F100010D00121BA07816009D4780700F1AA8096
:102F2000380700F1B080204600F096FA02E0204613
:102F300000F0A4FA0025F80500F18480F80300F100
:102F4000AA80300707D51BF0100004D0206845F494
:102F500000751021C160700708D51BF0080005D06E
:102F600020680821C160204600F0EEF9B00706D5C0
:102F70002068C068800702D0204600F0F7F970068C
:102F800007D51AF0100004D0206845F480651021A0
:102F90000161B00608D51AF0080005D020680821A4
:102FA0000161204600F0F4F9F00606D520680069BA
:102FB000800702D0204600F0FDF9B00308D519F0D3
:102FC000100005D0206810214160204600F004FA6E
:102FD000F00308D519F0080005D0206808214160E9
:102FE000204600F0A5FA300440F18F805FEA497076
:102FF00040F1888006F4807008EA102028435FEAD8
:103000008871014648BF41F00201B20558BF014630
:103010005FEA48700D4648BF45F00405700558BF8B
:103020000D4630056ED518F070006BD010380009D1
:10303000052862D8DFE800F0035356595C5F45F07D
:1030400008055AE020684FF48071BA0581600AD4FF
:10305000780512D4380519D4204600F021FAF80377
:103060007FF56FAF17E0204600F02CFAF8037FF5EC
:1030700068AF10E04FF400655DE705F50055F80313
:103080007FF55FAF07E04FF4805554E705F58045C5
:10309000F8037FF556AF20684FF48031BA038160A2
:1030A0000AD478030FD4380313D4204600F01CFA56
:1030B00030073FF548AF4EE7204600F027FA3007CB
:1030C0003FF541AF47E705F5004530073FF53BAF1A
:1030D00041E705F5803530073FF535AF3BE745F073
:1030E00010050AE045F0200507E045F0400504E042
:1030F00045F0800501E045F480752068816921F084
:10310000700181612068042141602DB1606A28430B
:1031100060622046FFF71EFE01B0BDE8F08F0000A0
:10312000B0B5C8B1044690F8200010B9204600F0B0
:1031300071F82068016841F00101016000F0CEFCE7
:10314000054600BF20684168C90707D100F0C6FCEA
:10315000401B0B28F6D312E00120B0BD016821F01E
:103160000201016000F0BAFC054600BF206841681A
:1031700089070DD500F0B2FC401B0B28F6D3606A1E
:10318000052140F400306062012084F82010B0BDB9
:10319000217E0268012922F0800208BF803202608D
:1031A000617E0268012922F0400208BF40320260BD
:1031B000A17E0268012922F0200208BF20320260AD
:1031C000E17E0268012922F0100218BF103202606D
:1031D000217F0268012922F0080208BF083202603C
:1031E000617F0268012922F0040208BF04320260F4
:1031F000D4E901C2D4E9033561691A432A43114372
:10320000ACF101021143C16100200121606284F828
:103210002010B0BDB0B586B0006846F60002C4F21A
:10322000000200219042CDE90411CDE90211019183
:1032300036D046F20041C4F20001884240F082805C
:1032400040F21021C2F200010A6843F64000C4F2C5
:103250000200531C0B6052B900210091016841F03B
:1032600000710160016801F0007100910099002176
:10327000009150F8101C152441F0080140F8101C72
:1032800050F8100C142500F008000090009803205E
:10329000019040F20040C4F2020000F5006036E008
:1032A00043F64000C4F202000091016841F08061E1
:1032B0000160016801F080610091009940F21021E5
:1032C000C2F200010A68531C0B6052B90021009140
:1032D000016841F000710160016801F00071009126
:1032E00000990021009150F8101C412441F0020186
:1032F00040F8101C50F8100C402500F0020000901F
:1033000000986020019040F20040C4F202000221C7
:10331000029100210391032104910921059101A942
:1033200000F002FB28460521002200F05BFC284645
:1033300000F054FC20460521002200F053FC2046FA
:1033400000F04CFC06B0B0BD80B5FEF719FE0328B6
:1033500008BF80BD40F26811C2F20001342210FBA8
:103360000210C069002818BF804780BD80B5FEF7F5
:1033700007FE032808BF80BD40F26811C2F20001B9
:10338000342210FB02108069002818BF804780BDDE
:1033900080B5FEF7F5FD032808BF80BD40F2681137
:1033A000C2F20001342210FB0210406A002818BF4C
:1033B000804780BD80B5FEF7E3FD032808BF80BDD0
:1033C00040F26811C2F20001342210FB0210006AC0
:1033D000002818BF804780BD80B5FEF7D1FD0328C7
:1033E00008BF80BD40F26811C2F20001342210FB18
:1033F0000210806A002818BF804780BDB0B504461F
:1034000090F8200001281DD1022084F820002068B7
:10341000016821F00101016000F060FB054600BF7A
:1034200020684068C00713D000F058FB401B0B28F1
:10343000F6D3606A40F400306062052084F8200012
:103440000120B0BD606A40F4002060620120B0BD80
:1034500000206062B0BD000080B5FEF791FD03283A
:1034600008BF80BD40F26811C2F20001342210FB97
:103470000210C068002818BF804780BD80B5FEF7E5
:103480007FFD032808BF80BD3421484340F2681106
:10349000C2F200010858002818BF804780BD000014
:1034A00080B5FEF76DFD032808BF80BD40F26811AE
:1034B000C2F20001342210FB02100069002818BF7C
:1034C000804780BD80B5FEF75BFD032808BF80BD47
:1034D00040F26811C2F20001342210FB0210406871
:1034E000002818BF804780BD80B5FEF749FD03283E
:1034F00008BF80BD40F26811C2F20001342210FB07
:1035000002104069002818BF804780BD80B5FEF7D3
:1035100037FD032808BF80BD40F26811C2F20001E8
:10352000342210FB02108068002818BF804780BD3D
:1035300080B5FEF725FD032808BF80BD40F2681165
:10354000C2F20001342210FB0210C06A002818BF2A
:10355000804780BD70B5866D044600F0BFFA94F8D0
:103560003510022925D105462068216C026822F019
:1035700016020260426922F08002426109B9A16C20
:1035800019B1016821F008010160016821F0010111
:10359000016000BF20680068C0070ED000F09EFAEE
:1035A000401B0628F6D320206065032084F83500F0
:1035B0000CE080206065012008E0E06D3F2101FA09
:1035C00000F0B060012084F835000020002184F86C
:1035D000341070BD90F83510022909D1052180F80A
:1035E00035100068016821F001010160002070477A
:1035F0008021416501207047F0B581B0044600206C
:10360000009040F20000C2F200000268D4E91660A7
:1036100048F2B51337680821C1F64E33814039426C
:10362000A2FB03250CD0226813685B0708D513683A
:1036300023F004031360B160616D41F00101616525
:1036400001218140394208D022685269120604D50E
:10365000B160616D41F00201616504218140394230
:1036600008D022681268920704D5B160616D41F0FC
:103670000401616510218140394215D0206802683B
:10368000120711D5B16002680168520306D4C9055A
:1036900006D4016821F00801016001E0080342D46A
:1036A000216C09B120468847E16D202000FA01F223
:1036B0003A4244D020680368DB0640D5B26094F8F3
:1036C00035300268052B1ED122F0160202604269D5
:1036D00022F080024261226C0AB9A26C1AB102681F
:1036E00022F0080202603F208840B060012084F888
:1036F0003500216D0020002984F8340040D0204698
:10370000884701B0F0BD0168520310D4C90512D436
:10371000016821F010010160012084F835000020CB
:1037200084F8340007E0A16C0029BBD1BCE7080392
:1037300001D4616C00E0E16B09B120468847606DFF
:10374000F0B1606DC00717D0052084F835002068FF
:10375000A90A026822F00102026000BF009A013249
:103760008A42009202D80268D207F7D1012084F879
:103770003500002084F83400E16C09B12046884708
:1037800001B0F0BD2DE9F041044600F0A7F9C4B145
:103790000546022084F835000020216884F83400B2
:1037A000086820F00100086026683068C0070BD068
:1037B00000F094F9401B0528F6D9032120220320AC
:1037C00042E00120BDE8F081306848F23F01CFF2CD
:1037D0001001251D00EA010C2ECDD4E9050E41EAA9
:1037E0000C01114319432943D4E90778084340EAFF
:1037F0000E01606A3943042841EA080103D1D4E983
:103800000B231143194331607169042821F007012A
:1038100041EA00050CD1D4E90A1045EA010538B1A6
:103820002046FFF759F918B10121402201200BE091
:1038300020467561FFF732F9E16D3F2202FA01F18E
:103840008160002201210020626584F83510BDE806
:10385000F0810000B0B5044690F83400012828D06B
:10386000012084F83400A56D94F8350001281DD19D
:10387000022084F83500002060652046FFF754F9E7
:10388000E26D3F23206803FA02F2216CAA6002680D
:1038900042F01602026019B1016841F008010160AE
:1038A000016841F0010101600020B0BD002084F8F2
:1038B00034000220B0BD0000B0B5044600F00EF99F
:1038C000054640F2F800C2F200000078611C18BF03
:1038D000044400BF00F002F9401BA042FAD3B0BD7F
:1038E00070B540F2D01604460025C2F2000603E08F
:1038F0000135102D08BF70BD24FA05F0C007F7D0C0
:1039000056F82500002818BF8047F1E780B543F638
:103910001441C4F201010A68024208BF80BD086078
:10392000FFF7DEFF80BD00002DE9F04F83B000F10E
:103930003E4202F1FF724FEAB22241F60047019285
:10394000C4F2020708224FF0010E00254FF0000AD2
:103950004FF00008B84208BF072200920AE000BFFB
:1039600008F101080AF1040AB8F1100F05F1020587
:1039700000F0A4800C680EFA08FB14EA0B09EFD0E3
:103980004C6804F0030CACF1010EBEF1010F11D82C
:103990000322876802FA05F6CA68B743AA403A4389
:1039A00082604268C4F3001722EA0B0207FA08F7A4
:1039B0003A434260BCF1030F1CD0C26803238E68F7
:1039C00003FA05F7BA4306FA05F73A43BCF1020FCA
:1039D000C2600FD16FF0030202EA580202440AF0FB
:1039E0001C060F23176A03FA06F40B69A743B340BA
:1039F0003B431362026803234F68AB409A4307F0CE
:103A00000303AB401A4317F4403F4FF0010E02602E
:103A1000A6D0002243F644030292C4F202031A68BD
:103A200043F6004442F480421A601A68C4F201046A
:103A300002F480420292029A28F003024FF6084BE9
:103A40002244CFF6FF7B52F80B300AF00C070F260A
:103A5000BE4023EA060C019B009E072B38BF1E4682
:103A600006FA07F747EA0C0342F80B30A2684B68E6
:103A700042EA090743F60C4CDE0258BF22EA090766
:103A8000A760C4F2010CDCF800209E0242EA09079C
:103A900058BF22EA0907CCF8007062689E0342EA28
:103AA000090758BF22EA090767602268DB0342EA78
:103AB000090358BF22EA0903236051E703B0BDE8B8
:103AC000F08F00000069084018BF01207047000017
:103AD000002A08BF090481617047000045F66000B4
:103AE000C2F200000068704740F2F80045F660013D
:103AF000C2F20000C2F2000100780A6810440860B7
:103B00007047000080B543F60040C4F2020001682F
:103B100041F400710160016841F480610160016855
:103B200041F480710160032000F06CF80F2000F078
:103B300005F800F02BF8002080BD0000B0B540F281
:103B4000F802C2F2000240F200011278C2F2000153
:103B50004FF47A730968B3FBF2F20446B1FBF2F159
:103B6000084601F05DF80F2C4FF001050CD858B94C
:103B70004FF0FF3021460022002500F033F840F2DC
:103B8000FC00C2F2000004602846B0BD80B582B0DF
:103B9000002043F640010190C4F202014A6842F459
:103BA00080424A604A6802F480420192019A009081
:103BB0000868002240F08050086008680F2100F07B
:103BC0008050009000986FF0010000F00BF802B0F8
:103BD00080BD000080B503F0A1FE80BD80B503F07C
:103BE000B1FE80BD70B514460D46064603F0BAFE20
:103BF0002946224602F0F4FB0146304603F0BAFEA5
:103C000070BD000080B503F0CFFE80BD2DE9F0410E
:103C1000002800F08B8043F60808C4F2020804462E
:103C2000D8F8F8030D4600F00700884207D288F85C
:103C3000F853D8F8F80300F00700A84276D12068BE
:103C4000810717D5410705D5D8F8001041F4E05198
:103C5000C8F80010010705D5D8F8001041F46041FC
:103C6000C8F80010D8F80010A26821F0F001114344
:103C7000C8F80010C0073FD1D8F8F80300F00700DB
:103C8000A84207D988F8F853D8F8F80300F00700DD
:103C9000A8424BD12068410707D5D8F80010E26848
:103CA00021F4E0511143C8F80010000708D5D8F8F6
:103CB0000000216920F4604040EAC100C8F800001B
:103CC00000F07EF8D8F800104CF2C872C1F303116E
:103CD000C0F60002515C40F2000220FA01F140F20D
:103CE000FC00C2F200000068C2F200021160FFF79F
:103CF00025FF0020BDE8F0816068811E022907D2FF
:103D000058F8081C89015CBF0120BDE8F08110E073
:103D1000012807D158F8081C89035CBF0120BDE8C1
:103D2000F08106E058F8081C890702D40120BDE89C
:103D3000F081D8F8001021F003010843C8F8000012
:103D4000FFF7CCFE064641F2883700BFD8F80000E6
:103D5000616800F00C00B0EB810F8DD0FFF7BEFE64
:103D6000801BB842F2D90320BDE8F08140F2000088
:103D7000C2F200000068704780B5FFF7F7FF43F616
:103D80000801C4F2020109684CF2D872C1F3822121
:103D9000C0F60002515CC84080BD000080B5FFF74E
:103DA000E5FF43F60801C4F2020109684CF2D8723B
:103DB000C1F34231C0F60002515CC84080BD000032
:103DC00010B543F60404C4F20204606800F00C006D
:103DD00008280AD0042819BF42F20040C0F2F400BB
:103DE00041F60030C0F2B70010BD2068216823689A
:103DF000490241F60031C0F2B70100F03F02C3F3BF
:103E000088105CBF42F20041C0F2F401A1FB000146
:103E10000023FCF729FA21680222C1F3014102EBD9
:103E20004101B0FBF1F010BD2DE9F04182B0002856
:103E300000F0A2800446007843F60006C007C4F2F2
:103E4000020643D0B06800F00C00042805D13068A9
:103E500080033BD56068C8BB8EE0B06800F00C0002
:103E6000082802D170684002F1D46568B5F5A02F2A
:103E70000AD0B5F5803F0BD0306820F48030306038
:103E8000306820F4802006E0306840F48020306004
:103E9000306840F480303060FFF720FE002D05468A
:103EA00011D000BF3068800310D4FFF717FE401B0D
:103EB0006428F7D922E100BFFFF710FE401B6428F9
:103EC0004FF0030055D830688003F5D42078800780
:103ED0001AD5B06810F00C0F09D0B06800F00C00D3
:103EE000082840F08A807068400200F186803068BF
:103EF000800702D5E06801283ED13068216920F0B2
:103F0000F80040EAC10030602078000738D42078FB
:103F100040074CD4A5695DB3B06800F00C000828D8
:103F200040F09E80012D27D07068E16900F4800286
:103F30008A4221D1216A00F03F028A421CD147F611
:103F4000C071626A0140B1EB821F15D1A26A0023E1
:103F5000CFF6FF7303EBC23200F440316FF30F0270
:103F6000914209D1E16A00F07060B0EB016F03D1BA
:103F7000002002B0BDE8F081012002B0BDE8F08170
:103F80006069002840F20000C4F2472057D00121A8
:103F9000C0F8801EFFF7A2FD054600BF706F8007C6
:103FA000B5D4FFF79BFD401B0228F7D9A6E0306C83
:103FB00010F080580AD100200190306C40F0805001
:103FC0003064306C00F080500190019847F2000797
:103FD000C4F200073868C00524D4386840F4807003
:103FE0003860FFF77BFD05463868C0051AD4FFF737
:103FF00075FD401B0228F7D980E0E068002851D009
:104000000020C4F2472001210160FFF767FD05464B
:10401000306880073FF571AFFFF760FD401B022855
:10402000F6D96BE0A568052D50D0012D52D0306F28
:1040300020F001003067306F20F004004DE00021D7
:10404000C0F8801EFFF74AFD054600BF706F80076D
:104050007FF55DAFFFF742FD401B0228F6D94DE02A
:104060000027C4F2472700203866FFF737FD022DEE
:1040700005460BD13068800158D5FFF72FFD401B56
:1040800002284FF00300F5D973E700BF30688001C4
:104090007FF56EAFFFF722FD401B02284FF00300B3
:1040A000F4D966E70020C4F2472000210160FFF741
:1040B00015FD0546306880077FF526AFFFF70EFD3A
:1040C000401B02284FF00300F4D952E7306F40F054
:1040D00004003067306F40F001003067FFF7FEFCEE
:1040E000002D054641F2883714D000BF306F80079D
:1040F00013D4FFF7F3FC401BB842F7D9032002B0FA
:10410000BDE8F081FFF7EAFC401BB8424FF0030026
:104110003FF62FAF306F8007F4D4B8F1000F7FF473
:10412000F9AE306C20F080503064F3E604F11C05E9
:104130002FCD08430021CFF6FF7140EA821001EB3A
:10414000C3316FF30F0140EA05600843706001203E
:104150003866FFF7C3FC0446306880013FF508AFBE
:10416000FFF7BCFC001B02284FF00300F4D900E766
:1041700080B502F089FC022808BF80BD40F21821FA
:10418000C2F2000101EB40108069002818BF80478F
:1041900080BD000070B538B10446406A30B10020DF
:1041A000206104F1140007E0012070BD6068B0F5E3
:1041B000827F03D004F11C00002101600026A6626A
:1041C00094F8510020B9204684F8506000F03CF883
:1041D000022084F8510094E80F0001F48271056810
:1041E00002F4044225F040050560114403F4006226
:1041F0002369114403F002026369114403F00102D0
:10420000A369E569114403F40072114405F0380212
:10421000256A114405F08002A56A114305F4005295
:1042200011430160626A042101EA134102F01002A5
:1042300011444160C16921F40061C16101206665DA
:1042400084F85100304670BD2DE9F04F87B0044628
:1042500043F200070068C4F201070026B842069640
:10426000CDE904660396029602D007B0BDE8F08F50
:1042700043F630000196C4F20200416902AD41F4F8
:1042800080514161416946F2404801F480510191F9
:104290000199019601684FF0020941F002010160A5
:1042A00001684FF0030A01F00201019101990196A2
:1042B00001684FF0050B41F00101016000682946DB
:1042C00000F00100019001981820029007F5544079
:1042D000C4F20208CDE90396CDF814A0CDF818B0C9
:1042E000FFF722FB8020CDE9020904A880E8400CFA
:1042F00007F550402946FFF717FB40F6D015C2F2EC
:1043000000054FF440304FF0C0674FF48069C5E9B5
:1043100008062846C5E90087C5E90266C5E904968E
:10432000C5E90666FFF72EFA002818BFFEF740FC25
:10433000E564AC6340F6302508F11800C2F20005D0
:104340004021C5E9000705F10800002280E80602C7
:104350004FF40030C5E908022846C5E90522EA61A4
:10436000FFF710FA002818BFFEF722FCA564AC6323
:1043700007B0BDE8F08F00002DE9F04182B004469F
:1043800090F85100012815D10E4600294FF0010088
:1043900060D01746002A5DD060681D46B0F5827F68
:1043A00002D1A068002858D0FFF798FB94F850106D
:1043B000012903D1022002B0BDE8F081804601202E
:1043C00084F85000042084F8510000206065A66342
:1043D000A787E7872063A086E086A1682064B1F5FF
:1043E000004F606408D12068016821F0400101603D
:1043F000016821F48041016020680168490603D406
:10440000016841F040010160E168E08F91B300284C
:1044100055D06E1C0BE000BFC068A16B21F8020BE9
:10442000A163E08F0138E087E08F002847D0206843
:104430008168C907F0D1FFF751FB002EF4D0A0EB43
:104440000800A842F0D3012084F85100002084F82D
:104450005000032002B0BDE8F081042084F8510030
:104460002046314632463B46009500F09FF902B0A7
:10447000BDE8F08118B36E1C0BE000BF007BA16BA0
:104480000870A06B0130A063E08F0138E087E08FF7
:10449000A8B120688168C907F0D1FFF71FFB002E83
:1044A000F5D0A0EB0800A842F1D3012084F8510018
:1044B000002084F85000032002B0BDE8F0812046BF
:1044C0002946424602F052FA00281CBF20206065AF
:1044D000012084F85100002084F85000606D00280D
:1044E00018BF012002B0BDE8F081000010B50446FD
:1044F00090F8510001281CBF022010BD13460A4647
:1045000000294FF0010018BF002B00D110BDA0689A
:1045100058B96168B1F5827F07D1042084F8510051
:104520002046114600F03EFA10BD94F850100129C3
:1045300004BF022010BD012184F85010042184F82A
:1045400051100021B0F5004F6165A263A387E38796
:10455000C4E91011A186E18608D12068036823F020
:1045600040030360036823F480430360E06C46F675
:10457000150E46F63903C0F6000EC0F60003C0E97A
:104580000F3E46F2F173C0F60003D4F800C0C0E954
:104590001331E38F0CF10C01FFF75CF940B1606D52
:1045A00040F010006065002084F85000012010BD2C
:1045B00021680868400603D4086840F0400008609D
:1045C000002084F850004A6842F020024A604A689D
:1045D00042F001024A6010BD80B502F055FA02288F
:1045E00008BF80BD40F21821C2F2000101EB40106B
:1045F0004068002818BF804780BD000080B502F0E9
:1046000043FA022808BF80BD40F21821C2F200011F
:1046100001EB40100069002818BF804780BD0000F2
:104620002DE9F04182B01D4616460F460446FFF7BD
:1046300055FA94F8511001290DD18046002F4FF002
:10464000010018BF002E02D102B0BDE8F08194F83D
:104650005000012803D1022002B0BDE8F081012002
:1046600084F85000032084F851000020606527631F
:10467000A686E686A063A087E087A168C4E910004B
:10468000B1F5004F08D12068016821F040010160B8
:10469000016841F48041016020680168490603D443
:1046A000016841F0400101606168731EE268B1FA7F
:1046B00081F1B3FA83F349095B09B2F5006F41EA6E
:1046C000030124D139B1216B0988C160B81C206372
:1046D000E08E0138E086E08E002846D06E1C09E0AE
:1046E000216B31F8022BC2602163E08E0138E08635
:1046F000E08ED0B3206881688907F1D4FFF7EEF926
:10470000002EF5D0A0EB0800A842F1D323E039B188
:1047100039780173206B01302063E08E0138E08628
:10472000E08E10B36E1C0AE0216B09780173206BD8
:1047300001302063E08E0138E086E08EA8B1206869
:1047400081688907F0D4FFF7C9F9002EF5D0A0EBF6
:104750000800A842F1D3012084F85100002084F819
:104760005000032002B0BDE8F081204629464246B1
:1047700002F044F900281CBF20206065A06838B909
:10478000002001902068C168019180680190019823
:10479000012084F85100002084F85000606D00284A
:1047A00018BF012002B0BDE8F08100002DE9F04300
:1047B00081B01E4615460F460446FFF78FF994F860
:1047C00051108146012909D06068B0F5827F14D16B
:1047D00004294FF0020007D1A16829B9002F4FF03A
:1047E000010018BF002D02D101B0BDE8F083002EFA
:1047F000FAD094F85000012803D1022001B0BDE89E
:10480000F083012084F8500094F85100002104281E
:104810001CBF052084F851006165A563E687A68763
:104820002763E6862068A6862164616401684906DC
:1048300003D4016841F0400101606168731EE268C1
:10484000B1FA81F1B3FA83F3DDF8208049095B09FD
:10485000B2F5006F41EA030139D139B1216B098802
:10486000C160B81C2063E08E0138E086012608F1A3
:10487000010500BFE08E10B9E08F00286CD02068E1
:10488000816889070CD5E18E012E09D141B1216BD8
:10489000002631F8022BC2602163E18E0139E186E6
:1048A0008168C9070AD0E18F41B1C068A16B0126B8
:1048B00021F8020BA163E08F0138E087FFF70EF9C2
:1048C000002DD7D0A0EB09004045D3D33AE039B151
:1048D00039780173206B01302063E08E0138E08667
:1048E000012608F1010500BFE08E08B9E08F98B3FA
:1048F0002068816889070DD5E18E012E0AD149B162
:10490000216B002609780173206B01302063E08E53
:104910000138E08620688168C9070BD0E18F49B172
:10492000C068A16B01260870A06B0130A063E08F06
:104930000138E087FFF7D2F8002DD5D0A0EB0900B1
:104940004045D1D3012084F85100002084F8500064
:10495000032001B0BDE8F083204641464A4602F0FC
:104960004DF840B120206065002084F850000120FF
:1049700001B0BDE8F083A06838B90020009020683D
:10498000C1680091806800900098012084F851006F
:10499000002084F85000606D002818BF012001B08D
:1049A000BDE8F08370B5044690F85100012806D1A7
:1049B00000294FF0010018BF002A0CD170BD6568B6
:1049C000B5F5827F0ED104284FF00200F6D1A5681C
:1049D000002DEDD0F2E7002B08BF70BD94F8500019
:1049E000012801D1022070BD012084F8500094F804
:1049F0005100002604281CBF052084F8510066657C
:104A00002163A386E386A263A387E387C4E91066D4
:104A100094F8510046F6150146F62D03C0F6000144
:104A2000C0F60003042808BF0B4646F6390046F6D8
:104A30001111C0F60000C0F6000108BF0146E06C8D
:104A40002568C0E90F1346F2F171C0F60001C0E914
:104A50001316E38F05F10C01FEF7FCFE38B1606D13
:104A600040F010006065012084F8506070BD22683D
:104A7000216BA06C536843F001035360C0E90F66DB
:104A8000C0E91366E38E0C32FEF7E4FE40B1606DC0
:104A900040F010006065002084F85000012070BDD7
:104AA00021680868400603D4086840F040000860A8
:104AB000002084F850004A6842F020024A604A68A8
:104AC00042F002024A6070BD10B5044690F85100F1
:104AD00001280AD100294FF0010018BF002A00D197
:104AE00010BD94F85000012801D1022010BD012012
:104AF00084F850000320002384F85100636521638B
:104B0000A286E286A363C4E91033A387E387A06883
:104B1000B0F5004F08D12068026822F04002026020
:104B2000026842F480420260A06C46F6210C46F610
:104B3000A102C0F6000CC0F60002C0E90F2C46F23C
:104B4000F172C0F60002D4F800E0C0E91323E38E4E
:104B50000EF10C02FEF77EFE40B1606D40F01000D9
:104B60006065002084F85000012010BD21680868AD
:104B7000400603D4086840F040000860002084F834
:104B800050004A6842F020024A604A6842F002023D
:104B90004A6010BD80B501F077FF022808BF80BDD4
:104BA00040F218214001C2F200010858002818BF45
:104BB000804780BD80B501F067FF022808BF80BD37
:104BC00040F21821C2F2000101EB4010C068002839
:104BD00018BF804780BD000080B501F055FF022856
:104BE00008BF80BD40F21821C2F2000101EB401065
:104BF0008068002818BF804780BD000080B501F0A4
:104C000043FF022808BF80BD40F21821C2F2000114
:104C100001EB40104069002818BF804780BD0000AC
:104C200080B501F0C9FF80BD002804BF0120704796
:104C300010B5044690F83D0028B9002084F83C00E7
:104C4000204600F01FF8022084F83D002068211D56
:104C500002F030F8012084F8460084F83E0084F821
:104C60003F0084F8400084F8410084F8420084F852
:104C7000430084F8440084F8450084F83D00002097
:104C800010BD000081B0006844F20041C4F201018F
:104C9000884201D001B070470020009043F64400E4
:104CA000C4F20200016841F400310160006800F4C0
:104CB00000300090009801B07047000080B586B0C9
:104CC00044F200410068C4F20101002288420592CA
:104CD000CDE903220292019201D006B080BD43F6D5
:104CE00030000092C4F20200036843F02003036026
:104CF000006800F020000090009840200190022001
:104D0000CDE9020204900320059001F5504001A96D
:104D1000FEF70AFE06B080BDB0B5044690F83C0030
:104D2000012804BF0220B0BD0D464FEAB2010120A8
:104D3000032984F83C0037D8DFE801F0020A122288
:104D40002068294602F05EF8206850F8181F0EE02F
:104D50002068294602F088F8206850F8181F16E0ED
:104D60002068294602F0B6F8206850F81C1F41F070
:104D700008010160016821F00401016029690FE068
:104D80002068294602F0DAF8206850F81C1F41F428
:104D900000610160016821F48061016029690902F4
:104DA0000268114301600020002184F83C10B0BD6E
:104DB000002804BF0120704710B5044690F83D005C
:104DC00028B9002084F83C00204600F01FF802209B
:104DD00084F83D002068211D01F06CFF012084F85B
:104DE000460084F83E0084F83F0084F8400084F8D0
:104DF000410084F8420084F8430084F8440084F8B9
:104E0000450084F83D00002010BD00007047000000
:104E100010B5044641B1082909D0042914BF04F192
:104E2000410004F13F0004E004F13E0001E004F120
:104E30004000007801281CBF012010BD022041B1B4
:104E4000082909D0042914BF84F8410084F83F00E0
:104E500004E084F83E0001E084F84000206801226C
:104E600001F0BEFF206841F2FF71C4F200018842E8
:104E70000FDC40F2FF71C4F20001884217DCB0F190
:104E8000804F49D040F20041C4F20001884243D033
:104E900049E040F2FF32C4F20102904214DC41F6D4
:104EA0000003C4F20003984236D0002314E040F619
:104EB0000001C4F2000188422ED040F60041C4F245
:104EC0000001884228D02EE044F20003C4F201031E
:104ED000984221D040F20043C4F20103984222D10B
:104EE000436C884243F400434364C2DD904207DCD4
:104EF00041F60001C4F2000188420DD0002107E014
:104F000044F20001C4F20101884205D040F20041A0
:104F1000C4F20101884206D1816801F00701062927
:104F200004BF002010BD016841F0010101600020B4
:104F300010BD00007047000080B502F053FB03284D
:104F400008BF80BD40F2382100EBC000C2F2000172
:104F500001EB80000069002818BF804780BD000079
:104F6000B0B582B0036804461868D9685A6900F081
:104F70002F05202D01F0200505D125B1204602F096
:104F800041FB02B0B0BD5FEA007C1EBF02F0010E23
:104F900001F4907212EB0E024AD1226B0840C10656
:104FA0003DD5012A3BD10020019018680190586836
:104FB000019001985869400642D4A08DE18DE28DA0
:104FC000002A1CBF401A5FEA004101D102B0B0BD07
:104FD000216851E8031F226821F4907142E803130D
:104FE000002BF5D1216851E8051F226821F001014D
:104FF00042E80513002BF5D1202184F8421000214E
:10500000216300BF216851E8031F226821F01001CD
:1050100042E80313002BF5D10221616354E001063D
:1050200054D44006D2D5204602F0C2FA02B0B0BD38
:10503000C20718BF11F480725DD1420761D467E0E6
:10504000E06B016849688AB2002A44D0A38D9A4275
:1050500041D2E185C069B0F5807F30D0206850E84A
:10506000030F216820F4807041E80302002AF5D183
:10507000206850E8050F216820F0010041E8050292
:10508000002AF5D1206850E8050F216820F0400083
:1050900041E80502002AF5D1202084F842000020D2
:1050A000206300BF206850E8030F216820F0100043
:1050B00041E80302002AF5D1E06BFEF74BFA02202B
:1050C0006063A08DE18D401A81B20FE0204602F0AE
:1050D000C1FB02B0B0BDA18D91427FF477AFC06932
:1050E000B0F5807F7FF472AF022060632046FFF747
:1050F00021FF02B0B0BD626C42F00102626442075F
:1051000006D5BEF1000F03D0626C42F00202626469
:10511000820706D5BEF1000F03D0626C42F0040294
:105120006264BCF1000F06D55EEA050203D0626C32
:1051300042F008026264626C002A3FF447AF084004
:10514000800602D5204602F05DFA20684069616C55
:1051500000F0400001F00801401827D0204602F07E
:10516000FFF92068406940061BD500BF206850E861
:10517000050F216820F0400041E80502002AF5D122
:10518000E06B70B147F26141C0F600010165FEF7C6
:1051900021FA00283FF41AAFE06B016D884702B096
:1051A000B0BD2046FFF7C8FE02B0B0BD2046FFF7F5
:1051B000C3FE0020606402B0B0BD0000002804BF40
:1051C0000120704710B5044690F8410028B900202E
:1051D00084F84000204600F021F8242084F84100A3
:1051E0002068C16821F40051C160204602F06EFAC7
:1051F0002068016921F490410161416921F02A018F
:105200004161C16841F40051C16000202021606407
:1052100084F8411084F84210606310BD2DE9F04716
:1052200086B00446006844F60001C4F2000100267E
:105230008842CDE90466CDE90266019677D041F255
:105240000041C4F20101884200F0BE8041F2000139
:10525000C4F20101884240F02B81002743F6300060
:105260000097C4F202004169002541F0100141613C
:105270004169C4F2020501F0100100910099009704
:10528000016801AE41F00201016001684FF00208BF
:1052900001F0020100910099009701684FF00309A5
:1052A00041F00101016000684FF0070A00F00100C1
:1052B000009000988020019005F580603146CDE98E
:1052C0000287CDF81090CDF814A0FEF72DFB4FF417
:1052D0000070CDE9010803A880E880062846314621
:1052E000FEF722FB46F22800C4F2020040F69025A9
:1052F00000F58C60C2F200054FF0006185E8830084
:105300004FF440304FF48062C5E908072846C5E9EC
:105310000372C5E90577EF61FEF734FA002818BF7C
:10532000FDF746FCE56305F138002525B7E043F6B7
:1053300030000096C4F20200016941F4802101614D
:10534000016901F48021009100990096016841F003
:1053500004010160006801A900F0040000900098B9
:105360004FF4406001900220CDE902060320049032
:10537000072005900020C4F2020000F50060FEF74F
:10538000D3FA40F6F02546F22800C2F20005C4F236
:1053900002004FF000614FF480624FF4807385E8A3
:1053A00043002846C5E90362C5E90566C5E9073635
:1053B0006E62FEF7E7F9002818BFFDF7F9FBE56319
:1053C00005F1380027256AE0002643F630000096F4
:1053D000C4F20200416946F2280841F0200141610F
:1053E0004169C4F2020801F0200100910099009681
:1053F000016841F040010160006801A900F040002F
:10540000009000984FF4844001900220CDE90206FC
:1054100003200490082005900020C4F2020000F54B
:10542000C050FEF781FA40F6503508F58060C2F2B0
:1054300000054FF0206A4FF48069C5E9000A4FF477
:1054400080372846C5E90266C5E90496C5E90666BF
:10545000C5E90876FEF796F9002818BFFDF7A8FB06
:10546000E563AC6340F6B03508F58F60C2F2000525
:105470004021C5E9000A05F1080080E842022846FB
:10548000C5E90566C5E907676E62FEF77BF9002886
:1054900018BFFDF78DFBA56305F1380047250460B3
:1054A000284605210022FEF79DFB2846FEF796FBC5
:1054B00006B0BDE8F087000080B590F84230202BA0
:1054C0001CBF022080BD00294FF0010318BF002A35
:1054D00001D1184680BD0023036302F065F903463D
:1054E000184680BD80B502F07DF8032808BF80BD56
:1054F00040F2382100EBC000C2F2000101EB800055
:10550000C068002818BF804780BD000080B502F049
:1055100069F8032808BF80BD40F2382100EBC000C5
:10552000C2F2000101EB80008068002818BF8047AC
:1055300080BD000080B502F055F8032808BF80BD8B
:1055400040F2382100EBC000C2F2000101EB800004
:105550004068002818BF804780BD0000FEE70000BB
:1055600045F6DF1110EE100AC5F63771B6EE001AD7
:10557000A1EB600020EE011A00EE100A21EE002AD5
:1055800022EE002AB7EE083A33EE422A22EE000A53
:1055900021EE001A20EE011A33EE411A20EE010A24
:1055A0007047000040F26111884204BF012070473B
:1055B000B0F5806F04BF03207047A0F29F60B0FA7F
:1055C00080F040094000704700284FF0FE0018BFEF
:1055D000002901D140B27047032008700020C1F8B3
:1055E0001300C1F81700C1F81B00C1F81F00C1F873
:1055F0002300C1F82700C1F82B00C1F82F0040B2EA
:1056000070470000000000002DE9F0412DED088BEF
:1056100040F2F821C2F200014A788B78044663F325
:105620000A2200EE102AB8EEC00A80ED000A88783F
:10563000CA780B79C0084F7962F34A1000EE100A5D
:10564000980040EA921007F00102B8EEC00A40EA62
:10565000822084ED030A00EE100AB8EEC00A84ED41
:10566000010A48798A79400862F3CA10CB7901EEC1
:10567000100AB8EEC11A100984ED021A63F30A1079
:10568000A083087A4A7A400040EAD31002F003036C
:105690008F7A40EA4320CE7A2082900867F38A10FE
:1056A0006083F00040EA57102083087B4A7B8B7BA5
:1056B00062F30A20CF7BE082D00863F34A100A7CB1
:1056C000A082B80040EA931002F00103497C40EA4E
:1056D00083209FED5B8A9FED5B9A60825008BFEE4E
:1056E00000AAB7EE00BA61F3CA10F0EE480AB0EEB5
:1056F000491AF0EE4A1AB0EE4B2AE08302F09EFA05
:1057000094ED001A84ED010AB0EE410AF0EE480A69
:10571000B0EE491AF0EE4A1AB0EE4B2A02F08EFAB9
:1057200094ED021A84ED000AB0EE410AF0EE480A48
:10573000B0EE491AF0EE4A1AB0EE4B2A02F07EFAA9
:1057400094ED031A84ED020AB0EE410AF0EE480A25
:10575000B0EE491AF0EE4A1AB0EE4B2A02F06EFA99
:105760002068B0EE408A84ED030A06F0EDFE9FED5E
:10577000300B074658EC106B324643460D4606F098
:105780002AFF58B99FED2C0B384653EC102B2946B5
:1057900006F013FF002804BF00202060606806F0B8
:1057A000D3FE3246434605460F4606F014FF58B96D
:1057B0009FED210B284653EC102B394606F0FDFED9
:1057C000002804BF00206060A06806F0BDFE3246DD
:1057D000434605460F4606F0FEFE58B99FED160BF0
:1057E000284653EC102B394606F0E7FE002804BF8C
:1057F0000020A06018EE100A06F0A6FE32464346CE
:1058000005460F4606F0E7FE58B99FED0B0B2846FC
:1058100053EC102B394606F0D0FE002804BF0020C0
:10582000E0600120BDEC088BBDE8F08100BF00BF47
:105830007B14AE47E17A84BF7B14AE47E17A843FA4
:105840000080B04300E0D34410B52DED088B88B341
:10585000B0EE408A90ED010A90ED069A90ED021AA2
:1058600090ED07AA29EE000A38EE400A2AEE011A46
:1058700030EE41BA04461BEE100A02F047F8002849
:1058800008BFB0EE4B8A94ED030A94ED041A94ED30
:10589000052A20EE080A29EE011A30EE010A2AEE46
:1058A000021A30EE010A84ED068A84ED079ABDECF7
:1058B000088B10BD9FED020ABDEC088B10BD00BF28
:1058C00000000000002808BF704710B5F5EE400A40
:1058D0000446C0ED000A0020F1EE10FAA061E0617C
:1058E0002EDD80EE200A9FED1E1A81EE000A05F0E3
:1058F0001DFD9FED1C1AB7EE002A20EE011A31EEB5
:10590000023A20EE000ABFEE005A30EE033A30EEC3
:10591000055A32EE411A80EE034A35EE055A30EE52
:10592000010A85EE035A80EE030A34EE041A84ED70
:10593000034A84ED041A84ED054A84ED015A07E018
:105940004FF07E519FED050AC4E90310606160606D
:1059500084ED020ABDE81040704700BF000000005F
:10596000DB0F4940F304B53F10B52DED048B10B3A8
:10597000B0EE408A90ED030A90ED041A90ED052AEE
:1059800030EE010A30EE020A88EE009A044619EE63
:10599000100A01F0ABFF00282046B0EE480A08BF0D
:1059A000B0EE489A84ED069A84ED079AFFF74CFF13
:1059B000BDEC048B10BD9FED020ABDEC048B10BD45
:1059C00000000000002814BF90ED050AB8EE000AA0
:1059D00070470000002814BF90ED060AB8EE000AD8
:1059E00070470000B0B5012802D9FF2040B2B0BD19
:1059F00040F2F025C2F20005044655F8200060B9D7
:105A00004820FCF76FF9002845F82400EDD0482124
:105A1000FAF7EFFC55F824000470002040B2B0BD46
:105A2000B0B584B048B304780546204600F064F869
:105A300028B36988A1F201210A295BD8012202FA60
:105A400001F10A071DD111F0F00F30D040F2FF1123
:105A5000009108218DF804100A3000216A4600BF29
:105A600000EB41035B7802EB41056B7110F81130DC
:105A700001310429AB71F3D131E0FE2037E0FC2085
:105A800035E04FF40071009108218DF804100230C8
:105A900000216A4600EB41035B7802EB41056B7124
:105AA00010F8113001310429AB71F3D117E040F245
:105AB000FF21009108218DF80410123000216A4660
:105AC00000EB41035B7802EB41056B7110F811307C
:105AD00001310329AB71F3D10020ADF80B00694609
:105AE0002046FBF79BFF002818BF4FF0FF3040B265
:105AF00004B0B0BDFF20FAE701288FBF002040F2BC
:105B0000F021C2F2000151F82000704748B102288C
:105B10000BD0012814BF4FF6FF704FF4804000B245
:105B2000704742F2107000B2704747F2305000B236
:105B300070470000022905D2A0F2012189B206298E
:105B400009D805E007D1A0F2052189B2052902D8BC
:105B5000013840B27047FF2040B27047F0B581B0C5
:105B600008B307460078FFF7C7FFE0B1014690F899
:105B70004400C0B101F11802002306E0012585B1FF
:105B800091F844500133AB420DD252F82340002C1F
:105B9000F4D065887E88B542F0D100252046002DDE
:105BA000EED101B0F0BD002001B0F0BD022884BFED
:105BB000B7EE000A704740B202A101EB800090ED01
:105BC000000A7047000010422CA099410000803F5D
:105BD00070B538B104460078FFF704FF28B1FF2004
:105BE00040B270BDFE2040B270BD2078FFF784FF48
:105BF0000028F4D090F8442005469AB105F1180029
:105C0000002104E095F84420013191420AD250F875
:105C10002120002AF6D0528863889A42F2D1FD20D2
:105C200040B270BD0A2ADAD85020FCF75BF8002891
:105C3000D5D0064620686168C6E9000106F1180063
:105C40002821FAF7D6FB62792078618886F8282027
:105C50000322FBF79DFD18B13046FBF7BFFFBEE7FF
:105C600095F8440005EB8001013085F844000020E0
:105C700040B28E6170BD000070B52DED048B002820
:105C80003ED005460078B0EE408AFFF735FFC8B336
:105C9000B7EE000AB4EE408AF1EE10FAC8BFB0EEDB
:105CA000408ABFEE000AB4EE408A0446F1EE10FAD4
:105CB000B8BFB0EE408A6879B1EE489A002828460D
:105CC00008BFB0EE489AFFF749FFE8B12E7968881F
:105CD0003146FFF72FFF002818D405463046FFF75E
:105CE00015FF00EE100AB8EEC00A29EE000ABDEE5C
:105CF000C00A10EE100A04EB45014880002006E0BF
:105D0000FE2004E0FC2002E0FC2000E0FF2040B286
:105D1000BDEC048B70BD00002DE9F04F87B000286A
:105D200052D004460078FFF7E7FE00284ED0054623
:105D300090F8440000284BD005F11806E8464FF0D3
:105D4000010A40F2E93B4FF0000908E00121002977
:105D500041D095F8441009F1010989453AD256F825
:105D60002970002FF2D07A8861888A42EED120789B
:105D700042460023FBF706FC70B1FCF76FF8D7E949
:105D80000823801A9941B0EB0B0071F1000016D383
:105D900000203876FC2013E087F818A0FCF75EF8A6
:105DA000C7E908013846414600F06AFA07F10803DE
:105DB0000FCB07F12C0C8CE80F00002000E0FF2037
:105DC00000210029C5D106E0FE2004E0FC2002E00D
:105DD000FC2000E0FC2040B207B0BDE8F08F0000DE
:105DE0002DE9F04100254FF0000804E0B8F1000F64
:105DF00008F101081ED15FFA88F0FFF77DFE002848
:105E0000F4D0044690F844000028EFD004F11807BD
:105E1000002604E094F8440001368642E6D257F8A2
:105E200026000028F6D0FFF777FF002818BF4FF0B4
:105E3000FF35EFE768B2BDE8F081000080B540F6BD
:105E4000801046F20041C2F20000C4F200010322B9
:105E5000002380E80E0000F10C014FF4A02C4FF459
:105E6000C00E81E8085083618383FDF759F900284B
:105E700018BFFCF79DFE80BD80B540F6A81046F621
:105E80000001C2F20000C4F200010322002380E8F6
:105E90000E0000F10C014FF4A02C4FF4C00E81E86D
:105EA000085083618383FDF73BF9002818BFFCF796
:105EB0007FFE80BD80B582B0002043F630010190A6
:105EC000C4F202010A6842F480020A600A6802F41D
:105ED00080020192019A00900868002240F40010AC
:105EE00008600868052100F40010009000980C205C
:105EF000FDF778FE0C20FDF771FE39200521002208
:105F0000FDF770FE3920FDF769FE3A2005210022D9
:105F1000FDF768FE3A20FDF761FE3B2005210022D7
:105F2000FDF760FE3B20FDF759FE442005210022CD
:105F3000FDF758FE4420FDF751FE452005210022C3
:105F4000FDF750FE4520FDF749FE02B080BD000080
:105F500080B546F6AD304CF62C12C0F60000C0F607
:105F60000002002102F050F940F66811C2F200016F
:105F7000086046F68D704CF6B002C0F60000C0F620
:105F80000002002102F040F980BD00002DE9F04739
:105F900086B0002643F630000596CDE90366CDE9CC
:105FA00001660096C4F202000168002441F002017B
:105FB00001600168C4F2020401F00201009100993D
:105FC0000096016804F5E05741F040010160016866
:105FD000002201F0400100910099009601684FF401
:105FE000E05A41F001010160016801F001010091F6
:105FF00000990096016841F008010160016801F014
:106000000801009100990096016841F004010160C7
:10601000016801F00401009100990096016841F0C7
:1060200080010160016801F08001009100990096F3
:10603000016841F02001016000684FF4E05100F078
:106040002000009000983846FDF742FD20461021C0
:1060500001224FF010090125FDF73AFD04F5806893
:10606000404601210122FDF733FD0396022001AED7
:10607000049038463146CDE901A5FDF755FC4FF4B3
:106080008817204631460195CDE90275FDF74CFC95
:1060900020463146CDE90195CDE90355FDF744FC95
:1060A0003020CDE9010704F5006031460395FDF786
:1060B0003BFC40463146CDE90155CDE90355FDF79E
:1060C00033FC062005210022FDF78CFD0620FDF79C
:1060D00085FD0A2005210022FDF784FD0A20FDF739
:1060E0007DFD172005210022FDF77CFD1720FDF71F
:1060F00075FD06B0BDE8F08710B540F6104043F2DC
:106100000001C2F20000C4F201014FF482720023C8
:106110004FF0010C4FF4007E182480E80E000A2195
:10612000C0E90333C0E905CEC461C0E90833C0E962
:106130000A31FEF72FF8002818BFFCF739FD10BD13
:1061400080B588B040F6684044F200420021C2F2B7
:106150000000C4F201024FF6FF730791CDE905116B
:10616000CDE90311CDE90111C0E90021C0E9021315
:1061700001618161FEF758FD002818BFFCF718FD8A
:1061800040F66840C2F20000FEF712FE002818BF79
:10619000FCF70EFD602001900020CDE90200059083
:1061A00040F66840C2F2000001A90022FEF7B4FDEB
:1061B000002818BFFCF7FCFC40F66840C2F2000063
:1061C000FEF77CFD08B080BD80B540F6B04041F2DE
:1061D0000001C2F20000C4F2010100234FF00C0CD8
:1061E0004FF4E13280E80E00C0E90333C0E905C393
:1061F000C361FEF7E3FF002818BFFCF7D9FC80BDA0
:1062000010B540F6F84044F6000C48F2A062C2F225
:106210000000C4F2000CC0F201024FF480530021D0
:106220004FF4806E0C24C0E900C2C0E90231C0E91D
:1062300004E4C0E90611FEF7C1FF002818BFFCF70F
:10624000B7FC10BD80B540F6405041F20041C2F2AB
:106250000000C4F2010100234FF00C0C4FF4E132B6
:1062600080E80E00C0E90333C0E905C3C361FEF74F
:10627000A5FF002818BFFCF79BFC80BDFEE70000CF
:106280002DE9F0478846B1F80D10044608BA4FEAE8
:106290001049B8F811002679B8F80F1005BA304641
:1062A00091FAB1FAFFF732FC07463046FFF77EFC61
:1062B00001EE109A9FED453AB8EE412A9FED441A3F
:1062C00022EE032A22EE014A02EE10AA15FB27F065
:1062D000B8EEC23A02EE100AA0799FED3E5AB8EE2F
:1062E000C22A22EE052A48B1B4F84000A9EB00000A
:1062F000B0F5805F0CDD4FF0FF300DE00020A4F81A
:106300004090C4E9110084ED024A84ED033A1CE098
:1063100010F5805F03DA0120616C0844606494ED3D
:10632000115A83EE003AB8EEC55A25EE015A34EE02
:10633000054A84EE004AA4F8409020EE022A84ED3B
:10634000033A84ED124A84ED024A94ED020A84ED88
:10635000042AB5EE400AF1EE10FA08DA30EE010A2E
:10636000B5EE400AF1EE10FAF8DB84ED020A94ED86
:10637000020AB4EE410AF1EE10FA0ADB9FED162A8A
:1063800030EE020AB4EE410AF1EE10FAF8DA84EDCA
:10639000020A94F8280078B131EE400A84ED020A2E
:1063A00094ED030A94ED041AB1EE400A84ED030A59
:1063B000B1EE410A84ED040A98F8130000EE100AC9
:1063C000B8EE400A84ED050ABDE8F0870000003908
:1063D000DB0FC94000008038DB0FC9C0FEE70000BA
:1063E00000F0070080F00703042B28BF04234FF0C0
:1063F000FF3C03380CFA03F338BF00209943814077
:106400000CFA00F022EA000008437047B0B52DED09
:106410000A8B044610EE100AB0EE618AB0EE419A83
:10642000B0EE60AAB0EE40BA01F068FA002800F0C1
:106430009C801AEE100A01F061FA002800F09580A5
:1064400019EE100A01F05AFA002800F08E8018EEBA
:10645000100A01F053FA002800F087806068B0EE5F
:106460004B0A90ED071AF0EE4A0AFCF7C3FA60688F
:10647000B0EE40BA90ED001A04F11C0020EE01CA03
:1064800021EE0A0AFFF7E0F9207888B1012811D13E
:1064900094ED051A94ED022A30EE411AB4EE428AC8
:1064A000F1EE10FAC8BFB0EE482A81EE029A01E080
:1064B0009FED309A19EE100A84ED04BA84ED050AB6
:1064C00001F01CFA65689FED2B0A002808BFB0EEAA
:1064D000409A95ED010A95ED032A2CEE000A29EE6B
:1064E000022A95ED021A30EE42AA94ED030A9FEDBE
:1064F000229A2CEE082A32EE008AB4EE491AF1EE06
:1065000010FA28EE01BA1ADD18EE100A01F0F6F9B9
:10651000A8B13AEE0B0A95ED051AB0EEC00AB4EE3A
:10652000410AF1EE10FA0ADC95ED040AB0EEC81A41
:10653000B4EE401AF1EE10FAD8BF84ED038A3AEEB9
:106540000B8A18EE100A01F0D9F970B1D5ED050AE1
:10655000F4EE490AF1EE10FA05DDB0EE480AFAF75A
:106560005DFDB0EE408A84ED068A94ED060ABDEC2E
:106570000A8BB0BD00000000BD37863570B52DED2B
:10658000048B90B3044650681646B0EE408A0D4620
:1065900001F0B4F958B3B06801F0B0F948B3F0684D
:1065A00001F0ACF938B3306901F0A8F928B370698B
:1065B00001F0A4F918B3B7EE000A80EE089A6660FD
:1065C00019EE100A01F09AF9D8B1D6ED060A04F1D5
:1065D0001C00B0EE480A84ED029AFFF773F92046DA
:1065E000257000F013F800200CE0FF200AE0FF20E7
:1065F00008E0FF2006E0FF2004E0FF2002E0FF208B
:1066000000E0FF2040B2BDEC048B70BD10B568B156
:1066100000F11C0100249FED070AC0E90344C0E912
:1066200005440846FFF7A0F960B210BDFF2460B230
:1066300010BD00BF000000000000000000000000CE
:10664000EFF30980BFF36F8F154B1A681EF0100F20
:1066500008BF20ED108A20E9F04F10602DE90900F5
:106660004FF0500080F31188BFF34F8FBFF36F8F4F
:1066700002F02AFF4FF0000080F31188BDE8090006
:1066800019680868B0E8F04F1EF0100F08BFB0ECB2
:10669000108A80F30988BFF36F8F704700BF00BF77
:1066A000FC0E002010B501F0ABFD41F24441C2F2F6
:1066B00000010860A8B146F2A572C0F600020020F1
:1066C00003210024FBF720FC40F2F820C2F2000076
:1066D000C0E90044C0E90244C0E90444047660B261
:1066E00010BDFE2460B210BD70B500284FF0FE0052
:1066F00052D01546002A4FD00120087028460C467B
:1067000001F11306FEF780FFA868B060E868F0604A
:106710002868306068687060B5F91000FEF742FFC5
:10672000B5F9121084F823000846FEF73BFFB5F9CF
:10673000141084F824000846FEF734FFB5F91660FB
:1067400084F825003046FEF72DFFB5F9181084F8BF
:1067500026000846FEF726FFB5F91A1084F8270030
:106760000846FEF71FFFB5F91C1084F828000846FC
:10677000FEF718FFB5F91E1084F829000846FEF749
:1067800011FF40F29F618E4284F82A0006D128460C
:106790002146FEF719FF002040B270BD002040B234
:1067A00070BD000080B541F24440C2F200000068B4
:1067B000012101F087FC80BD80B50020FBF776FB4E
:1067C00040F2F821C2F200011922FEF775FE0028FE
:1067D00018BF4FF0FF3080BD80B502460120012177
:1067E00001F0B0FC0138B0FA80F0400980BD000033
:1067F00080B5806B01684A6822F003024A60416DEF
:1068000041F010014165012180F85110FDF7B0FC05
:1068100080BD000080B5806BFDF7F0FE80BD0000FC
:1068200080B5806BFEF7C6F980BD000080B5806B37
:10683000FEF7E4F980BD0000B0B5846B0546FDF7B6
:106840004DF929680968C90526D402462068A1685F
:10685000436823F02003436031B96168B1F5827F5A
:1068600002D16FF0030101E06FF0010143681940AC
:1068700041602046642100F079F800281CBF2020E8
:1068800060650020E087012084F85100606D18B138
:106890002046FDF76DFCB0BD2046FDF79DFEB0BD66
:1068A000B0B582B0846B0546FDF718F92968096810
:1068B000C90528D402462068416821F020014160C2
:1068C000416821F0020141602046642100F096F801
:1068D00018B1606D40F020006065A06838B90020F4
:1068E00001902068C16801918068019001980020A2
:1068F000E086012084F85100606D20B12046FDF74C
:1069000037FC02B0B0BD2046FEF744F902B0B0BD7E
:10691000B0B5846B0546FDF7E1F829680968C9053B
:106920001FD402462068416821F0200141602046C2
:10693000642100F063F818B1606D40F020006065DC
:106940002068416821F0030141600020E086E08773
:10695000012084F85100606D18B12046FDF708FC55
:10696000B0BD2046FEF738F9B0BD0000B0B582B02A
:10697000044640680B46B0F5827F20D1A168B1F58E
:10698000004F02D0B1F5806F04D121680D6825F069
:1069900040050D60B0F5827F11D1A068B0F5806F21
:1069A0001DD10092204601210022002500F076F83A
:1069B00090B1606D032540F0200060650CE000920E
:1069C000204601210022002500F068F820B1606D0A
:1069D000032540F020006065284602B0B0BD00925B
:1069E000204680210022002500F058F80028F3D02E
:1069F000606D032540F020006065EDE770B582B062
:106A00000D461646022101222B460446009600F050
:106A100045F838B1606D032540F0200060652846D8
:106A200002B070BD40F20000C2F20000006849F6FA
:106A30008171C1F25E61A0FB0101480D4FF47A71D2
:106A4000484301906068B0F5827F0FD120468021D5
:106A500000222B460096002500F020F80028DED00A
:106A6000606D032540F020006065D8E7019840B1D3
:106A7000019801380190206880680006F6D400254E
:106A8000CDE70025CBE70000006843F20001C4F227
:106A90000101401A18BF0120400070472DE9F0475E
:106AA00082B00A9C984615460E468146FDF716F8B8
:106AB000201A00EB0804FDF711F840F20001C2F2C1
:106AC00000010968C1F3CB3161430191D9F800108D
:106AD00089683140891BB1FA81F14909A94203D182
:106AE000002002B0BDE8F087824608F101070CE003
:106AF000019801380190D9F8000080683040801B6F
:106B0000B0FA80F04009A842EAD0002FF3D0FCF799
:106B1000E5FFA0EB0A00A04204D201980028E7D1CB
:106B20000024E8E7D9E900014268B1F5827F22F04C
:106B3000E00242600BD1D9F80810B1F5004F02D045
:106B4000B1F5806F03D1016821F040010160D9F8EF
:106B50002810B1F5005F07D1016821F400510160F0
:106B6000016841F400510160012089F851000020C2
:106B700089F85000032002B0BDE8F0870000000053
:106B8000074B19680868B0E8F04F80F30988BFF335
:106B90006F8F4FF0000080F31188704700BF00BF77
:106BA000FC0E002080B500F0F7FE80BD80B501F03E
:106BB00027FB01F083FB80BDB0B501380024B4EBA6
:106BC000106F1CBF0120B0BD4EF21005CEF20005C3
:106BD00068604FF0FF300F2100F0CCFE0720AC6062
:106BE00028602046B0BD000080B5FCF77DFF03F0B3
:106BF0006DFB012818BF02F03FFD80BD70B592B05B
:106C000006AC20463021F9F7F4FB002543F640009E
:106C10000595CDE90355CDE901550095C4F2020073
:106C20000168022641F080510160006800F0805048
:106C30000090009847F200000095C4F2000001683F
:106C400041F480410160006800F4804000900098A9
:106C5000012006904FF4803007904FF480000D9093
:106C600006200E90A820CDE90F06042011902046A2
:106C70000C96FDF7D9F888B90F20CDE901064FF43D
:106C8000A05004904FF48050059001A80521039571
:106C9000FCF7BCFF002804BF12B070BDFBF788FFF3
:106CA0004EF68850CEF20000016841F47001016098
:106CB00070470000B0B540F6FF3E0568C4F2000E14
:106CC00040F2004C7045C4F2010C0FDCB0F1804F73
:106CD00019D040F20043C4F20003984213D040F6AA
:106CE0000003C4F2000398420DD011E040F60043C7
:106CF000C4F20003984206D0604504D00023C4F2D9
:106D00000103984204D14B6825F0700243EA020562
:106D100041F6FF73C4F2000398420DDC70451FDC9E
:106D2000B0F1804F41D040F20043C4F200039842DA
:106D30003BD040F6000321E043F6FF73C4F20103A9
:106D4000984220DC42F20003C4F2000398422CD0A7
:106D50000023C4F20103984227D0604525D029E0E2
:106D600040F60043C4F2000398421ED041F60003EF
:106D7000C4F20003984218D041F60043C4F2000365
:106D8000984212D016E044F20003C4F20103984284
:106D90000BD044F60003C4F20103984205D044F23C
:106DA0000043C4F20103984204D1CB6825F4407239
:106DB00043EA02050A688C684B69C46240F4806447
:106DC0008262644504BF09690163026825F080019D
:106DD00042F0040219430260012242610160B0BD29
:106DE00080B501F01F014FF0010CD0F820E00CFA43
:106DF00001F32EEA03030362036A02FA01F1194365
:106E0000016280BDB0B5026A036A40F2004523F01A
:106E100001030362D0F804E0D0F818C08C6822F0B7
:106E2000020240F48063C4F20105AB4242EA04026C
:106E300005D1CC6822F00C0224F0040422430C6833
:106E4000AB4207D1D1E905532EF4407E45EA0E0549
:106E500045EA030E2CF073032343C0F804E083617A
:106E6000496841630262B0BD70B5026A036A40F2CC
:106E7000004423F010030362D0F804E0D0F818C0F7
:106E80008D6822F0200240F48063C4F20104A34222
:106E900042EA051207D1CD686FF0400622F0C00229
:106EA00006EA05152A430D68A34207D1D1E9056416
:106EB0002EF4406343EA860343EA840E2CF4E6434F
:106EC00043EA0523C0F804E08361496881630262F4
:106ED00070BD000070B5026A036A40F2004423F4FA
:106EE00080730362D0F804E0D0F81CC08D6822F4EF
:106EF000007240F48063C4F20104A34242EA052216
:106F000007D1CD6840F2FF462D0222F44062B5431E
:106F10002A430D68A34207D1D1E905642EF44053FA
:106F200043EA061343EA041E2CF073032B43C0F814
:106F300004E0C3614968C163026270BD70B5D0F8F6
:106F400020C0026A40F2004622F480520262426887
:106F5000C3690C68D1F808E040F48065C4F201060A
:106F6000B54204D14D6922F4804242EA851223F4ED
:106F7000E64343EA04234260C3612CF400564968A7
:106F800046EA0E320164026270BD000010B500F0E6
:106F9000C3FE47F279004CF62002C0F60000C0F6AE
:106FA0000002002101F030F941F2AC34C2F20004D9
:106FB000206047F271304CF6D402C0F60000C0F6F3
:106FC0000002002101F020F9606047F2C9104CF680
:106FD0004402C0F60000C0F60002002101F014F9DE
:106FE000A06047F299204CF66802C0F60000C0F697
:106FF0000002002101F008F9E06047F231304CF660
:107000008C02C0F60000C0F60002002101F0FCF87E
:10701000206147F221404CF6F802C0F60000C0F6AD
:107020000002002101F0F0F8606102200A21002234
:1070300000F008FFA06102202F21002200F002FFD3
:10704000E06102201821002200F0FCFE20620220F4
:107050000C21002200F0F6FEE06202200C2100224A
:1070600000F0F0FEA06200F087FE01F0C9F801F028
:1070700025F910BD0000000000F036FE04F06DFEA2
:107080009FED4B0B53EC102B04F0A4FC04F038FEE6
:107090008246002000F0E0FD00F01CFE41F2AC3919
:1070A00040F2A825C2F20009C2F20005044609F127
:1070B00040012846FAF708F82846F9F7DFFF40F2C2
:1070C000842BC2F2000B40F6D851C2F200015846A0
:1070D000F9F7A2FA40F6985040F2D8029FED360A2E
:1070E000C2F20000C2F200020021FFF747FA0020BE
:1070F000FAF72AFE9FED318A9FED319A40F68C58BF
:1071000004EB0A0705F1100405F11C06C2F20008A1
:10711000FAF728F9F9F79EFFF9F7A8FFF9F7BEFF8C
:10712000F9F7CAFF00F0F8FD2846FAF76FF828468D
:10713000FAF7B6F840F6D853584621463246C2F21E
:107140000003F9F72BFB40465946F9F7F7F9D9F850
:10715000280000F00FFFD9F8280031460022002354
:1071600000F0C0FED9F82C0000F004FFD9F82C0084
:1071700041460022002300F0B5FE00F0FDFDD5EDF4
:107180000A0A40F69850C2F20000B0EE480AB0EE8B
:10719000491AF0EE491AFFF739F90020FAF7A6FD6F
:1071A000384600F069FD5744B2E700BF00BF00BF9A
:1071B0000000000000407F400000FA430000204231
:1071C000000000000000000086B000F08DFD04F01B
:1071D000C4FD9FED2D0B53EC102B04F0FBFB04F0D2
:1071E0008FFD80460020002700F036FD00F072FD84
:1071F0000446FBF71DFC40F21835C2F200059FED76
:10720000240A0146284600F0DFFB41F2AC3A40F682
:10721000201904EB0806C2F2000A05F20C4B05F532
:107220007D74C2F2000910E028466946CDE9047772
:10723000CDE90277CDE90077FAF724FF2846FBF77E
:1072400011F8304600F018FD4644DAF82C00594693
:107250000022002300F0B2FDDAF8280021460022C7
:10726000002300F0ABFDDAF820004946002200239D
:1072700000F0A4FD0028D7D12846FBF735FB2846AF
:107280004946D9E700BF00BF0000000000407F4032
:107290000000FA430000000000F026FD04F05DFD50
:1072A0009FED210B53EC102B04F094FB04F028FD10
:1072B0008046002000F0D0FC00F00CFD40F60815E0
:1072C000C2F2000506462846FAF7A0FE41F2AC34A9
:1072D00041F27C374644C2F20004C2F2000712E0D9
:1072E00028463946FAF75EFE00F046FD206A00F0B7
:1072F00041FE206A29460022002300F0F3FD3046BB
:1073000000F0BAFC464400F007FDE069394600226F
:10731000002300F053FD0028E2D128463946FAF751
:1073200079FEDDE700BF00BF0000000000407F40A5
:1073300000F0DAFC04F011FD9FED0B0B53EC102B69
:1073400004F048FB04F0DCFC0446002000F084FC60
:1073500000F0C0FC051900BF284600F08DFC254454
:10736000FAE700BF00BF00BF0000000000407F4000
:1073700000F0BAFC04F0F1FC9FED270B53EC102B4E
:1073800004F028FB04F0BCFC0446002000F064FC80
:1073900000F0A0FC0546FFF785F940F66C1840F6B2
:1073A000381740F6E85941F2AC3640F2802A2544BD
:1073B000C2F20008C2F20007C2F20009C2F20006DF
:1073C000C2F2000A4FF0010B19E000BF40463946F7
:1073D000FBF7C2FB48463946FEF7F6F8F06900F0C5
:1073E000C9FDF06939460022002300F07BFD00282A
:1073F000284608BFCAF800B000F03EFC2544FFF75D
:10740000DBF91420FFF7E8F90028DFD040463946C1
:107410004A46FFF769F9E1E70000000000407F40BD
:1074200000F062FC04F099FC9FED0B0B53EC102B69
:1074300004F0D0FA04F064FC0446002000F00CFCD8
:1074400000F048FC051900BF284600F015FC254453
:10745000FAE700BF00BF00BF0000000000407F400F
:1074600080B5806B0021C185FDF766FD80BD000001
:1074700010B5846B2068406994F84110212907D128
:1074800010F0800004D00020E084204600F09CF83A
:107490002068406994F84210222907D110F040007A
:1074A00004D00020E085204600F05AF8606C40F0DF
:1074B000100060642046FDF73FFD10BD80B50168F7
:1074C000806B0968C9052FD40021C185016851E886
:1074D000031F026821F4807142E80313002BF5D1E9
:1074E000016851E8051F026821F0010142E8051317
:1074F000002BF5D1016851E8051F026821F0400119
:1075000042E80513002BF5D1202180F84210016BD1
:10751000012909D1016851E8031F026821F0100117
:1075200042E80313002BF5D100214163016B0129CF
:1075300003D1818DFDF7FEFC80BDFDF7D3FF80BD3B
:1075400080B5806B01214163016B012904D1818DDC
:107550004908FDF7EFFC80BDFDF7D8FF80BD0000B6
:10756000016851E8031F026821F4907142E8031397
:10757000002BF5D1016851E8051F026821F00101D7
:1075800042E80513002BF5D1016B01290AD100BF98
:10759000016851E8031F026821F0100142E803135B
:1075A000002BF5D1202180F84210002101637047A3
:1075B00080B50168CA6822F04002CA60202180F8C4
:1075C0004110FDF7B7FF80BD016851E8031F026855
:1075D00021F0C00142E80313002BF5D1202180F8EF
:1075E0004110704744F600010068C4F2000101F543
:1075F0004C420323904208BF0123401A18BF18468B
:107600007047000080B582B090F8421022291ED148
:107610008268B2F5805F02D1016900294AD0816A8F
:10762000B2F5805F07D00AB9026922B102685268D8
:1076300002F07F0201E0026852680A700121826A4A
:1076400011448162C18D01390A04C18501D002B0A3
:1076500080BD0168CA6822F02002CA60CA6822F4AC
:107660008072CA604A6922F001024A61202180F8D2
:10767000421000214163026B012A23D1016300BF44
:10768000016851E8031F026821F0100142E803136A
:10769000002BF5D101680A68D20606D500220192B6
:1076A0000A680192496801910199818DFDF742FCB8
:1076B00002B080BD0168826A49686FF35F21118062
:1076C0000221BCE7FDF70EFF02B080BD10B50446F5
:1076D0000068D4E902C22369016921F440511143D1
:1076E0000161626943EA0C01E3691143C26819430D
:1076F00049F20C639A431143C1604169A26921F4C4
:10770000407141F20043114340F48062C4F201032E
:107710009A42416102D1FCF741FB01E0FCF72CFBEE
:10772000E16963681922B1F5004FA0FB02011CD189
:107730005A00DB0FF8F798FD48F21F51C5F2EB1124
:10774000A0FB01235A096FF0630302FB03003223FD
:1077500003EBC000A0FB01014FF4F87000EA111028
:1077600000EB0210C1F342111AE09A009B0FF8F7E8
:107770007BFD48F21F51C5F2EB11A0FB01235A0912
:107780006FF0630302FB0300322303EB0010A0FB46
:107790000101F02000EA511000EB0210C1F3431187
:1077A00022680843906010BDF0B581B013460027F1
:1077B0000446816283854764222084F84200E06B9E
:1077C00047F2BD4547F241560A462168C0F600051A
:1077D000C0F60006C0E90F5647F27146C0F6000633
:1077E0000431C0E91367FCF735F838B11020606444
:1077F000202084F84200012001B0F0BD00972068ED
:1078000001680091406800900098206950B100BF65
:10781000206850E8030F216840F4807041E80302BB
:10782000002AF5D1206850E8050F216840F00100DA
:1078300041E80502002AF5D1206850E8050F2168CB
:1078400040F0400041E80502002AF5D1002001B0D7
:10785000F0BD000090F84110212923D18168B1F5D5
:10786000805F01D1016931B1016A02684B1C03627A
:107870000978516007E0016A036831F8022B6FF361
:107880005F225A600162C18C01390A04C18418BFA9
:1078900070470068C16821F08001C160C16841F093
:1078A0004001C1607047000080B540F6B040C2F2B0
:1078B0000000FDF755FB80BD10B540F6F844C2F25C
:1078C00000042046FDF74CFB2046FAF7FFFA10BDF6
:1078D00010B540F64054C2F200042046FDF740FBCC
:1078E0002046FAF7F3FA10BDFEE7000000F0FF4073
:1078F000B0F1FF4018BF01207047000000F0FF40CA
:10790000B0F1FF4018BF01207047000020F0004098
:10791000A0F1FF40B0FA80F040097047002848BF4E
:10792000704700F01F01012202FA01F14EF28012AD
:107930004009CEF2000242F82010BFF34F8FBFF390
:107940006F8F7047002848BF704700F01F01012269
:1079500002FA01F14EF200124009CEF2000242F8A2
:10796000201070474EF60C50CEF200000068C0F3B5
:10797000022070474EF6145300F00F02CEF20003BF
:1079800009011A4400F16043B0F1FF3FC8BF03F59D
:1079900064421170704700004EF61F50CEF2000096
:1079A00000210170704700004EF60C51CEF200012C
:1079B0000A684FF6FF031A4060F30A2242F0806023
:1079C00040F0FD700860704770B52DED048B0446E3
:1079D00000284FF0FF0018BF002900F0B380B5EE7B
:1079E000400AB0EE408AF1EE10FA40F3AB8000207E
:1079F000C4F828142073F9F705FE6025D4F828048C
:107A00002844FEF7E5F80835802DF7D1802500BF22
:107A1000D4F828042844FEF7DBF80835A02DF7D168
:107A20004CF61C10C0F6000090E80E00C06804F58B
:107A3000836C04F5387500268CE80E00C4F8240425
:107A4000D4F82814A81901F140020121B0EE480A27
:107A5000FEF794FD3C36F02EF2D16FF0EF0500BF3B
:107A60006619D4F8282406F538700121B0EE480ACA
:107A7000FEF784FDD4F8281406F5F87001F1200211
:107A80000121B0EE480AFEF779FD3C35E8D1B3EEAE
:107A9000049A04F24C40B0EE480AF0EE490AFDF7B1
:107AA00011FF04F26C40B0EE480AF0EE490AFDF70F
:107AB00009FF04F28C40B0EE480AF0EE490AFDF7E7
:107AC00001FF04F2AC40B0EE480AF0EE490AFDF7BF
:107AD000F9FE04F2CC40B0EE480AF0EE490AFDF798
:107AE000F1FE04F2EC40B0EE480AF0EE490AFDF770
:107AF000E9FE04F20C50B0EE480AF0EE490AFDF738
:107B0000E1FE04F22C50B0EE480AF0EE490AFDF70F
:107B1000D9FE04F24C50B0EE480AF0EE490AFDF7E7
:107B2000D1FE04F26C50B0EE480AF0EE490AFDF7BF
:107B3000C9FE04F28C50B0EE480AF0EE490AFDF797
:107B4000C1FE002040B2BDEC048B70BD40F6DB717D
:107B500010EE100AC3F6C97161F31E0000EE100AA0
:107B600070470000F0B581B0F0B1044640F6FC600B
:107B7000C2F200000068A0421FD001F0C5F940F633
:107B80000470C2F200006569076840F60C70C2F22A
:107B90000000066801F0DCF9BD424FF0020018BF9A
:107BA000B5420DD101B0F0BD4FF0500080F3118807
:107BB000BFF36F8FBFF34F8FFEE7002001B0F0BD22
:107BC00046F20400C2F2000085420CD046F21801D1
:107BD0000120C2F20001002D08BF04208D4208BF21
:107BE000042001B0F0BDA06A10B1022001B0F0BDC8
:107BF00094F858100320012908BF022001B0F0BDFD
:107C0000FBF780FFFEF7FAFFFEF7C0F9FEF752F927
:107C1000FEF714F9FEF730F9FEF76EFAFEF7F0FA08
:107C2000FEF710FBFEF78CFAFEF7CEFA00F060F8D4
:107C3000FEF78EF900F086F8FEE7000030EE600AED
:107C400032EE612A20EE020A31EE601A80EE010A5D
:107C500030EE210A70470000EFF3058100291CBFB8
:107C60006FF005007047002804BF0020704780B502
:107C700001F04EFA002080BD10B582B0EFF305810F
:107C800019B16FF0050002B010BD044602F032FBDE
:107C9000211A0129019005DB01A801F063FA0020F7
:107CA00002B010BD6FF0030002B010BD80B502F04D
:107CB0000DFB022808BF80BD08B9032080BD40F23B
:107CC0001420C2F2000000680138B0FA80F04009C8
:107CD00080BD000080B5EFF3058010B102F010FB0D
:107CE00080BD02F007FB80BD4FF47A707047000042
:107CF000EFF3058000281CBF6FF00500704740F2CD
:107D00001420C2F200000168002911BF4FF0FF30BB
:107D1000012101600020704780B5EFF30580002845
:107D20001CBF6FF0050080BD02F0D0FA28B1022818
:107D300005D101F0C1FB002080BD012080BD4FF0C6
:107D4000FF3080BD10B5EFF3058000281CBF6FF039
:107D5000050010BD40F21424C2F20004206801287E
:107D60001CBF4FF0FF3010BDFEF71CFF022020604B
:107D700001F050FB002010BD10B5EFF3058018B1E5
:107D80006FF00504204610BD02F0A0FA02280ED0C4
:107D900080B902F08DFC01284FF001040CD002F0F4
:107DA00095FA002808BF4FF0FF34204610BD00248C
:107DB000204610BD4FF0FF34204610BD10B582B0F4
:107DC0001C46B0FA80F3B1FA81F25B095209EFF375
:107DD000058CBCF1000F42EA030219D0002C18BF39
:107DE0000124224315D10022019201AA01F048FF8B
:107DF00001281AD10198A8B14EF60450CEF2000025
:107E00004FF080510160BFF34F8FBFF36F8F09E0D8
:107E10001AB16FF0030002B010BD224601F06EFEF1
:107E2000012806D1002002B010BD6FF0020002B0A0
:107E300010BD6FF00100002C08BF6FF0020002B00F
:107E400010BD0000B0B582B0144600294FF0000507
:107E5000EFF3058218BF002802D1284602B0B0BD5A
:107E6000002AFAD19CB1A568D5B1E268502A16D390
:107E70002269A2B1D4F814C001FB00F2002394459A
:107E80004FF0000228BF012210D24DB10EE00123B5
:107E900000226AB9E3B1002201F024FC0EE01DB912
:107EA000E2680AB92269C2B100220023002AF1D097
:107EB000A36822690025009501F038FC054655B1FC
:107EC000002C14BF21680021284601F0EBF8C4E71C
:107ED0000025002DF4D10025BFE76269B2FA82F2D5
:107EE0005309D5E7B0B582B01C46B0FA80F3B1FAB9
:107EF00081F5EFF305825B096D09002A43EA05026B
:107F000007D0002C18BF0124224306D06FF00305D0
:107F10002CE0CAB16FF0030528E00022019201AA0B
:107F2000002301F061FD01281CD10198E8B14EF653
:107F30000450CEF200004FF080510160BFF34F8F2C
:107F4000BFF36F8F002511E022460023002501F0CA
:107F500079FC01280AD06FF00105002C08BF6FF0F2
:107F6000020503E06FF0020500E00025284602B09C
:107F7000B0BD000010B5EFF3058119B16FF0050435
:107F8000204610BD00280FBF6FF00304002100241D
:107F900001F018FC204610BD10B50C46EFF305812A
:107FA00000291CBF6FF0050010BD014620F0010044
:107FB00050B111F001010AD1214601F0B7FE0128AC
:107FC00004BF002010BD09E06FF0030010BD214682
:107FD00001F090FF012804BF002010BD6FF00100E8
:107FE000002C08BF6FF0020010BD000070B5EFF369
:107FF0000581B9B90028044614BF60680020010754
:1080000010D494B1A36843B1E26800214F2A4FF025
:10801000000288BF01220AD84BB9E168B1FA81F1A8
:10802000490903E00025284670BD0121002200F027
:1080300001063AB1A168002E0CBF0120042001F016
:108040003FFB06E0C9B1002E0CBF0120042001F067
:108050002BFB054635B1002C14BF216800212846B2
:1080600001F020F8B5FA85F0400986F001010843D7
:1080700008BF45F00105284670BD0025002DEAD156
:10808000F0E7000080B5EFF3058100291CBF6FF019
:10809000050080BD014620F0010040B111F0010152
:1080A00008D100210022002301F0CCFB04E06FF096
:1080B000030080BD01F000FD013818BF6FF0020021
:1080C00080BD0000B0B584B048B3B1F1FF3F26DDFC
:1080D00004464FF0FF300390EFF3058018B30025FE
:1080E0000DF1080C2046012200230295CDF800C0B6
:1080F00002F050F803AB204600210022009502F068
:1081000049F80298D0B14EF60450CEF200004FF07C
:1081100080510160BFF34F8FBFF36F8F0EE06FF0A0
:10812000030003900AE020460122002301F0B4FF7F
:1081300003AB20460021002201F0AEFF039804B0FB
:10814000B0BD00002DE9F04F83B00C46EFF3058180
:1081500029B16FF00507384603B0BDE8F08F05463A
:10816000002849D44FF0000B9246A00758BFAB46F9
:1081700002F0C0F800906FF0010804F001005446CE
:108180000027BAF1000F08BF6FF00208019002E06B
:108190004746002EDFD00020594602AA234602F0AF
:1081A00063F906460128F3D1029807EA050140EA7F
:1081B00001090198002809EA050007D100286FF09D
:1081C000020718BF4F4607D0C5E700BFA8426FF0AF
:1081D000020708BF4F46BED0BAF1000FBBD002F075
:1081E00089F800994F46401A241A4FF0000038BF12
:1081F0000446002ECFD1AEE76FF00307ABE70000D7
:1082000080B502F05DF880BD70B584B08E46002167
:1082100000280391EFF3058146D0002944D1FAB13B
:108220009369002B08BF1823382B16D81179C9077A
:1082300013D15569946811684FEA950C002D08BF59
:108240004FF0800CFCB1D6685C2E1BD3D5B11569FC
:10825000C5B10024012555B91BE0002004B070BD54
:108260000124002118234FF0800C00258DB1946863
:1082700012690294CDE900326246734601F0D0FEE5
:10828000039011E00CB9D4689CB100250024002DA6
:10829000EDD14CB103AC00931FFA8CF273460194FC
:1082A00001F08AFE012802D1039804B070BD0020BD
:1082B000E6E71469B4FA84F46409D6E710B5EFF37D
:1082C000058100291CBF6FF0050010BD044660B198
:1082D0002046FFF747FC042804BF6FF0020010BDE2
:1082E000204600F093FF002010BD6FF0030010BD8A
:1082F000F0B581B00D4646F22C0140F6FC66C2F2A4
:108300000001C2F200060F6831680446081D00F043
:1083100087FD601C0AD14DB13068011D46F2040092
:10832000C2F2000000F0D8FD01B0F0BD3068E419E1
:1083300044600AD340F60C70C2F200000068316855
:10834000043100F0ABFD01B0F0BD40F60470C2F2A4
:10835000000000683168043100F0A0FD45F690701F
:10836000C2F2000001688C4238BF046001B0F0BD69
:1083700070B5044600F0C8FD45F66400C2F2000086
:10838000016840F6FC6501310160C2F20005296810
:1083900045F6F876C2F2000641B1306860B9286847
:1083A000E16AC06A884298BF2C6005E02C600068D2
:1083B000012801D100F0DEF945F67000C2F200009C
:1083C000016801310160616445F67401C2F2000187
:1083D000E06A0A68904288BF086040F6147100EBBA
:1083E0008000C2F2000101EB8000211D00F074FD4D
:1083F00000F0AEFD306880B12868E16AC06A88424A
:1084000028BF70BD4EF60450CEF200004FF08051F0
:108410000160BFF34F8FBFF36F8F70BD70B582B037
:1084200000F072FD46F23006C2F20006306850BB22
:1084300045F63074C2F20004204600F01FFD45F6F8
:108440004475C2F20005284600F018FD40F60070A1
:10845000C2F20000046040F61070C2F2000040F664
:10846000086240F6A86305600025C2F20002C2F26D
:1084700000030A201021009501F058F9306010B176
:1084800003A100F00FFE00F063FD02B070BD00BF5D
:10849000546D725100000000F0B581B045F66805DA
:1084A000C2F200052868E0B146F2180645F66407F6
:1084B000C2F20006C2F2000700F026FDF068C468B0
:1084C000201D00F0ADFC386801383860286801389C
:1084D000286000F03DFD204600F058F8286800288C
:1084E000EAD101B0F0BD000080B5026C002A08BFDF
:1084F00080BDD0E902C31344C360634524BF036851
:10850000C360C36808461946F7F726FF80BD000020
:1085100070B5866B036C0446E3B115461AB3E06888
:108520001A46F7F719FFE168206C2268091A914290
:10853000E16003D2A16840420844E060A81EB0FA9E
:1085400080F040093146002E18BF01210840361A3C
:10855000002516E02068002598B9A06801F0CCFF3E
:10856000A56005460DE060681A46F7F7F5FE216C38
:10857000D4E90102002508446060904224BF2068CD
:108580006060711C2846A16370BD000010B50446F0
:1085900090F85900022808BF10BD012803D030B957
:1085A000206B00F0EDFC204600F0EAFC10BD4FF01F
:1085B000500080F31188BFF36F8FBFF34F8F00BF60
:1085C000FEE70000416A00290FBF0020006B006831
:1085D000C0F138007047000040F60071C2F200019F
:1085E00009680A68B2FA82F35B090360002A0EBFC9
:1085F0000020C8680068704741F65840C2F2000089
:10860000C21D22F0070210F0070CA0EB020318BFF6
:10861000104645F6FC72C2F200020021C2E90001D8
:108620004FF47052BCF1000F18BF03F570520244B2
:10863000083A40F6087322F00702C2F200031A60FB
:10864000C2E90011111A1A68C0E9002145F68C70C0
:10865000C2F20000016045F68470C2F200000160C1
:1086600045F65870C2F20000012101707047000009
:1086700040F614744EF60455C2F20004CEF2000522
:108680004FF08056FFF708FF20680228FAD32E60CB
:10869000BFF34F8FBFF36F8FF4E70000002808BFD0
:1086A000704780B500210160C0E90211002100225D
:1086B000002301F0C7F8BDE880407047B0B5049DC5
:1086C000002914BF2A602D60C5E90F012846012149
:1086D0001C4601F077F885F84C40B0BD2DE9F04715
:1086E0000A9C8246206B16460F46DDE90859910028
:1086F000A5229846F7F775FE206B00EB8600A0F1E7
:10870000040020F007067FB104F13400002100BF0F
:108710007A5C42547A5C1AB10F2901F10101F7D356
:10872000002084F8430002E0002084F83400002791
:10873000201D372D28BF3725E562C4E9135700F007
:10874000A9FB04F1180000F0A5FBC5F13800A061F9
:1087500030465146424624616462676584F8587029
:1087600000F04AFBB9F1000F206018BFC9F80040C3
:10877000BDE8F087B0B540F614750024C2F20005DC
:10878000281900F07BFB1434B4F58C6FF8D145F652
:108790005C74C2F20004204600F070FB45F6707570
:1087A000C2F20005284600F069FB45F6A470C2F24B
:1087B000000000F063FB46F21800C2F2000000F077
:1087C0005DFB46F20400C2F2000000F057FB40F6E9
:1087D0000470C2F20000046040F60C70C2F20000A7
:1087E0000560B0BD80B545F6FC72C2F2000200BF64
:1087F000114612688242FBD3D1F804C001EB0C038E
:10880000834203D14068604448600846D0F804C001
:1088100000EB0C03934201D013460BE040F60873C3
:10882000C2F200031B689A4204D0D2E9003E0EEB6C
:108830000C0242608142036018BF086080BD0000E6
:1088400080B58C46014641F804CF9445006108D9B3
:108850009A4201D29C4511D240F60070C2F200004B
:1088600007E08069D21A824208D240F61070C2F244
:108870000000006800F012FB002080BD012080BDD8
:1088800010B5044600F040FBA06BB0FA80F044093C
:1088900000F05EFB204610BD10B5044600F034FB2E
:1088A000A06BE16B401AB0FA80F0440900F050FB75
:1088B000204610BD08480068006880F308884FF023
:1088C000000080F3148862B661B6BFF34F8FBFF328
:1088D0006F8F00DF00BF00BF08ED00E070B582B011
:1088E00040F60072C2F2000212680546D2680E46D7
:1088F000D468201D00F094FA94F82800410704D4AD
:1089000000F0FE0084F8280010E0A069324641190A
:1089100020462B46FFF794FF40B100262046002159
:108920002A460023009601F087FF20B1216A2046E5
:10893000884702B070BD4FF0500080F31188BFF33C
:108940006F8FBFF34F8F00BFFEE700002DE9F041AE
:1089500086B046F23007C2F20007386802A900224A
:108960004FF0000801F0CAF800286AD001AC02AD4F
:108970000BE000F0FE0086F8280000BF38682946AA
:10898000002201F0BBF800285BD00298B0F1FF3F55
:1089900003DCDDE903200599904702980028EDD417
:1089A000049E706910B1301D00F03AFA204600F0C4
:1089B000B3F802990929E1D80246DFE801F0080876
:1089C00008052A390808052A96F82800D1E796F8FC
:1089D0002800039BB16940F0010086F82800194483
:1089E0003046FFF72DFF0028C8D0316A304688474F
:1089F00096F828004007C1D50398B16900230A18EA
:108A000030460021CDF8008001F016FF0028B5D1D6
:108A100023E096F8280040F00101039886F828101A
:108A2000B06188B1811830461346FFF709FFA5E70A
:108A300096F8280081073FF59CAF304600F0A0FA79
:108A40009CE706B0BDE8F0814FF0500080F311883C
:108A5000BFF36F8FBFF34F8FFEE74FF0500080F3EF
:108A60001188BFF36F8FBFF34F8F00BFFEE7000089
:108A700070B582B00E46044600F01EFD01A800F05D
:108A80004BF8019919B101F013FE02B070BD054613
:108A90004EB9A54207D301F00BFE20462946FFF749
:108AA0001DFF02B070BD4EB140F61070C2F2000062
:108AB00000680068B0FA80F0420900E0002246F247
:108AC0003000C2F200000068611B00F0FFFA01F004
:108AD000EFFD0028D9D14EF60450CEF200004FF041
:108AE00080510160BFF34F8FBFF36F8F02B070BD35
:108AF00040F60470C2F200000168096821B1006804
:108B0000C068C068406801E04FF0FF3045F69071E2
:108B1000C2F200010860704770B5044601F0EAFB3C
:108B200040F6F866C2F2000631680546884203D274
:108B300000F008F8012000E00020206028463560A1
:108B400070BD00002DE9F04182B040F60077C2F21E
:108B500000073868016891B34FF0000809E000BFD2
:108B6000606038682946246100F098F93868016827
:108B700029B3C068C4680668251D284600F050F96E
:108B8000216A2046884794F828004007EED5A0695E
:108B90003044B042E4D82046002132460023CDF8CC
:108BA000008001F049FE0028E0D14FF0500080F332
:108BB0001188BFF36F8FBFF34F8F00BFFEE740F602
:108BC0001071C2F200010A6808603A6002B0BDE8A4
:108BD000F081000081B00020009040F20010C2F24D
:108BE000000000684FF0500181F31188BFF36F8FD0
:108BF000BFF34F8F013001D0FEE700BF009800287F
:108C0000FCD001B07047000082B001AC2046FFF7F5
:108C1000E3FC0199FFF72CFFFFF798FEF6E7000051
:108C2000F0B581B0044600F06FF994F94560012E6B
:108C30000FDB04F1240500BF286850B1284601F07D
:108C4000EFFC002818BF00F051FB70B2013E012874
:108C5000F2DCFF2684F8456000F07AF900F054F960
:108C600094F94470012F0EDB04F11005286850B10F
:108C7000284601F0D5FC002818BF00F037FB78B279
:108C8000013F0128F2DC84F8446000F061F901B092
:108C9000F0BD00002DE9F04381B0044600F00CFC6B
:108CA00040F60876C2F200063068002808BFFFF7D9
:108CB000A3FC45F65878C2F2000898F80000002896
:108CC00018BF4FF0004020420DD0002401F0F0FC0E
:108CD00060071ED04FF0500080F31188BFF36F8FF4
:108CE000BFF34F8FFEE7C4B114F0070004F1080191
:108CF0001EBF081A00F108015FEA41700ED04FF064
:108D0000500080F31188BFF36F8FBFF34F8F00BF08
:108D1000FEE7204601B0BDE8F083002145F68479E6
:108D2000C2F20009D9F800004A1E8242CDD245F6AF
:108D3000FC70C2F2000005682F4657F8042F8A42E3
:108D400011D22B685BB100BF1F4657F8042F28468D
:108D50001D468A4207D22B68002BF5D103E045F669
:108D6000FC70C2F2000033689D42AED004682B68EC
:108D7000521A112A036010D36818430709D04FF024
:108D8000500080F31188BFF36F8FBFF34F8F00BF88
:108D9000FEE742603960FFF725FD45F68C703968C3
:108DA000D9F80020C2F200000368511A9942C9F8AC
:108DB000001038BF016098F80000396800284FF0B3
:108DC000000018BF41F00041286045F69870C2F2DB
:108DD0000000026808343960511C016076E7000029
:108DE00040F6FC60C2F20000016819B101680A6D2A
:108DF00001320A6500687047034648F6D530C0F670
:108E000000004FF0807C21F0010103E903106FF0B6
:108E1000020043F8240CA3F1440043F8202C7047CF
:108E2000D0E9013201699A60D1F804C082688445B2
:108E3000536008BF4A600022026108680138086078
:108E40000868704745F67823C2F20003036045F6D0
:108E50007800C2F2000008608020106070470000B7
:108E600045F6D463C2F20003036045F6D420C2F293
:108E7000000008604FF48070106070474FF0FF31C1
:108E8000024642F8081F00214260C0E90322016047
:108E900070470000002101617047000080B5D1F8E3
:108EA00000C01CF1010207D000F108039E465B6878
:108EB0001A686245FAD901E0D0F810E0DEF8042023
:108EC00008614A609160C1F808E0CEF804100168BA
:108ED0000131016080BD0000D0F800C04368086126
:108EE0009A684B608A609A68996051600CF1010140
:108EF00001607047DFF80C00016841F47001016007
:108F0000704700BF88ED00E04FF0500080F31188FB
:108F1000BFF36F8FBFF34F8F40F20010C2F200001B
:108F200001684A1C026001B170474EF60450CEF24F
:108F300000000068000608BF70474FF0500080F343
:108F40001188BFF36F8FBFF34F8F00BFFEE70000A4
:108F500040F20010C2F20000016839B1013901602D
:108F600018BF7047002080F3118870474FF0500001
:108F700080F31188BFF36F8FBFF34F8FFEE70000C0
:108F8000B0B5002808BFB0BD044645F65870C2F21F
:108F90000000007854F8041C002818BF4FF000406F
:108FA00008420CD0A4F108052A6892B14FF0500095
:108FB00080F31188BFF36F8FBFF34F8FFEE74FF041
:108FC000500080F31188BFF36F8FBFF34F8F00BF46
:108FD000FEE721EA000044F8040C00F06DFA45F6C3
:108FE0008471C2F2000154F8040C0A68104408604D
:108FF0002846FFF7F7FB45F69C70C2F200000168B7
:109000000131016001F054FBB0BD00004EF21000D0
:10901000CEF2000000210160816040F20001C2F246
:109020000001096844F6D352C1F26202A1FB0212A8
:109030004FF0FF3101EB9211416007210160704751
:10904000EFF30580102814D34EF2F031CEF2000178
:10905000405C45F65801C2F200010978884208D206
:109060004FF0500080F31188BFF36F8FBFF34F8F25
:10907000FEE74EF60C50CEF2000045F65C010068AB
:10908000C2F20001096800F4E060884298BF7047AE
:109090004FF0500080F31188BFF36F8FBFF34F8FF5
:1090A000FEE7000045F6B87C0022C2F2000C00BFCB
:1090B0005CF8323023B10132082A08BF7047F7E765
:1090C0000CEBC2034CF832105860704770B515466F
:1090D0000E460446FFF718FF94F84400FF2804BF2B
:1090E000002084F8440094F84500FF2804BF0020C5
:1090F00084F84500FFF72CFFA06B28B904F1240089
:1091000031462A4600F014F92046FFF789FD70BD6C
:1091100010B5D8B1044645F66C00C2F200000068F4
:1091200048B14FF0500080F31188BFF36F8FBFF349
:109130004F8F00BFFEE700F0BFF920460021FFF788
:10914000D7F801F0B5FA002818BF10BD4EF604504C
:10915000CEF200004FF080510160BFF34F8FBFF39C
:109160006F8F10BDB0B590B10D46D1B1044645F634
:109170006C00C2F200000068E8B14FF0500080F3CC
:109180001188BFF36F8FBFF34F8F00BFFEE74FF023
:10919000500080F31188BFF36F8FBFF34F8F00BF74
:1091A000FEE74FF0500080F31188BFF36F8FBFF3DD
:1091B0004F8F00BFFEE700F07FF946F22C00C2F2AD
:1091C000000000682268904202EB050102D2914241
:1091D00002D309E0914201D3814205D92160081AE6
:1091E0000021FFF785F800E0216001F061FA002816
:1091F00018BFB0BD4EF60450CEF200004FF08051C3
:109200000160BFF34F8FBFF36F8FB0BD70B50446E1
:10921000FFF77AFE40F6FC66002CC2F2000608BF9B
:109220003468251D2846FFF7FBFDA06A18B104F13C
:109230001800FFF7F5FD45F67000C2F20000016866
:1092400001310160306884420CD045F66400C2F2FE
:1092500000000168013901602046FFF797F9FFF728
:1092600047FC0DE046F21800C2F200002946FFF765
:1092700033FE45F66800C2F200000168013101606A
:10928000FFF766FE45F6F870C2F200000068E8B12C
:109290003068844218BF70BD45F66C00C2F2000011
:1092A000006840B14FF0500080F31188BFF36F8F1A
:1092B000BFF34F8FFEE74EF60450CEF200004FF0A2
:1092C00080510160BFF34F8FBFF36F8F70BD0000FF
:1092D00045F69471C2F200010968016046F22C0162
:1092E000C2F20001096841607047000046F2380090
:1092F000C2F20000012101607047000010B568B1A2
:109300000C4640F6FC61C2F2000109681831FFF713
:10931000C5FD20460121FEF7EBFF10BD4FF05000C8
:1093200080F31188BFF36F8FBFF34F8FFEE700000C
:10933000B0B590B10D4640F6FC61C2F2000109687B
:1093400014461831FFF7C8FD002C18BF4FF0FF3549
:1093500028462146FEF7CCFFB0BD4FF0500080F309
:109360001188BFF36F8FBFF34F8F00BFFEE7000080
:1093700070B528B3026D04461AB3E06C884238BF5A
:109380000846012A1CD1E16A814208BF70BD40F63F
:10939000FC62C2F200021268A2421CD0A269E06222
:1093A000002A5CBFC0F13800A06140F61476606905
:1093B00001EB8101C2F2000606EB8101884214D064
:1093C00070BD4FF0500080F31188BFF36F8FBFF373
:1093D0004F8F00BFFEE74FF0500080F31188BFF3BE
:1093E0006F8FBFF34F8F00BFFEE7251D2846FFF7A5
:1093F00017FD45F67401C2F20001E06A0A68904266
:1094000088BF086000EB800006EB80002946FFF76C
:1094100063FD70BD10B586B0002405A804A903AA99
:10942000CDE90444FFF70EFDDDE903200599002393
:10943000CDE9010148F27160C0F600001CA1009462
:1094400000F0EEFD45F68871C2F20001086010B12F
:1094500001F0B8F90446601C20D0012C1CD14FF05B
:10946000500080F31188BFF36F8FBFF34F8F45F625
:109470009070C2F200004FF0FF31016045F6F870C5
:10948000C2F200000121016046F22C00C2F200008D
:109490000021016000F066F806B010BD4FF05000EA
:1094A00080F31188BFF36F8FBFF34F8FFEE700BFCC
:1094B00049444C450000000045F66C00C2F2000033
:1094C000016801310160704745F66C00C2F200008E
:1094D000006830B146F23800C2F20000012101609C
:1094E000704746F23800C2F20000002145F6740CC5
:1094F0000160C2F2000CDCF8001040F6147201EBBF
:109500008103C2F2000252F8230048B902EB830043
:10951000A0F11403D9B153F8140901390028F9D086
:1095200001EB810002EB800252F8040F4368101D2A
:109530008342136001D158681060106840F6FC62E5
:10954000C068C2F200021060CCF8001070474FF003
:10955000500080F31188BFF36F8FBFF34F8F00BFB0
:10956000FEE7000080B582B04EF20040CEF200006F
:109570004CF27021C4F20F11D0F800294B1C9A4212
:1095800009D14FF0500080F31188BFF36F8FBFF304
:109590004F8F00BFFEE7D0F800298A4209D14FF073
:1095A000500080F31188BFF36F8FBFF34F8F00BF60
:1095B000FEE7017845F658020191FF21017001781C
:1095C000C2F200028DF803109DF8031001F0500163
:1095D000117045F65C01C2F2000107220A609DF994
:1095E0000320B2F1FF3F0CDC0A6800BF9DF8033096
:1095F000013A5B008DF803309DF90330002BF5D460
:109600000A600A68032A2DD14FF4E06303EA0222BC
:109610000A6001990170D0F8201941F47001C0F876
:109620002019D0F8201941F07041C0F82019FFF737
:10963000EDFC40F20010C2F2000000210160FFF7D3
:1096400059FC4EF63470CEF20000016841F0404102
:109650000160FFF72FF9FFF737FFFFF7BBFA002094
:1096600002B080BD4FF0500080F31188BFF36F8FC0
:10967000BFF34F8FFEE7000080B54FF0500080F33E
:109680001188BFF36F8FBFF34F8F00F043FE30B1EF
:109690004EF60450CEF200004FF0805101600020E1
:1096A00080F3118880BD000010B502460120002122
:1096B00000F018F80446FEF7F1FF204610BD000048
:1096C00010B582B00B468446012000210022CDF85F
:1096D00000C000F02BF80446FEF7E0FF204602B081
:1096E00010BD0000F0B581B0B0B105464843503020
:1096F00014460E46FFF7CEFA074650B1002007F198
:10970000500287F846002846314623460097FEF768
:10971000D5FF384601B0F0BD4FF0500080F31188FE
:10972000BFF36F8FBFF34F8FFEE70000B0B582B07D
:1097300068B11D46ABB1F1B9EAB14FF0500080F30A
:109740001188BFF36F8FBFF34F8F00BFFEE74FF05D
:10975000500080F31188BFF36F8FBFF34F8F00BFAE
:10976000FEE74FF0500080F31188BFF36F8FBFF317
:109770004F8F00BFFEE751B14AB94FF0500080F360
:109780001188BFF36F8FBFF34F8F00BFFEE75023E9
:109790000193019B502B0AD1069B019C012485F863
:1097A00046400095FEF78AFF284602B0B0BD4FF054
:1097B000500080F31188BFF36F8FBFF34F8F00BF4E
:1097C000FEE7000070B5F8B104460E46FFF79CFBBB
:1097D0002068D4E90F12002502FB0103013901FBC7
:1097E0000201A563C4E90103FF20E16084F844009D
:1097F00084F8450004F110007EB1FFF73FFB04F14F
:109800002400FFF73BFB18E04FF0500080F3118875
:10981000BFF36F8FBFF34F8FFEE7016869B100F0B0
:10982000FFFE50B14EF60450CEF200004FF08051D2
:109830000160BFF34F8FBFF36F8FFFF789FB0120EC
:1098400070BD00002DE9F04F83B00292B8B11D4603
:109850000E460446E9B1022D03D1E06B012840F029
:109860009A8000F033FD00BB0298F0B14FF0500039
:1098700080F31188BFF36F8FBFF34F8FFEE74FF078
:10988000500080F31188BFF36F8FBFF34F8F00BF7D
:10989000FEE7206C0028DED04FF0500080F31188E6
:1098A000BFF36F8FBFF34F8FFEE7FFF72DFBA06B6A
:1098B000022D58D0E16B884255D304F110080120E5
:1098C0006F464FF0000B0DF108094FF0805A00BFB2
:1098D0000299002900F07B80C00702D03846FFF7CC
:1098E000F7FCFFF735FBFFF7E7FDFFF70DFB94F8FB
:1098F0004400FF2808BF84F844B094F84500FF28CE
:1099000008BF84F845B0FFF723FB3846494600F00E
:109910000FFB00285ED12046FEF7BEFFA0B10299E2
:109920004046FFF7EBFC2046FFF77AF900F0C0FE57
:1099300078B94EF60450CEF20000C0F800A0BFF394
:109940004F8FBFF36F8F04E02046FFF769F900F0F7
:10995000AFFEFFF7D9FAA06B022D04D0E16B88426D
:109960004FF00000B4D2204631462A46FEF7D0FD23
:1099700054F8241FC9B1204600F052FE08B34EF639
:109980000450CEF200004FF080510160BFF34F8FC2
:10999000BFF36F8F15E04FF0500080F31188BFF3D5
:1099A0006F8FBFF34F8F00BFFEE750B14EF60450EC
:1099B000CEF200004FF080510160BFF34F8FBFF334
:1099C0006F8FFFF7C5FA012003B0BDE8F08FFFF7F6
:1099D000BFFA04E02046FFF723F900F069FE0020FB
:1099E00003B0BDE8F08F00002DE9F04381B0E8B18D
:1099F0001E46914605460F4609B3022E02D1E86B7A
:109A0000012837D1FFF71CFBEFF311884FF050000E
:109A100080F31188BFF36F8FBFF34F8FA86B022EB7
:109A200019D0E96B884216D300203FE04FF0500078
:109A300080F31188BFF36F8FBFF34F8FFEE7286C61
:109A40000028DAD04FF0500080F31188BFF36F8FF9
:109A5000BFF34F8FFEE795F84540A86B284639467F
:109A60003246FEF755FDFF2C0DD0601C85F84500F1
:109A700001201BE04FF0500080F31188BFF36F8F7F
:109A8000BFF34F8FFEE755F8240F70B1284600F062
:109A9000C7FD0146B9F1000F4FF0010006D00029C3
:109AA0001CBF0120C9F8000000E0012088F31188E4
:109AB00001B0BDE8F0830000B0B5A8B185680446E8
:109AC00000F0FEFB85421CBF0020B0BDE0680138FD
:109AD000E0601CBF0120B0BD204600210022002311
:109AE000FFF7B0FE0120B0BD4FF0500080F31188A9
:109AF000BFF36F8FBFF34F8FFEE700002DE9F04FEC
:109B000085B0049298B10C460546002900F0A58066
:109B100000F0DCFBA8B9049898B14FF0500080F336
:109B20001188BFF36F8FBFF34F8F00BFFEE74FF079
:109B3000500080F31188BFF36F8FBFF34F8F00BFCA
:109B4000FEE705F1240005F11009019002AF0DF1C7
:109B5000100A4FF000080AE02846FFF761F800F00D
:109B6000A7FD2846FEF78CFE002840F08480FFF712
:109B7000CBF9D5F838B0BBF1000F1DD028462146EF
:109B8000FEF7B2FCABF10100A863286970B148464A
:109B900000F046FD50B14EF60450CEF200004FF0FA
:109BA00080510160BFF34F8FBFF36F8FFFF7D0F984
:109BB00000200126A0B95FE0049850B1B8F1000F71
:109BC00002D13846FFF784FB4FF00108012038B975
:109BD00052E0FFF7BDF90026002000284CD000BF5E
:109BE000FFF7B6F9FFF768FCFFF78EF995F8440028
:109BF000FF2804BF002085F8440095F84500FF28A1
:109C000004BF002085F84500FFF7A2F93846514609
:109C100000F08EF900289FD12846FEF731FEB0B142
:109C200004990198FFF76AFB2846FEF7F9FF00F058
:109C30003FFD00289BD14EF60450CEF200004FF0BD
:109C400080510160BFF34F8FBFF36F8F8FE72846BE
:109C5000FEF7E6FF00F02CFD89E7286C00283FF4B2
:109C600057AF4FF0500080F31188BFF36F8FBFF3F1
:109C70004F8F00BFFEE70026304605B0BDE8F08FED
:109C80002DE9F04381B000B3914605460E4631B34D
:109C9000FFF7D6F9EFF311884FF0500080F31188E9
:109CA000BFF36F8FBFF34F8FAC6B24B395F8447045
:109CB00028463146FEF718FC601EFF2FA8631CD013
:109CC000781C85F8440001202AE04FF0500080F312
:109CD0001188BFF36F8FBFF34F8F00BFFEE7286C73
:109CE0000028D5D04FF0500080F31188BFF36F8F5C
:109CF000BFF34F8FFEE7002012E055F8100F70B150
:109D0000284600F08DFC0146B9F1000F4FF001002C
:109D100006D000291CBF0120C9F8000000E0012086
:109D200088F3118801B0BDE8F08300002DE9F04F01
:109D300085B0049158B10446006C90B14FF05000CA
:109D400080F31188BFF36F8FBFF34F8FFEE74FF0A3
:109D5000500080F31188BFF36F8FBFF34F8F00BFA8
:109D6000FEE700F0B3FA50B9049840B14FF050004C
:109D700080F31188BFF36F8FBFF34F8FFEE704F1BD
:109D8000240004F1100501904FF0000802AF0DF11E
:109D9000100A4FF000094FF0000B0AE02046FEF7D2
:109DA0003FFF00F085FC2046FEF76AFD002840F0EA
:109DB0007F80FFF7A9F8A06BF0B10138A06320689D
:109DC00010B9FFF70DF8A060286870B1284600F0C0
:109DD00027FC50B14EF60450CEF200004FF08051F7
:109DE0000160BFF34F8FBFF36F8FFFF7B1F801260C
:109DF0000020B8B96FE000BF049850B1BBF1000F6C
:109E000002D13846FFF764FA4FF0010B012048B940
:109E100061E0B9F1000F62D1FFF79AF80020002647
:109E2000002858D0FFF794F8FFF746FBFFF76CF8CF
:109E300094F84400FF2808BF84F8448094F8450053
:109E4000FF2808BF84F84580FFF782F8384651465E
:109E500000F06EF80028A1D12046FEF711FD28B9C8
:109E60002046FEF7DDFE00F023FCA2E7206838B9AB
:109E7000FFF74AF8A06800F089FB8146FFF768F811
:109E800004990198FFF73AFA2046FEF7C9FE00F060
:109E90000FFC00287FF48DAF4EF60450CEF2000088
:109EA0004FF080510160BFF34F8FBFF36F8F80E79A
:109EB000B9F1000F0ED0FFF727F82046FEF782FB1E
:109EC000A168024608461146FFF752FAFFF740F82C
:109ED000002600E00026304605B0BDE8F08F4FF0C8
:109EE000500080F31188BFF36F8FBFF34F8F00BF17
:109EF000FEE7000070B568B1866804460D4600F0C4
:109F0000DFF986420FD020462946FFF70FFF58B9E8
:109F1000002070BD4FF0500080F31188BFF36F8FA9
:109F2000BFF34F8FFEE70120E1680131E16070BDB2
:109F3000B0B5D0B10D4611B30446FEF7E5FF46F2C9
:109F40002C00C2F2000001682868421C21D045F6AE
:109F500094736268C2F20003D3F800C091421AD32E
:109F600023689C4517D0012422E04FF0500080F375
:109F70001188BFF36F8FBFF34F8F00BFFEE74FF025
:109F8000500080F31188BFF36F8FBFF34F8F00BF76
:109F9000FEE700240CE0891A884206D9401A28609E
:109FA0002046FFF795F9002402E0002001242860F4
:109FB000FEF7CEFF2046B0BD2DE9F04383B0074643
:109FC0009000984615468946FEF764FE78B106462D
:109FD0005C20FEF75FFE38B10446066354B94FF0CB
:109FE000FF3003B0BDE8F0833046FEF7C9FF002420
:109FF000002CF4D0DDE90A10002284F85920CDE9C4
:10A000000010384649462A4643460294FEF766FB4E
:10A010002046FEF7ADF9012003B0BDE8F083000053
:10A0200070B586B00B9CCCB10C9E06B35C25049534
:10A03000049D5C2D25D1049DDDF828C0022586F8FD
:10A04000595005AD3463CDE900C50296FEF746FBD5
:10A050003046FEF78DF9059806B070BD4FF0500000
:10A0600080F31188BFF36F8FBFF34F8FFEE74FF080
:10A07000500080F31188BFF36F8FBFF34F8F00BF85
:10A08000FEE74FF0500080F31188BFF36F8FBFF3EE
:10A090004F8F00BFFEE70000F0B581B0D0B11D4684
:10A0A000174604460E46FEF72FFF002D1CBF606DBD
:10A0B000286094F858000221042F84F8581012D810
:10A0C0000125DFE807F023031C262000616D3143E2
:10A0D00061651FE04FF0500080F31188BFF36F8F70
:10A0E000BFF34F8FFEE7616D013113D04FF0500089
:10A0F00080F31188BFF36F8FBFF34F8FFEE7616D61
:10A100000131616506E0022803D1002501283CD118
:10A1100003E066650125012837D1261D3046FEF78C
:10A120007FFE45F67401C2F20001E06A0A689042BF
:10A1300088BF086040F6147100EB8000C2F2000195
:10A1400001EB80003146FEF7C7FEA06A48B14FF030
:10A15000500080F31188BFF36F8FBFF34F8F00BFA4
:10A16000FEE740F6FC61C2F20001E06A0968C96AD4
:10A1700088420AD94EF60450CEF200004FF08051CA
:10A180000160BFF34F8FBFF36F8FFEF7E1FE2846EC
:10A1900001B0F0BD2DE9F04120B31D46174604463D
:10A1A0000E46FEF74DFFEFF311884FF0500080F39D
:10A1B0001188BFF36F8FBFF34F8F002D1CBF606DF1
:10A1C000286094F858000221042F84F8581012D8FF
:10A1D0000125DFE807F023031C262000616D3143D1
:10A1E00061651FE04FF0500080F31188BFF36F8F5F
:10A1F000BFF34F8FFEE7616D013113D04FF0500078
:10A2000080F31188BFF36F8FBFF34F8FFEE7616D4F
:10A210000131616506E0022803D10025012849D1FA
:10A2200003E066650125012844D1A06A48B14FF0DA
:10A23000500080F31188BFF36F8FBFF34F8F00BFC3
:10A24000FEE745F66C00C2F20000006830B145F64A
:10A25000A47004F11801C2F2000015E0261D30467A
:10A26000FEF7DEFD45F67401C2F20001E06A0A68FD
:10A27000904288BF086040F6147100EB8000C2F283
:10A28000000101EB80003146FEF726FE40F6FC613E
:10A29000C2F20001E06A0968C96A88420AD90698D0
:10A2A00000281CBF0121016046F23800C2F2000004
:10A2B0000121016088F311882846BDE8F081000083
:10A2C00040F6FC60C2F200000068704745F6F87086
:10A2D000C2F200000068002804BF0120704745F664
:10A2E0006C00C2F200000068B0FA80F04009400043
:10A2F0007047000046F22C00C2F200000068704770
:10A3000080B5FEF79DFE46F22C00C2F20000006808
:10A3100080BD00002DE9F04F81B045F66C00C2F21F
:10A320000000006840B145F6A070C2F2000001686C
:10A3300000240131016092E046F22C00C2F20000DC
:10A3400001684E1C066021D340F60470C2F2000082
:10A350000168096849B14FF0500080F31188BFF3DC
:10A360006F8FBFF34F8F00BFFEE740F60C72C2F253
:10A37000000201681368036045F694701160C2F230
:10A380000000016801310160FEF7B2FB45F69071F3
:10A39000C2F20001086840F6FC6A40F61478864272
:10A3A000C2F2000AC2F2000801D2002445E040F6E1
:10A3B0000477C2F2000738680024006898B345F6B5
:10A3C000740BC2F2000B19E0D9F82C00DBF8001076
:10A3D000884288BFCBF8000000EB800008EB8000CB
:10A3E0002946FEF779FDD9F82C00DAF80010C96A81
:10A3F0003A68884228BF01241068B8B13868C0683C
:10A40000D0F80C904D4655F8040F864210D32846DC
:10A41000FEF706FDD9F828000028D5D009F118006C
:10A42000FEF7FEFCD0E74FF0FF3005E04FF0FF30C5
:10A4300045F69071C2F200010860DAF80000C06AC7
:10A4400000EB800058F82000012846F23800C2F2E4
:10A45000000088BF01240068002818BF012420469E
:10A4600001B0BDE8F08F00002DE9F0411E46154611
:10A4700088460746FEF748FD40F6FC64C2F2000439
:10A48000206890F85800022819D02068416D21EA10
:10A490000701416520684FF0010180F8581076B13E
:10A4A00030460121FDF724FF4EF60450CEF20000A5
:10A4B0004FF080510160BFF34F8FBFF36F8FFEF7F6
:10A4C00047FDFEF721FD15B12068406D286020682A
:10A4D000002590F858100020022905D12168012597
:10A4E0004A6D22EA08024A65216881F85800FEF7A1
:10A4F0002FFD2846BDE8F081B0B580B1044640F696
:10A50000FC60C2F200000068A0420AD04FF0500088
:10A5100080F31188BFF36F8FBFF34F8FFEE70020EA
:10A52000B0BD206D38B3013820654FF0000018BF72
:10A53000B0BDE16AE26C91421CD0251D2846FEF7B1
:10A540006FFCE06CC0F13801A16145F67401E06276
:10A55000C2F200010A68904288BF086040F6147198
:10A5600000EB8000C2F2000101EB80002946FEF7FB
:10A57000B3FC0120B0BD4FF0500080F31188BFF351
:10A580006F8FBFF34F8F00BFFEE70000F0B581B0C3
:10A5900000B340F6FC66C2F200060446C06A3168A9
:10A5A000C96A884219D2A169002904D43168C96AEC
:10A5B000C1F13801A16140F61477616900EB8000B8
:10A5C000C2F2000707EB800081420FD03068C06AFA
:10A5D000E06221E0002001B0F0BDE16C3068C26AA9
:10A5E0000020914238BF012001B0F0BD251D284652
:10A5F000FEF716FC306845F67401C06AC2F200012D
:10A60000E0620A68904288BF086000EB800007EBB8
:10A6100080002946FEF760FC012001B0F0BD00007B
:10A62000B0B5C068C5687DB105F118042046FEF7D5
:10A63000F7FB45F66C00C2F20000006868B145F611
:10A64000A470C2F200001DE04FF0500080F31188AA
:10A65000BFF36F8FBFF34F8FFEE72C1D2046FEF731
:10A66000DFFB45F67401C2F20001E86A0A68904215
:10A6700088BF086040F6147100EB8000C2F2000150
:10A6800001EB80002146FEF727FC40F6FC61C2F298
:10A690000001E86A0968C96A884291BF002046F251
:10A6A0003801C2F20001012088BF0860B0BD00007F
:10A6B0002DE9F04F81B045F66C04C2F20004206829
:10A6C00068B1FEF721FC206801382060206880B165
:10A6D0000024FEF73DFC204601B0BDE8F08F4FF0AE
:10A6E000500080F31188BFF36F8FBFF34F8F00BF0F
:10A6F000FEE745F66400C2F20000006800285DD065
:10A7000045F6A476C2F20006306846F23808C2F276
:10A71000000890B345F6740740F6147940F6FC6BD8
:10A72000C2F20007C2F20009C2F2000B4FF0010AA8
:10A73000F068C56805F11800FEF772FB2C1D204675
:10A74000FEF76EFBE86A3968884288BF386000EB24
:10A75000800009EB80002146FEF7BEFBE86ADBF8CB
:10A760000010C96A884228BFC8F800A030680028D5
:10A77000DED1002D18BFFEF7BBF945F6A074C2F27A
:10A780000004256855B10126FFF7C4FD002818BF55
:10A79000C8F80060013DF7D100202060D8F8000023
:10A7A00070B14EF60450CEF200004FF080510160BF
:10A7B000BFF34F8F0124BFF36F8F8AE7002488E730
:10A7C000002486E780B586B0FDF728FE46F230000B
:10A7D000C2F20000006808B30020CDE9040005A81B
:10A7E00004A903AAFEF73CFBDDE903200221DDF802
:10A7F00014C0CDE9001048F60940C0F600000CA1D5
:10A800000023CDF808C0FFF70BFC46F23401C2F27A
:10A810000001086010B1012006B080BD4FF050006B
:10A8200080F31188BFF36F8FBFF34F8FFEE700BF38
:10A83000546D72205376630010B584B0A8B146F20F
:10A840003004C2F2000484462068C0B10529CDE975
:10A850000012CDF808C015DCFFF738FD014620686E
:10A86000022916D1069A694615E04FF0500080F390
:10A870001188BFF36F8FBFF34F8F00BFFEE700203B
:10A8800004B010BD69461A460023FFF7ADF804B0C6
:10A8900010BD694600220023FEF7D4FF04B010BDAE
:10A8A00003B401984100009850EAC12018BF042069
:10A8B0004A0D18BF40F0010040F2FF72B2EB515F49
:10A8C00008BF40F00200012808BF052002B0704711
:10A8D0004100080218BF04200A0E18BF40F0010012
:10A8E0004FF07F4232EA010108BF40F00200012828
:10A8F00008BF05207047000010B54FF00E402DED49
:10A90000028BB0EE408A18EE104A00EB4400B0F122
:10A91000506F4AD84FF0FC40B0EB440F22D2B0EE5B
:10A92000C80AF7EE000A30EEC00AF6EE000A60EE42
:10A93000208A18EE900A00F03BFF01EE100A14F096
:10A94000004F1DBFDFED2D0A9FED2D0AB1EE411A1C
:10A95000DFED2C0A08BF9FED2C0AF8EE001A21EE5D
:10A96000218A05E0DFED290A68EE088AB0EE600A68
:10A970009FED271ADFED271A30EE080A48EE811AFC
:10A980009FED251A08EEA11ADFED241A48EE811A70
:10A990009FED231A08EEA11A68EE281ABDEC028B6F
:10A9A00001EE810A30EE200A10BD4FF0E440B0EB1A
:10A9B000440F0CD918EE100AFFF78AFF042808BFCD
:10A9C00000F030FEB0EE480ABDEC028B10BD4FF037
:10A9D0007F40B0EB440F07D2B0EE480ABDEC028BCB
:10A9E000BDE8104000F010BE0120F5F731FDBDECD0
:10A9F000028BBDE8104000F00DBE00000000C9BF92
:10AA000022AAFDB90000C93F22AAFD3900000000BA
:10AA100024FE1C3DC78AD83C1E67383D1B93993DD8
:10AA2000AFAA2A3E0000000070B59B482DED020B36
:10AA30002DED068B079D25F00044A04218DC9748B9
:10AA4000844202DC0AD1069840B19DED060BBDECB4
:10AA5000068B02B0BDE8704000F0A2BD002DCCBF57
:10AA60009FED8F0B9FED900BBDEC068B02B070BD80
:10AA70008F48A04215DD8F48A042D8BF4FF0FF3469
:10AA800058DD9DED060B51EC100BFFF709FF042874
:10AA900008BF00F0A9FD9DED060BBDEC068B02B0D2
:10AAA00070BD9DED060B51EC100B00F075FECDE96D
:10AAB000060181489FED828BA0423CDD8248A04286
:10AAC0001FDD00249FED82AB9DED060B53EC1A2B8E
:10AAD00051EC100B00F0CAFE9DED060B41EC190B7A
:10AAE00053EC1A2B51EC100B01F0C2F953EC182B5C
:10AAF00001F03CFC53EC192B00F06CFFCDE9060192
:10AB000049E09DED060B012453EC182B51EC100B82
:10AB100000F0ACFE9DED060B41EC190B53EC182B2D
:10AB200051EC100B01F022FC53EC192B00F052FFFA
:10AB3000CDE906012FE06848A0421FDD02249FED09
:10AB4000689B9DED060B53EC192B51EC100B01F09B
:10AB50008FF953EC182B00F089FE9DED060B41ECAC
:10AB6000180B53EC192B51EC100B01F0FFFB53ECBD
:10AB7000182B00F02FFFCDE906010CE09DED060B30
:10AB8000032453EC102B9FED580B51EC100B00F0ED
:10AB900021FFCDE906019DED060B53EC102B51EC86
:10ABA000100B01F065F941EC180B53EC182B01F078
:10ABB0005FF941EC190B4E480621B0EE490AF0EE60
:10ABC000690A784400F070FC53EC182B51EC100B20
:10ABD00001F04EF941EC180B4648B0EE490AF0EE90
:10ABE000690A0521784400F05FFC53EC192B51EC05
:10ABF000100B01F03DF941EC100B51EC180B53EC2C
:10AC0000102B002C0EDA00F031FE9DED061B53ECEC
:10AC1000112B01F02DF99DED061B53EC112B01F0CA
:10AC2000CDFA35E000F022FE9DED061B53EC112B12
:10AC300001F01EF941EC100B2F48784400EBC400E2
:10AC400090ED001B51EC100B53EC112B01F08EFB1F
:10AC50009DED061B53EC112B01F088FB41EC100B12
:10AC60002648784400EBC40090ED001B51EC100B1B
:10AC700053EC112B01F0A2FA41EC100B002DA2BFF6
:10AC8000BDEC068B02B070BD51EC100B00F0AFFDB7
:10AC900041EC100B01E70000000010440000F07FC1
:10ACA000182D4454FB21F93F182D4454FB21F9BFC2
:10ACB0000000DC3F0000203E0000F33F00000000E9
:10ACC000000000000000F03F0000E63F0000000030
:10ACD0000000000000000040008003400000000071
:10ACE000000000000000F83F000000000000F0BF7E
:10ACF000AA1B0000601B0000EA1A0000A21A000054
:10AD000070B56F4E2DED040B2DED048B82B0DDF888
:10AD100024C0DDE907235C422CF000411C4341EADA
:10AD2000D474069D22F00040B44205D86C422C43F6
:10AD300040EAD474B4420BD99DED081B9DED060B7F
:10AD400002B0BDEC048B04B0BDE8704000F032BC32
:10AD5000ACF14054A4F17F641C430BD0022404EAFC
:10AD6000AC7444EAD27405439FED578B9FED582B8A
:10AD700007D015E09DED060B51EC100B00F004FD23
:10AD800042E0002C11BF012C9DED060B02B0BDEC82
:10AD9000048B04BF04B070BD022C38D0032C3BD010
:10ADA0000B439FED4D1B9FED4E0B0AD0B14218D1C6
:10ADB000B04209D121F0804120F0804009910790F4
:10ADC0000FE0002A15DA10E0474B7B44002C08BF47
:10ADD00093ED000B0DD0012C10D0022C17D0032CBA
:10ADE0001AD0B0421DD1002A03DAB0EE410AF0EECB
:10ADF000610A02B0BDEC048B04B070BD93ED000B92
:10AE000051EC100B00F0F3FC41EC100BF1E7B0EE4D
:10AE1000480AF0EE680AECE7B0EE420AF0EE620A89
:10AE2000E7E7401A00159FED329B3C28C8BF8DED27
:10AE3000000B17DCBCF1000FBCBF10F13C0F8DED17
:10AE4000009B0FDB9DED080B53EC102B9DED060BCB
:10AE500051EC100B00F0BEFD00F09EFC00F094FCE5
:10AE6000CDE90001B4B1012C10D0022C9FED220BD2
:10AE700053EC102B9DED000B51EC100B19D001F091
:10AE800075FA53EC182B01F071FABDE7019880F0C8
:10AE9000004001909DED000B53EC192B51EC100B71
:10AEA00000F0F2FE04BF0220F5F7D2FA9DED000B90
:10AEB0009FE701F05BFA53EC182B01F07FF9A3E751
:10AEC0000000F07F00000000182D4454FB210940D1
:10AED000182D4454FB2109C0182D4454FB21F9BFFF
:10AEE000182D4454FB21F93FD21900000000000046
:10AEF0000000000000000000075C143326A6A13CFF
:10AF000070B54FF068422DED048BF0EE408A18EEDC
:10AF1000900AB0EE608A18EE101A02EB4003B3F10B
:10AF2000654F3CBF02EB4102B2F1654F7DD200BFDD
:10AF3000C0F3C753C1F3C7529A1A1B2A09DD10F098
:10AF4000004F14BF9FED830A9FED830ABDEC048B75
:10AF500070BD12F11A0F36DA11F0004F09D010F05F
:10AF6000004F0CBF9FED7D0A9FED7D0ABDEC048B69
:10AF700070BD88EE889A19EE100AFFF7A9FC042824
:10AF800008BF00F04FFB18EE900AFFF7A1FC054642
:10AF900018EE100AFFF79CFC044619EE100AFFF7A2
:10AFA00097FC042D18BF052D08D1042C18BF052CC3
:10AFB00004D1002804BF0220F5F74AFAB0EE490A8E
:10AFC000BDEC048B70BD4200B2EB410F3AD910F0DA
:10AFD000004F19BFDFED630A9FED630ADFED630ADF
:10AFE0009FED630AB0EE481A0A46B1EE688A80F017
:10AFF0000041F0EE418A10460A1A5200B2F1807FF9
:10B0000034D2484010F0004FDFED5A1A9FED5A2A13
:10B010001DBFBEEE001A70EEE10A30EE420AB6EE37
:10B02000001A08BF70EEA10A00E040E008BF30EE51
:10B03000020AB0EE682A01EE482A08EE818AC2EEC2
:10B04000081A15E011F0004F04BF9FED4C0AF0EE16
:10B05000400AD1D010F0004F19BFDFED490A9FED33
:10B06000490ADFED490A9FED490AC5E7C8EE881A8B
:10B0700021EEA11A9FED462ADFED462A41EE022A73
:10B080009FED452A01EE222ADFED442A41EE022AF5
:10B090009FED432ABDEC048B01EE222A21EE811A9A
:10B0A00001EE020A30EE210A30EE200A70BD4FF0A8
:10B0B0007F42B2EB400F28BFB2EB410F09D2F0EE56
:10B0C000480AB0EE680ABDEC048BBDE8704000F0A1
:10B0D0009EBA40EA01035B0008BF41F0FF410BD07C
:10B0E000B2EB400F08BFB2EB410F08D120F0804017
:10B0F00008EE900A21F0804108EE101A18E7B2EB32
:10B10000400F12BF5FEA410340F0FF4001F00041F1
:10B110003FF40EAFB2EB410F12BF5FEA400200F006
:10B12000004041F0FF413FF403AF4A0092EA400380
:10B130003FF5FEAE002AACBF9FED1A0A9FED1A0A3A
:10B1400068EE808A28EE008A18EE900A18EE101A2F
:10B15000EEE60000DB0FC9BFDB0FC93FDB0F494044
:10B16000DB0F49C00000C9BF22AAFDB90000C93FDA
:10B1700022AAFD390060ED3EC30ACE370000000070
:10B18000000049C022AA7DBA0000494022AA7D3AA7
:10B190002DAD65BD8FB8D53D0FB511BE61C84C3E14
:10B1A000A8AAAABE0000804F0000802F10B52DED88
:10B1B000040B86B09DED060B10EE100A10EE901AEF
:10B1C0008DED000B002818BF0120084320F000403F
:10B1D000C0F17F6000F1E040C00F21D19DED080B70
:10B1E00010EE101A10EE900A8DED000B002918BF1A
:10B1F0000121084320F00040C0F17F6000F1E040F1
:10B20000C00F0DD129490798B1EB400F04BF069834
:10B21000002842D00998400004BF089800283CD07C
:10B220009DED080B53EC102B9DED060B51EC100B14
:10B2300000F016FFCDE902019DED020B40F2FF7117
:10B2400010EE900A8DED000B31EA105021D00798D6
:10B25000039900F0004001F00041884219D09DEDB3
:10B26000080B8DED040B9DED020B8DED000B10EE28
:10B27000900A059961F31E0005909DED041B9DED5C
:10B28000020B51EC110B53EC102B00F097FFCDE9A2
:10B2900002019DED020B0AB010BD0120F5F7D8F8B0
:10B2A0000AB0BDE8104000F08FB900000000E0FFD8
:10B2B00000B52DED048BB0EE409AF0EE609A83B0AD
:10B2C00051EC190B00F086FF41EC180B18EE100A38
:10B2D00018EE901A8DED008B002818BF012008434E
:10B2E00020F00040C0F17F6000F1E040C00F14D0BA
:10B2F00019EE101A19EE900A8DED009B002918BF67
:10B300000121084320F00040C0F17F6000F1E040DF
:10B31000C00F04BF0120F5F79BF8B0EE480A03B058
:10B32000F0EE680ABDEC048B00BD000000B510EE25
:10B33000101A2DED028B81B04D4A6846B2EB410FD9
:10B340003CD94FF0E640B0EB410F94BF00204FF0E6
:10B35000FF3000900098B0EE408A00285FDB28EEB6
:10B36000080ADFED440A9FED441A00EE201ADFEDD3
:10B37000430A40EE010A9FED421A00EE201ADFED6B
:10B38000410A10F0010F40EE010A9FED3F1A00EE56
:10B39000201A61EE000AB0EE480A08EE200A02BF49
:10B3A00001B0BDEC028B00BDBFEE001A01B0C1EED2
:10B3B000000ABDEC028BB0EE600A00BD334B21F0F9
:10B3C0000042934228D911F0004FDFED310A20EE00
:10B3D000201ADFED300A19BF31EE601A71EE200A33
:10B3E00031EE201A71EE600ABDEEE01A11EE100A7D
:10B3F0009FED291A00F0030000EEC10A9FED271A05
:10B40000009000EEC10A9FED261A00EEC10A9FEDE2
:10B41000251A00EEC10A9DE700F00CF99AE718EE34
:10B42000100A4000B0F17F4F0DD218EE100AFFF75E
:10B430004FFA042808BF00F0F5F8B0EE480A01B052
:10B44000BDEC028B00BD09D10120F5F701F801B078
:10B45000BDEC028B5DF804EB00F0DCB801B0B0EE9F
:10B46000480ABDEC028B5DF804EB00F0CDB800009B
:10B47000B61F927EBCE9223C0B6D063B8A76CE3C21
:10B48000ACB5593D35A1083E29AAAA3E490E494608
:10B4900083F9223F0000004B0000C93F00A0FD39A6
:10B4A0000020A2331A61342C70B504462DED028BB6
:10B4B0004D1E00EBC500B0EE408AF0EE608A90EDC4
:10B4C000000B35F0060017D053EC182B51EC100B85
:10B4D00000F0CEFC41EC100B6D1E04EBC50090EDAE
:10B4E000001B51EC100B53EC112B00F0BFF941EC99
:10B4F000100B35F00600E7D1022D36D0042D1CD0FC
:10B50000062D1CBFBDEC028B70BD53EC182B51EC0B
:10B51000100B00F0ADFC94ED0A1B53EC112B00F066
:10B52000A5F953EC182B00F0A3FC94ED081B53EC89
:10B53000112B00F09BF941EC100B53EC182B51EC44
:10B54000100B00F095FC94ED061B53EC112B00F052
:10B550008DF953EC182B00F08BFC94ED040B53EC9D
:10B56000102B00F083F941EC100B53EC182B51EC2D
:10B57000100B00F07DFC94ED021B53EC112B00F03E
:10B5800075F953EC182B00F073FC94ED001B53EC91
:10B59000112B00F06BF9BDEC028B41EC100B70BD70
:10B5A00010B553EC102B51EC100B00F05FF941EC8F
:10B5B000100B10BD10B553EC112B51EC100B00F01B
:10B5C00055F941EC100B10BD9FED050B10B553EC78
:10B5D000102B51EC100B00F0FDF941EC100B10BDDD
:10B5E00000000000000000009FED050B10B553ECBB
:10B5F000102B51EC100B00F03BFC41EC100B10BD7C
:10B60000000000000000001030EE000A704730EE2D
:10B61000200A7047DFED020A80EEA00A70470000A2
:10B62000000000009FED020A20EE000A70470000B3
:10B63000000000102DE9F0014FF07F42B2EB410F06
:10B640009FBF4FF0FF310160BDE8F00170474FF040
:10B65000004242EA0123C1F3C752783A551112F071
:10B660001F0C434CCCF120067C44C1F3C752A2F11D
:10B6700078024FEA621204EB820254F8254008BFB8
:10B68000D2E9015612D0556804FA0CF425FA06F7EF
:10B690003C43976805FA0CF527FA06F8D26807FAD2
:10B6A0000CFCF24045EA08054CEA0206A4FB034CF8
:10B6B000A5FB0352A6FB03631D449D4234BF012634
:10B6C00000261319334416B1934202D903E0934282
:10B6D00001D2012200E00022624402F1200C920615
:10B6E000DC0C42EA443200EE102A5B03DFED210A53
:10B6F000F8EEC01A00EE103A4FEA9C1C11F0004F11
:10B70000B8EE400AC0F800C020EE201A00EE105A31
:10B71000DFED190AB8EE400A20EE200A71EE810A28
:10B7200070EE800A10EE902A02F500626FF30B02B1
:10B7300000EE902A70EEE11A31EEC11ADFED101A18
:10B7400030EE411A9FED0D0A20EE800A01EE210A2B
:10B750009FED0C1A00EE810A04BFBDE8F0017047AE
:10B76000CCF180510160BDE8F001B1EE400A7047B4
:10B770003C110000000000360000802C22AAFD29A8
:10B78000DB0FC92F0000C92F10B541EC100BFFF7DC
:10B790004BF951EC100B10BD82B0CDE9000121F046
:10B7A000004001909DED000B02B051EC100B704772
:10B7B00010B500EE100A2DED028BB1EEC08A18EE26
:10B7C000100A20F00040C0F1FF40C00F0AD010EE78
:10B7D000100A20F00040C0F1FF40C00F04BF01205C
:10B7E000F4F736FE18EE100ABDEC028B10BD81F0A6
:10B7F0000041704780F00040704721F000417047E1
:10B8000020F000407047000021F0004201F00043AA
:10B81000A2F16052B2F5801F28BFD2F17F6C0BD924
:10B820005FEA001C43EAC20242EB507018BF704747
:10B8300028BF20F001007047B2F5801FBCBF18463A
:10B8400070474FEA410C1CF5001F02D2084600F079
:10B8500053BF70B500F0B6FB00000089FFF7F6BFDC
:10B860004FF00040A0F580007047000010B591EA4D
:10B87000030F48BF83F0004300F18085841A71EB09
:10B88000030C05D2121943EB0C03001B61EB0C01F6
:10B890004FEA1154A4EB135CDFF81CE11EEA430FDE
:10B8A00018BF9EEA445F00F0748021EA045123EA45
:10B8B0000E0343F48013DCF1200E32D322FA0CFE87
:10B8C00010EB0E0023FA0CFE41EB0E01CCF1200E22
:10B8D00003FA0EFE10EB0E00CCF1200E51F1000128
:10B8E000B1F5801F32D201EB045112FA0EF2BDE81D
:10B8F000104058BF7047401C38BF5FEA420218BF73
:10B900007047002814BF20F0010041F100014FEA08
:10B91000410313F5001F38BF7047A1F1C04100F08B
:10B9200047BC012A43EB0302ACF1200CDCF11F0EF3
:10B9300032BF4FF0000E23FA0CF310EB030041EB83
:10B940000451B4EB115FD0D0A1EB045101F580118B
:10B95000490801EB04515FEA30000ED350F10000BA
:10B9600038BF12FA0EFE08D1BDE81040C9E7401CEE
:10B9700038BF5FEA4202CAD1C3E7BDE810404FEAD0
:10B98000410313F5001F38BF7047A1F1C04100F01B
:10B990000FBC9EEA445F08D011EA5E0FBDE810407C
:10B9A00004BF01F0004100207047BDE8104070B5B1
:10B9B00000F008FB64FBBE3E0000E0FF491058BFEA
:10B9C000C1F140415B1058BFC3F140438B42EFF3DC
:10B9D000008070472DE9C04130B4DFF8A4C23CEAD2
:10B9E000111418BF3CEA131400F0ED801CEA111486
:10B9F00081EA030544EAD57418BF1CEA131500F068
:10BA0000C880A4EB050404F17F7404F500344FF002
:10BA1000004545EAC12145EAC32341EA505143EAC2
:10BA200052534FEAC0204FEAC222994208BF9042C7
:10BA300000F09D804FEA13650FF24416765D4FEAE1
:10BA4000134506FB05F7C7F1807706FB07F74FEABA
:10BA5000D737A7FB03687642A7FB06CEC8F5803828
:10BA600038BFA8F1010807FB08E6A6FB028C4FF0DF
:10BA7000000EE6FB03CEDCF1000CCEF1004E38BF29
:10BA8000AEF1010EA6FB0C584FF00007E6FB0E8747
:10BA9000A1FB08C6A0FB07CE16EB0E064FF0000573
:10BAA00045F10005E1FB076515F1E04E7EBFA4F509
:10BAB00080345FEA46066D4116F1800745F10005C6
:10BAC0004FEA172747EA05674FEA15254FEA06664A
:10BAD000A6F1DE46B6F1805F20D9384605EBC47189
:10BAE00024F0010C01EB0C11BCF1FE6F02D8F0BC8C
:10BAF000BDE8008124425CBF01F5801E9EEAC47F40
:10BB000002D4F0BCBDE80081244200F13980A1F1EB
:10BB1000C041F0BCBDE8004100F04ABB4FEAD02074
:10BB200040EA41504FEAD1214FEAD22242EA435241
:10BB30004FEAD323A7FB028607FB036605FB0266D9
:10BB40001EEA0E0F58BFA6EB0056B6EB00564FEAA2
:10BB5000520E4EEAC37E18EB0E0E56EB530EBCD5BA
:10BB600018EB02085E417F1C55F10005B5E74FF464
:10BB700080154FF000074FF000064FF00008ACE7CB
:10BB800001F1C04101F000414FF00000F0BCBDE800
:10BB900000810CEA131511EA0C1F00D00CE013EA27
:10BBA0000C1F00F026804FF0000081EA030101F035
:10BBB0000041F0BCBDE80081F0BCBDE8004181EA75
:10BBC000030100F0F5BAF0BCBDE8004170B500F02B
:10BBD000F9F900BF097EFC3E00F007B84FF0000005
:10BBE00081EA030101F00041704781EA030100F09E
:10BBF000DFBAF0BCBDE8004122494FF000007047B9
:10BC0000FFFDFBF9F7F5F4F2F0EEEDEBE9E8E6E421
:10BC1000E3E1E0DEDDDBDAD8D7D5D4D3D1D0CFCDA8
:10BC2000CCCBCAC8C7C6C5C4C2C1C0BFBEBDBCBBE1
:10BC3000BAB9B8B7B6B5B4B3B2B1B0AFAEADACABDC
:10BC4000AAA9A8A8A7A6A5A4A3A3A2A1A09F9F9EB6
:10BC50009D9C9C9B9A999998979796959594939368
:10BC6000929191908F8F8E8E8D8C8C8B8B8A8989FF
:10BC70008888878786858584848383828281818082
:10BC80000000FF070000F87F51EA030C17D41CF5F1
:10BC9000801F58BFBCF5801F00F10680994218BF75
:10BCA000704708BF9042704707D711F5801F58BFF3
:10BCB00013F5801F19D499427047894270471CF5CB
:10BCC000801F08D5BCF5801FF7D58B4218BF704781
:10BCD00008BF824270474FF4001C1CEB410F38BF75
:10BCE0001CEB430F01D28B42704770B500F06AF92C
:10BCF000922449004FF000514FF08053FFF75EBE91
:10BD00004FEA1153A3F58063D3F11E03A8BFD3F10B
:10BD1000200C08DB4FF0004242EAC12252EA5052A6
:10BD200032FA03F0704709420BD4102BC4BF002035
:10BD3000704703F5787CBCF1FF3F05D04FF0FF3032
:10BD400070474FF00000704770B500F03BF900BF3E
:10BD50004992248000207047F0E7B0FA80F310FA8F
:10BD600003F10AD0C3F11D0303F580634FEA0352C8
:10BD70004FEA415002EBD12170474FF0000070476D
:10BD800051EA030C17D41CF5801F58BFBCF5801F67
:10BD900000F10680994218BF704708BF9042704773
:10BDA00007D711F5801F58BF13F5801F19D499428A
:10BDB0007047894270471CF5801F08D5BCF5801F6D
:10BDC000F7D58B4218BF704708BF824270474FF4C7
:10BDD000001C1CEB410F38BF1CEB430F01D28B4200
:10BDE000704770B500F0EEF8922449004FF0805192
:10BDF0004FF00053FFF7E2BD51EA030C17D41CF5D6
:10BE0000801F58BFBCF5801F00F10680994218BF03
:10BE1000704708BF9042704707D711F5801F58BF81
:10BE200013F5801F19D499427047894270471CF559
:10BE3000801F08D5BCF5801FF7D58B4218BF70470F
:10BE400008BF824270474FF4001C1CEB410F38BF03
:10BE50001CEB430F01D28B42704770B500F0B2F873
:10BE6000922449004FF000514FF08053FFF7A6BDD8
:10BE700070B5DFF848C11CEA111E1EBF1CEA13157D
:10BE80009EEA0C0F95EA0C0F00F06F8081EA030424
:10BE90004EEAD47EAE4421EA4C1123EA4C1341F41D
:10BEA000801143F48013AEF17F7EA1FB024CA0FB16
:10BEB0000365361955EB0C05A1FB034C4CF100034F
:10BEC000A0FB021C16EB0C06654153F1000309426E
:10BED00018BF46F0010613F4007F0BD14FEA03317F
:10BEE0004FEA053041EA155140EA165034036FF02D
:10BEF00003020AE04FEAC3214FEAC52041EA555147
:10BF000040EA5650F4026FF0020202EB2E4201EBBF
:10BF1000025585EACE710AD05FEA440C18BF24F0BE
:10BF2000004450F1000041F1000120EAD47040F2D9
:10BF3000FE7C624500D270BDA84214BF4FF0804421
:10BF40004FF04044002E08BF0024BEF1806FA8BF10
:10BF5000A1F1C041BDE8704080F22A8101F1C041E9
:10BF600001F000414FF0000070470CEA13159EEA03
:10BF70000C0F18BF95EA0C0F06D081EA030E4FF0A4
:10BF800000000EF0004170BD00F01CF88900013E79
:10BF900000F007B800F009B84FEA430C5FEA5C5CB8
:10BFA00008D081EA030100F003B94FEA410C5FEACF
:10BFB0005C5CF6D102494FF0000070470000FF07BB
:10BFC0000000F87F0EF1020E2EF0030E5EF8046BF7
:10BFD000364205D4012A43EB030515F5001F12D89C
:10BFE000012841EB010C1CF5001F0CD80ED14FEAC3
:10BFF000D17C0CEB4C0C0CF1020C15F5001F08BFAA
:10C000004CEBD37C04E04FF0080C01E04FEAD37C0A
:10C010000CEB4C0526FA05F606F00706B6F1040C03
:10C0200006D20EEB860CBDE870404CF0010C604768
:10C03000DFE80CF0090B02024FF00041A1F50021EE
:10C040004FF0000070BD19461046012851EB010465
:10C0500018BFD4F5001484BF002001F0004170BD6A
:10C0600070B5DFF844C13CEA111418BF3CEA13155F
:10C0700000F08F8011F1004F0CEA11141CEA131527
:10C0800068BF45F0050518BF11EA0C1F00F0798064
:10C0900021EA4C1123EA4C1341F4801143F480133C
:10C0A0002E46A5F58035AC423DDDA4F58036801ADC
:10C0B000994109D54042C1F1000134BFB1F10101FC
:10C0C000B1F1000185F0010511F4F01F08D011F461
:10C0D000801FE8D1400041EB0101A4F58034F6E770
:10C0E00021F00041B1FA81F6202E04BFB0FA80FEA3
:10C0F0000EF12006A6F10B06A4EB0644B6F1200EC5
:10C100000CD2C6F1200E01FA06F120FA0EF641EA31
:10C110000601CEF1200600FA06F003E000FA0EF167
:10C120004FF00000BFE750EA410E23D04FEA244E03
:10C13000BEEB254F0FDB994208BF904204D00AD3D3
:10C14000520043EB0303B0E74FEA1646B6EB144F39
:10C1500008BF85F00105B4F5803401EB041181EAD4
:10C16000C57100DB70BD01F1C04101F000414FF02D
:10C17000000070BD4FEA45714FF0000001F0004132
:10C1800070BD1CEA131F09D04FF0000001F0004100
:10C1900070BDFFF717FF00BFEDFFFF3EBDE8704029
:10C1A00002494FF0000070470000FF070000F87FD1
:10C1B0000808A0F500114FEA3101704710B591EA67
:10C1C000030F81F000413FF559AB83F0004300F0CD
:10C1D000D5B800002DE9F04101F5801CBCF5001F29
:10C1E000C0F2A9804FEA115C21EA0C5141F48011A0
:10C1F0000CF1FD0C5FEA5C0C0CF5C07C01D3400037
:10C200004941890241EA905187022EA48E0EA45D15
:10C210000A0C04FB04F602FB06F6C6F14046A4FB3A
:10C220000662F60D46EA422606FB06F4A4FB01234D
:10C230005242C3F1404338BF5B1EA6FB02420024BA
:10C24000E6FB0324D20B42EA4446A6FB0623A1FBED
:10C2500002E2A3FB07E4E3FB61426442C2F1404E09
:10C2600038BFAEF1010EA6FB04234FF00002E6FB3F
:10C270000E32A2FB03463400E2FB6264A1FB06E639
:10C28000A4FB07E8E4FB61687642C8F1405838BF78
:10C29000A8F10108A2FB06E4A3FB08E5E2FB685451
:10C2A000A1FB05E6A7FB04E8E1FB648618F1200585
:10C2B00056F10006A80940EA8660B109A8F11B08FA
:10C2C00008F03F08B8F10A0F1CD901EB0C51BDE88A
:10C2D000F08100BFFCF5EEE8E2DDD8D3CFCBC7C3D9
:10C2E000C0BDB9B6B4B1AEACA9A7A5A3A19F9D9B93
:10C2F0009A9896959392908F8D8C8B898887868556
:10C3000084838281A0FB006800FB01F208EB4208F5
:10C31000B8EB872807D5341858EB0104D5D5401C55
:10C3200051F10001D1E7341A78EB0104CDD4401E5D
:10C3300071F10001C9E75FEA4C0C5FEA9C5C0DD12A
:10C3400005D301F000414FF00000BDE8F081BDE8E9
:10C35000F04170B5FFF736FE6DDBFFBEBDE8F04182
:10C3600001494FF0000070470000F87F10B591EAD6
:10C37000030F48BF83F000433FF580AA841A71EB96
:10C38000030C07D28CF0004C121943EB0C03001B7A
:10C3900061EB0C014FEA1154A4EB135CDFF8A4E14C
:10C3A0001EEA430F18BF9EEA445F00F0B48021EA02
:10C3B000045123EA6E035242C3EB6E0338BF5B1E87
:10C3C000DCF1200E25D322FA0CFE10EB0E0043FA0E
:10C3D0000CFE41EB0E01CCF1200E03FA0EFE10EB29
:10C3E0000E00CCF1200E51F1000129D401EB0451D3
:10C3F00012FA0EF2BDE8104058BF7047401C1CBF37
:10C40000B2F1004F704700280CBF491C20F001001A
:10C41000704712EB020E43EB030218BF4FF0010E00
:10C420004EEA4202ACF1200CDCF11E0E56D943FA62
:10C430000CFE10EB0E00CCF11E0E51F1FF31D5D5E4
:10C440000EF1010E12FA0EFE404141EB010101EB2B
:10C45000445C5FEA5C5C10D901EB045110EBDE70C8
:10C4600038BFBEF1004FBDE8104018BF704700282C
:10C470000CBF491C20F00100704734D24FEAD42C85
:10C4800024F4006411F500111BD0B1FA81F20B3ACB
:10C49000A41AA41ED2F12003914030FA03F31943E9
:10C4A000904001EBCC7101EB0451002CBDE8104031
:10C4B000A8BF704701F1C04101F000414FF00000FA
:10C4C0007047B0FA80F310FA03F102D1BDE81040D2
:10C4D0007047E41A173C4805C90AE2E701EB04512A
:10C4E000BDE81040704749104FEA300001EB04519D
:10C4F000BDE8104002E04FF0000170474A0008BF5D
:10C500000042F8D0B2F5001F28BF704701F000418B
:10C510004FF0000070479EEA445F07D011EA5E0FBB
:10C52000BDE8104004BF002100207047BDE8104066
:10C5300070B5FFF747FD00BF40DFF63E104683F0C1
:10C54000004170470000E0FF43004FEAD30C4FEA80
:10C550003C0C43401FBF40070CF1605113F0FE4FED
:10C5600070471CF0006F03D10CF0004100207047B1
:10C570000CF0004343EA507040EACC0010B500F0E4
:10C5800068F800BF000000924FEA0001FFF710BEFC
:10C590004FF00041A1F500214FF00000704710B5A9
:10C5A000FFF772FB0CBF0120002010BD10B5FFF794
:10C5B0006BFB14BF0120002010BD10B5FFF7E0FB9E
:10C5C0008CBF0120002010BD10B5FFF7D9FB2CBF98
:10C5D0000120002010BD10B5FFF70EFC94BF012014
:10C5E000002010BD10B5FFF707FC34BF012000206C
:10C5F00010BD4FF07E5209E011F0004204D54042D8
:10C60000C1F1000138BF491E42F07E5202F1706252
:10C610000B0012BF20235FEA00017047B1FA81FCD2
:10C6200001FA0CF1A3EB0C0320FA03FC41EA0C0124
:10C6300002EBC352C3F1200310FA03FC5CEA416C25
:10C6400042EB112018BF5FF0806C28BF20F0010082
:10C6500070470EF1020E2EF0030E5EF8044B2442DA
:10C6600004D44FEA4102B2F17F4F11D84FEA4003A0
:10C67000B3F17F4F0CD80ED14FEAD07C0CEB4C0CB1
:10C680000CF1020CB2F17F4F08BF4CEBD17C04E0FF
:10C690004FF0080C01E04FEAD17C0CEB4C0324FA7C
:10C6A00003F404F00704B4F1040C06D20EEB840C7E
:10C6B000BDE810404CF0010C6047DFE80CF00708C3
:10C6C00002024FF00040A0F5800010BD0846420075
:10C6D00018BFD2F1807288BF00F0004010BDF1EEAB
:10C6E000100A4FF6FF71C0F2C03120EA010040F09D
:10C6F0004070E1EE100A7047FF2141EAD050C005BA
:10C7000070470000000000004FBB610567ACDD3FD3
:10C71000182D4454FB21E93F9BF681D20B73EF3F68
:10C72000182D4454FB21F93FE2652F227F2B7A3CE0
:10C73000075C143326A6813CBDCBF07A8807703C99
:10C74000075C143326A6913CC4EB98999999C9BF0C
:10C75000711623FEC671BCBF6D9A74AFF2B0B3BF41
:10C760009AFDDE522DDEADBF2F6C6A2C44B4A2BF01
:10C770000D5555555555D53FFF8300922449C23F6D
:10C780006E204CC5CD45B73F513DD0A0660DB13FA1
:10C79000EB0D76244B7BA93F11DA22E33AAD903FB3
:10C7A0000000000000000000000000006E83F9A2FD
:10C7B0002915444ED15727FCC0DD34F5999562DB2D
:10C7C0004190433CAB6351FE0000000000000000BC
:10C7D0000102030406070809000000000102030427
:10C7E00001000000000002401000000000000240B4
:10C7F0000100000000040240100000000008024098
:10C80000200000000008024000040000001C02405C
:10C8100000080000001C024000100000001C024044
:10C8200063C90008000000000000000000000000D4
:10C8300000000000000400001800000000000000DC
:10C840000000000074C900080000000000000000A3
:10C8500000000000000000000008000018000000B8
:10C8600000000000000000005FC900080000000098
:10C8700000000000000000000000000000080000B0
:10C880001800000000000000000000006DC9000852
:10C890000000000000000000000000000000000098
:10C8A000000400001800000000000000000000006C
:10C8B0007CC900080000000000000000000000002B
:10C8C0000000000000040000300000000000000034
:10C8D000000000005CC9000800000000000000002B
:10C8E0000000000000000000000800001800000028
:10C8F000000000000000000086C9000800000000E1
:10C900000000000000000000000000000004000023
:10C9100018000000000000000000000080E9334320
:10C9200020949643002CF14209B8964350C9000860
:10C9300000000000000000000000000000000000F7
:10C9400000020000180000000000000000000000CD
:10C9500064656661756C745461736B007263006327
:10C960006D6400617474695F657374690067696DF3
:10C9700062616C0063686173736973005461736B07
:10C980005F496E69740073686F6F7400B0C9000806
:10C990000000002008010000C4010008B8CA000817
:10C9A00008010020388F0000E001000800000000AE
:10C9B0000024F400022B073D0000803F0000003FF0
:10C9C000CDCCCC3D000000000000803F0000803F47
:10C9D000000080BF000080BFCDCC4C3E3D0A573EDA
:10C9E000CDCCCC3D000000000000803F0000F041B5
:10C9F000000080BF0000B443CDCC4C3E0000803E20
:10CA0000CDCCCC3D000000000000803F0000803F06
:10CA1000000080BF000080BF000001020100000094
:10CA200000000202010000000000030201000000FB
:10CA300000000402010000000000050202000000E6
:10CA400000000602020000000000070202000000D1
:10CA500000000802020000000000000000000000CA
:10CA600000000000000000000000000000000000C6
:10CA700000000000000000000000000000000000B6
:10CA800000000000000000000000803F0000C03FE8
:10CA900000000000000000000000803F0000803F18
:10CAA0000000000000000000010000001000000075
:08CAB000AAAAAAAA00000000D6
:040000050800018965
:00000001FF
